:020000040800F2
:100000005838002063050008AD040008650A02089E
:10001000B1040008B3040008B504000800000000A3
:10002000000000000000000000000000B70400080D
:10003000B904000800000000BB040008BD0400086B
:10004000BF040008C1040008C3040008C504000878
:10005000C7040008C9040008CB040008CD04000848
:10006000CF040008D1040008D3040008D504000818
:10007000D7040008D9040008DB040008DD040008E8
:10008000DF040008E1040008E3040008E5040008B8
:10009000E7040008E9040008EB040008ED04000888
:1000A000EF040008F1040008F3040008F504000858
:1000B000F7040008F9040008FB040008FD04000828
:1000C000FF040008010500080305000805050008F5
:1000D00007050008090500080B0500080D050008C4
:1000E0000F05000811050008130500081505000894
:1000F00017050008190500081B0500081D05000864
:100100001F05000821050008230500082505000833
:1001100027050008290500082B0500082D05000803
:100120002F050008310500083305000835050008D3
:1001300037050008390500083B0500083D050008A3
:100140003F05000841050008430500084505000873
:1001500047050008490500084B0500084D05000843
:100160004F05000851050008530500085505000813
:1001700057050008590500085B0500085D050008E3
:080180005F050008610500089D
:10020000DECEA5ED02003078463430370000000025
:1002100000000000000044433231365F3134313099
:100220000000000000004170706C69636174696FC8
:100230006E00000000000000000000000000000050
:10024000000000000000041ABB00DAF7DECEA5EDC6
:100250000200307846343037000000000000000013
:10026000000053504C6174436F6E74726F6C6C6518
:1002700072004170706C69636174696F6E00000098
:10028000000000000000000000000000000000006E
:0802900000000000FE00DAF797
:1002980001000208100000002500020818000000F4
:1002A800790102081700000009060208170000007B
:1002B8000509020803000000410F020806000000BB
:1002C8000114020809000000A11C02080200000035
:1002D800AD1D0208110000003122020810000000C4
:1002E800ED230208FF000000D12B02080C000000DB
:1002F800D93002080000000015330208050000008C
:1003080051590208120000004D5D02080A00000061
:10031800256302080A000000E56D020814000000C9
:100328003D78020808000000F57F02080700000079
:100338009D86020810000000AD8A02081300000024
:10034800559C02081300000061CA0208160000004C
:100358008D300308160000009132030817000000D2
:10036800A16A030816000000716B0308170000005B
:08037800217F030815000000BD
:100380002F49072291438D462E492F480A1A06D03D
:100390000722914381F30988022282F314882B48B3
:1003A0002B492C4A00F039F82B482C492C4A00F0F4
:1003B00034F82C482C492D4A00F02FF82C482D49B0
:1003C0002D4A00F02AF82D482D492E4A00F025F834
:1003D0002D482E492E4A00F020F82E482E490022A2
:1003E00000F026F82D482E49091A082903DB0022BF
:1003F0000260043001601F481F49884205D002682E
:10040000043003B4904703BCF7E700208646EC466F
:1004100000200021234A9047FEE7884207D0521A65
:1004200005D0037801300B700131013AF9D17047E2
:10043000884202D002700130FAE770471A487047CC
:1004400058380020584000205838002088F0030811
:1004500088010020FC0100200000020800000208C2
:10046000D8BD030888F00308880100208801002017
:10047000BC050008BC050008BC050008BC05000858
:10048000BC050008BC050008D8BD0308D8BD03089A
:1004900088F00308FC0100200C35002058350020AE
:1004A000583500204D410208FFFFFFFFFEE7FEE741
:1004B000FEE7FEE7FEE7FEE7FEE7FEE7FEE7FEE714
:1004C000FEE7FEE7FEE7FEE7FEE7FEE7FEE7FEE704
:1004D000FEE7FEE7FEE7FEE7FEE7FEE7FEE7FEE7F4
:1004E000FEE7FEE7FEE7FEE7FEE7FEE7FEE7FEE7E4
:1004F000FEE7FEE7FEE7FEE7FEE7FEE7FEE7FEE7D4
:10050000FEE7FEE7FEE7FEE7FEE7FEE7FEE7FEE7C3
:10051000FEE7FEE7FEE7FEE7FEE7FEE7FEE7FEE7B3
:10052000FEE7FEE7FEE7FEE7FEE7FEE7FEE7FEE7A3
:10053000FEE7FEE7FEE7FEE7FEE7FEE7FEE7FEE793
:10054000FEE7FEE7FEE7FEE7FEE7FEE7FEE7FEE783
:10055000FEE7FEE7FEE7FEE7FEE7FEE7FEE7FEE773
:10056000FEE71348854600F022F84EF68850CEF29A
:100570000000016851F47001016000BF00BF00BFBE
:10058000F1EE100A50F04070E1EE100A4FF000005A
:1005900080F314884EF63C71CEF20001086850F0EA
:1005A00040700860034804490160FFF7E9BE7047E6
:0C05B0000000022008ED00E00000000840
:020000040801F1
:1000000000000000000000000000000000000000F0
:1000100000000000000000000000000000000000E0
:10002000000000000000000000000000000004EAE2
:100030000F018600003D8601003D680120830042DB
:10004000F430F10B000E496E697469616C69736973
:100050006E672E2EF00400C000F411F40300790046
:100060000000F10A0006F10A0101F00201C085F169
:100070000A0001F00104C085095E8302A1F00001BD
:10008000C0008302DE8302C78304B5F10A0001F1D8
:100090000A0100F00200C000F10A0003F10A0101A8
:1000A000F00201C000F10500F00300C000F10B00F8
:1000B0000156F00400C0001E0000145D0B00CB4A86
:1000C000077108F42D00007D800085F419830387F3
:1000D000F00001C000F10B0010456E7465722059EC
:1000E0006561723A2020202020F00400C000F10B4E
:1000F00000023230F00400C0008F13028301B3818C
:100100000079830387F00001C000F10B000C456EFD
:10011000746572204D6F6E74683AF00400C0008FF1
:1001200013038301B38100CD830387F00001C00076
:10013000F10B000A456E746572204461793AF0044F
:1001400000C0008F13048301B3810102800154F4C5
:1001500019800128F41AF4114A00F420830387F06F
:100160000001C000F10B0010456E74657220486FED
:10017000757220283234293AF00400C0008F130031
:100180008301B381014F830387F00001C000F10BAD
:10019000000E456E746572204D696E757465733A14
:1001A000F00400C0008F13018301B381015CF412DD
:1001B0008000795E690020F10A0001F10A0100F077
:1001C0000200C000171301D001D801E001F502219F
:1001D000F41B83035780024AF41D83035780024AAD
:1001E000F10A0001F10A0102F00200C000F41B83D1
:1001F000035780024AF41DF303004783033EF41DB6
:10020000F10B00022028F00400C000F10200F00110
:1002100001C000F10B00022920F00400C0008002A0
:100220004AF41F83036FF10B00022028F00400C082
:1002300000F42FF423F303001583033EF10B0002B7
:100240002920F00400C00080024A830393F4028C4A
:100250000802658C0902805D0A029B5D0B029E68A4
:10026000002080024D17130271027602710276029D
:100270007BF4288001B7F4298001B7F42A8001B704
:100280001713028C0291028C02910296F4388001BD
:10029000B7F4398001B7F43A8001B74A00094A013E
:1002A00009F41300F41B870002B7F41D870002B79E
:1002B000F421877F02B7094A00F41C4A00F41E4A61
:1002C0007FF422F4140009F10A0001F10A0105F09B
:1002D0000200C000F411F416F00400C00009F10A95
:1002E0000000F10A0100F00200C000F419F423F349
:1002F00003001583033EF10B000120F00400C00051
:10030000F41F01890A0311F10B000120F00400C061
:1003100000F10200F00101C000F10B000120F00427
:1003200000C000F41DF303004783033EF10B0003FC
:10033000203230F00400C000F41B83035709F3118E
:1003400002F30BF30900F31103F30A0000F31F009B
:1003500000F00400C0000901890A0366F10B0001E6
:1003600030F00400C000F10200F00101C0000901FA
:10037000890A037EF10B000120F00400C000F102A5
:1003800000F00101C00009F40270084A0F52820314
:10039000875E09F40661002003A29948000084806A
:1003A00003A79920000082F40270084A0F528103CB
:1003B000BBF437F61C03A76900200968002009096F
:1003C000F00002C08509F10200F00100C08509F1CA
:1003D0000200F00101C08509F10A0000F00101C02E
:1003E0008509F10200F00104C08509F10200F00165
:1003F00005C08509F10200F00106C08509F102017E
:10040000F10200F00201C08509F10201F10200F0E1
:100410000202C085F10102F1010109F00500C08569
:10042000F1010009F00501C085F1010009F00502A4
:10043000C085F101004AFE525609F00503C085F15E
:10044000010009F00504C085F1010009F00600C0B3
:1004500085F10101F1010009F00601C085F10100FB
:10046000F1010109F00602C085F10101F101000965
:10047000F00608C085F10101F1010009F00603C092
:1004800085F10101F1010009F00606C085F10101C5
:10049000F1010009F10200F00607C085F10101F148
:1004A000010009F00702C085F1060009F00703C04A
:1004B00085F1060009F00704C085F1060009F0087F
:1004C00000C085F10103F10102F10101F101000910
:1004D000F00400C085F10102F1010109F00401C03E
:1004E00085F10103F10102F10101094D6F6E5475AF
:1004F0006557656454687246726953617453756ECA
:100500000000000300060009000C000F00124A6101
:100510006E4665624D61724170724D61794A756EC9
:100520004A756C4175675365704F63744E6F7644BE
:1005300065630000002300260029002C002F0032F4
:1005400000350038003B003E00410044FFFFFFFF44
:10055000FFFFFFFFFFFFFFFFFFFFFFFFFFFFFFFFAB
:10056000FFFFFFFFFFFFFFFFFFFFFFFFFFFFFFFF9B
:10057000FFFFFFFFFFFFFFFFFFFFFFFFFFFFFFFF8B
:10058000FFFFFFFFFFFFFFFFFFFFFFFFFFFFFFFF7B
:020000040802F0
:1000000000B583B04FF0000100914FF0F60301936B
:1000100008464FF007024FF0010303F0F7FB03B06F
:1000200000BD00BF10B54FF002004FF0F80117F00F
:1000300037F840F2B104C0F602044FF003004FF06D
:100040000001224604F0E6FB4FF0010040F2A5015A
:10005000C0F60201224604F0DDFB4FF0000001462D
:10006000224604F0D7FB4FF008004FF0090102468A
:1000700012F036FF4FF000004FF001014FF0030285
:1000800001F084FC4FF0010049F69A11C3F6996122
:1000900002F022FB4BF60C60C0F6030008F092FF62
:1000A00010BD00BF08B54FF00A0001F0AFFA08BD5F
:1000B00008B521B94FF0030017F0FCFE08BD012977
:1000C00004D14FF0010017F0F5FE08BD022903D15D
:1000D0004FF0000017F0EEFE08BD00BF11B101297E
:1000E00016D108E040F28811C2F200010B781370BB
:1000F0004FF00000704740F21000C4F202000168A7
:1001000081F01003C3F3001010704FF0000070472F
:100110004FF01400704700BF11B1012928D11AE037
:1001200042F63C01C4F200010B6813F4004F42F6A2
:100130003C00C4F2000001684FEAC1534FEAD350BB
:1001400008BF404207EE100AF8EEC70AC2ED000AE7
:100150004FF00000704740F2FC10C2F20000D0EDFA
:10016000007AB8EE670A82ED000A4FF0000070478F
:100170004FF01400704700BF30B585B04FF0010557
:1001800000954FF00304019402954FF000004FF0EA
:1001900005012246034601F049F9009501940295B4
:1001A0004FF0000021462246034601F03FF94FF48C
:1001B00000504BF64C61C0F6030140F20422C2F23B
:1001C00000020BF0E5FB05B030BD00BF38B51446AA
:1001D0004FF000031370002940F0838040F20020AC
:1001E000C2F20000016800297ED142F62402C4F266
:1001F00000024FF0CA0515604FF05303136042F63A
:100200000800C4F20000016841F40025056003689D
:1002100043F4000101604FF0FF00106043F6400519
:10022000C4F202052A6842F001032B604BF680619C
:10023000C0F60301086840F20003C4F2000318602E
:100240004FF0000540F20402C4F2000215604BF6C4
:100250002C61C0F60301086840F20802C4F20002F3
:10026000106040F22002C4F2000215604BF63061CB
:10027000C0F60301086840F21C01C4F200010860E6
:100280004BF63460C0F603000168116040F22C02A6
:10029000C4F200024FF0FF30106040F22801C4F2B7
:1002A00000010D801A8842F0010018804BF638607A
:1002B000C0F603004FF0070140F29932C0F6020287
:1002C00007F000FF40F20023C2F2000318604FF075
:1002D000010140F28812C2F200021170217028461A
:1002E00038BD4FF0140038BD4FF0000038BD00BFDE
:1002F00070B508F0B3FB054643F2D30440F2100694
:10030000C4F2000608F0AAFB401BA04209D940F243
:100310008813C2F200034FF0050119704FF000007E
:1003200070BD07F0DBFE336803F010018AB2002ACB
:10033000E8D040F24000C4F20000006870BD00BF89
:1003400030B583B005460C464FF0F60001A94FF0DA
:10035000020203F0AFFDBDF80430C3F340222A705F
:100360004FEAC3514FEAD153236003B030BD00BF01
:1003700000B583B04FF0000360F3492361F3080335
:1003800002A820F8043D4FF002014FF0F60203F0FE
:100390002DFE03B000BD00BFF8B54FF000000146D0
:1003A00001F08EFE40F24003C4F200031B68FFF729
:1003B0009FFF0646002800F0F980FFF799FF0746E7
:1003C000002800F0F380861B304617F02FFF04460C
:1003D0000D4687A3D3E9002318F08AFB002862D1D9
:1003E0002046294684A3D3E9002318F09DFB00286A
:1003F00059D140F2FC10C2F200000660FFF778FF0E
:100400000546002800F0D280C71BBE4294BFC6EB51
:100410000703C7EB0603012B66D940F2FC11C2F2B9
:1004200000010F60FFF764FF0446002800F0BE8063
:10043000461BB74294BFC7EB0603C6EB0703012B6D
:100440004FD940F2FC12C2F200021660FFF750FFD3
:100450000546002800F0AA80041BA64294BFC6EB04
:100460000403C4EB0603012B3ED940F2FC17C2F291
:1004700000073C60FFF73CFF0746002800F096802D
:10048000461BB44294BFC4EB0603C6EB0403012B26
:1004900029D940F2FC13C2F200031E60FFF728FFC7
:1004A000014640B982E040F28813C2F200034FF0E7
:1004B000020119707AE0C01BB04234BFC0EB0601E4
:1004C000C6EB000101290FD940F2FC12C2F2000272
:1004D000106040F28813C2F200034FF0020119705D
:1004E00064E03E4600E02646304617F09FFE024696
:1004F0000B4643A1D1E9000117F0BEFF17F080FFC2
:1005000017F062FF4FF000024FF00003C4F2E00367
:1005100018F0F8F83AA3D3E9002318F0A9F94FF03E
:1005200000024FF00003C4F2400318F0EBF817F09C
:1005300067FF044618F014FB0546204617F044FFF9
:1005400019F032F84FF000024FF00003C3F6E073E9
:1005500017F094FF17F0FEFE0446B0F5007F07D3B6
:1005600040F28810C2F200004FF0040202701DE059
:10057000003518BF01250DB1C0F50074284621468D
:1005800001F09EFD28462146FFF7F2FE38B940F201
:100590008813C2F200034FF00301197006E040F225
:1005A0008810C2F200004FF00002027042F62400F0
:1005B000C4F200004FF0CA0202604FF05303036020
:1005C00042F60802C4F2000211686FF3D3411160D1
:1005D00013686FF3D75313604FF0FF02026040F2CD
:1005E0000020C2F200004FF000010160F8BD00BF22
:1005F0000000000053126341000000004D136341EE
:1006000000000000D012634108B54FF440504BF693
:100610008461C0F6030140F21822C2F200020BF01E
:10062000B7F908BD70B582B00C461646684611464B
:100630004FF0080219F0B0FD009809F079FD40F282
:100640001023C2F200031860019809F071FD014601
:1006500040F21420C2F2000001600B2C00F2DD8099
:10066000DFE804F00613202D3A4754616EA2AFBCB8
:1006700040F21020C2F20000006818F053FE40F271
:100680002423C2F200031860B4E040F21024C2F246
:100690000004206818F0F4FA40F22422C2F20002AA
:1006A0001060A7E040F21023C2F20003186818F0AF
:1006B000DFFE40F22421C2F2000108609AE040F21D
:1006C0001020C2F20000006818F00AFD40F2242257
:1006D000C2F2000210608DE040F21021C2F200016F
:1006E000086818F0CFFC40F22424C2F20004206015
:1006F00080E040F21022C2F20002106818F014FDEF
:1007000040F22423C2F20003186073E040F210208C
:10071000C2F20000006818F0DFFF40F22424C2F2A9
:100720000004206066E040F21023C2F20003186863
:1007300018F042FF40F22421C2F20001086059E0A3
:1007400040F21025C2F20005286817F03DFE04466D
:100750000D464FF000024FF0000318F0ADF960B104
:10076000204629464FF000024FF00003C3F6E07325
:1007700017F084FE17F0C6FD0BE0204629464FF027
:1007800000024FF00003C3F6E07317F075FE17F098
:10079000B9FD07EE100AF8EEC77A40F22422C2F241
:1007A0000002C2ED007A25E040F21020C2F2000003
:1007B000006818F031FF40F22421C2F20001086005
:1007C00018E040F21024C2F20004206818F0A2FBE6
:1007D00040F22423C2F2000318600BE040F2102123
:1007E000C2F20001086818F0DBFA40F22422C2F2DB
:1007F0000002106040F22421C2F20001086809F0F2
:100800006DFC00904FF000040194304669464FF0B3
:10081000080219F0C1FC204601E04FF0140002B0BC
:1008200070BD00BF4BF6B863C0F603031A684EF6FE
:100830000C50CEF200000260FEE700BF08B5FFF7E3
:10084000F1FF00BF51E8002FBFF35F8F41E80003C5
:10085000012B3FF4F7AF1046704700BF13461A460E
:100860002DE9F00F0B460C460D460E460F46884606
:1008700089468A468B46092AC0F00780A0E8F80F0F
:10088000A2F10902092ABFF4F9AF4FF0080303FBF4
:1008900002F2144B1A44974600F020B800BF00BF84
:1008A000046000F01BB800BF80E8300000F016B80C
:1008B00080E8700000F012B880E8F00000F00EB898
:1008C00080E8F00100F00AB880E8F00300F006B814
:1008D00080E8F00700F002B880E8F00FBDE8F00F04
:1008E0007047134698080208EFF311804FF080011B
:1008F00081F3118870474FF0000000BF80F311882A
:10090000704700BF30B440F20003C0F6000340F26D
:100910008812C0F60002D01A4FEAA001B1F5C47FD8
:1009200004D81346264A9A4201D324E0FEE7254D17
:10093000254C601B20F003054FF0000340F200023D
:10094000C2F2000240F20001C0F6000105F104000D
:10095000C5F380045D589D5003F10403834226D102
:1009600009E05C589C5003F104035C58D45003F137
:1009700004038342F5D14EF60853CEF2000340F251
:100980000002C2F200021A604FF0B501CBF26B1107
:1009900043F25850C2F2000001604EF61453CEF2FA
:1009A00000031A6842F01001196030BC7047002C37
:1009B000D7D05C589C5003F104038342D1D1DAE7CD
:1009C00000000008040000088B01000810B4034672
:1009D00000283ED002F1100440F20000C2F20000F4
:1009E00040F82430002A0ADA12F10C0F35DB02F14C
:1009F0000C024EF61850CEF2000011542DE04EF2CB
:100A00000014CEF200040F299CBF0901C9B24EF2B6
:100A10000043CEF20003D1541146002AB8BF02F1C0
:100A20001F014FEA611004EB80014FF01F03C8F271
:100A300000031340002B05DA03F1FF3262F01F03BD
:100A400003F1010358B24FF0010202FA00F30B6008
:100A500003E0002AC8DB024CD5E710BC704700BF9A
:100A600080E100E01EF0040F0CBFEFF30880EFF30D
:100A7000098020E9F00F00F001B800BF10B502684E
:100A800043F20C53C2F200031A6041685960826855
:100A90009A60C168D96002691A61416959618269C5
:100AA0009A61C169D961026A1A62416A5962826AAD
:100AB0009A62C16AD962026B1A63416B5963826B95
:100AC0009A63C16BD96300F1400018644EF6285058
:100AD000CEF2000002685A641BF03EF9002800F0D4
:100AE000FB814BF6BC60C0F603001BF03BF94EF6F1
:100AF0002C54CEF200042368002B05DA4BF6CC60B0
:100B0000C0F603001BF02EF94EF62C51CEF2000178
:100B1000086810F0020F05D04BF6DC60C0F6030049
:100B20001BF020F94EF62852CEF200025478002C29
:100B300072D04BF6F460C0F603001BF013F94EF6CA
:100B40002853CEF20003597811F0010F05D04BF66F
:100B50000470C0F603001BF005F94EF62850CEF2E3
:100B60000000427802F00204E3B22BB14BF624708D
:100B7000C0F603001BF0F6F84EF62851CEF2000145
:100B8000487800F00402D4B22CB14BF64870C0F69D
:100B900003001BF0E7F84EF62853CEF20003597815
:100BA00001F00800C2B22AB14BF66C70C0F6030027
:100BB0001BF0D8F84EF62854CEF20004637803F008
:100BC0001001C8B228B14BF68C70C0F603001BF0C0
:100BD000C9F84EF62852CEF20002547804F02003F1
:100BE000D9B229B14BF6AC70C0F603001BF0BAF8CD
:100BF0004EF62850CEF20000427802F08004E3B2B4
:100C000053B14EF63851CEF2000109684BF6CC7064
:100C1000C0F603001BF0A6F84EF62850CEF20000F6
:100C2000428894B2002C5ED04BF6EC70C0F6030004
:100C30001BF098F84EF62853CEF20003598811F0B5
:100C4000010F05D04BF6FC70C0F603001BF08AF8CC
:100C50004EF62850CEF20000428802F00204A3B201
:100C60002BB14CF22800C0F603001BF07BF84EF6C7
:100C70002851CEF20001488800F0040294B22CB151
:100C80004CF24C00C0F603001BF06CF84EF62853F3
:100C9000CEF20003598801F0080082B22AB14CF26A
:100CA0008C00C0F603001BF05DF84EF62854CEF21F
:100CB0000004638803F4807188B228B14CF2BC0050
:100CC000C0F603001BF04EF84EF62852CEF200029A
:100CD000548804F4007399B229B14CF2D800C0F6DC
:100CE00003001BF03FF84EF62850CEF200000278C9
:100CF000002A63D04CF2F000C0F603001BF032F87B
:100D00004EF62854CEF20004237813F0010F05D0DC
:100D10004CF20010C0F603001BF024F84EF62851E8
:100D2000CEF20001087800F00202D4B22CB14CF2ED
:100D30002010C0F603001BF015F84EF62853CEF233
:100D40000003197801F00800C2B22AB14CF2381041
:100D5000C0F603001BF006F84EF62854CEF200044D
:100D6000237803F01001C8B228B14CF25C10C0F631
:100D700003001AF0F7FF4EF62852CEF20002147864
:100D800004F02003D9B229B14CF28010C0F6030060
:100D90001AF0E8FF4EF62850CEF20000027802F07A
:100DA0008004E3B253B14EF63451CEF2000109682B
:100DB0004CF2A010C0F603001AF0D4FF43F20C541A
:100DC000C2F20004216A4CF2CC10C0F603001AF003
:100DD000C9FF616A4CF2E010C0F603001AF0C2FFCE
:100DE000A16A4CF2F410C0F603001AF0BBFFE16AEE
:100DF0004CF20820C0F603001AF0B4FF21684CF250
:100E00001C20C0F603001AF0ADFF61684CF23020E0
:100E1000C0F603001AF0A6FFA1684CF24420C0F609
:100E200003001AF09FFFE1684CF25820C0F603005F
:100E30001AF098FF21694CF26C20C0F603001AF0FA
:100E400091FF61694CF28020C0F603001AF08AFF1E
:100E5000A1694CF29420C0F603001AF083FFE16907
:100E60004CF2A820C0F603001AF07CFF216B4CF274
:100E7000BC20C0F603001AF075FF216C4CF2D020A4
:100E8000C0F603001AF06EFF616B4CF2E420C0F66E
:100E900003001AF067FFA16B4CF20830C0F60300A4
:100EA0001AF060FF43F25450C2F2000002684CF2A4
:100EB0002C30C0F60300114612681AF053FF40F6BA
:100EC0004013C2F200031A684CF24430C0F603002B
:100ED000114612681AF046FFFFF7B0FC10BD00BFC4
:100EE00000B507F0A1FA002808BF5DF804FBEFF396
:100EF0000981EFF3118221E9F40F5DF804EB1EF094
:100F0000100F08BF21ED108A41F804ED0B4C226848
:100F1000002A18BF516007F0F9FA2268516851F8A9
:100F200004EB1EF0100F08BFB1EC108AB1E8F40F0B
:100F300082F3118881F3098870470000543500203E
:100F400008B540F6E160C0F602004FF0FF016FF017
:100F50000102FFF73BFD08BDF8B507460C461E46EB
:100F60000799089D14F0030F00D0FEE722B1A4EB0F
:100F70008500A0F1480401E004F14800012D01D8EA
:100F8000A16205E02A4602F0D3F9A7EB8507A76224
:100F90004FF0000363604FF01130E0624FF02231F8
:100FA00021634FF0333262634FF04433A3604FF05C
:100FB0005530E0604FF0663121614FF07732626169
:100FC0004FF08833A3614FF09930E0614FF0AA31C0
:100FD00021624FF0BB3262624FF0CC33A363E66311
:100FE000069820644FF0807161646FF00202226005
:100FF00005F11200F8BD00BF62B64EF60453CEF202
:1010000000031A6842F08050186000BF4FEA0010D9
:101010004CF25C33C0F603031A584CF6F461C0F688
:10102000030151F82200704738B504460D46FFF71A
:10103000EDFF4CF25C33C0F6030303EB041461686C
:10104000012902D0022903D101E0856038BD456144
:1010500038BD00BF2DE9F84F40F20401C4F202018F
:101060000C684CF27C42C0F60302136824EA0304C5
:101070004CF25445C0F60305286844EA00060E60A9
:1010800040F20447C4F202073968546821EA0401B7
:101090006B6841EA0300386040F60406C4F20206B9
:1010A0003768916827EA0107AC6847EA04033360B0
:1010B00040F60446C4F202063768D06827EA000703
:1010C000E96847EA0104346041F20406C4F202060A
:1010D0003368126923EA02032D6943EA0507376082
:1010E00041F20440C4F202000168016041F60404C8
:1010F000C4F202042668266041F60443C4F20203E7
:101100001A681A6042F20405C4F202052F682F60C3
:1011100040F20C01C4F202010C684CF27C36C0F6BD
:101120000306306824EA00044CF2F053C0F60303CF
:101130001A6844EA02050D6040F20C47C4F2020747
:101140003968746821EA0401586841EA00023A608B
:1011500040F60C05C4F202052F68B16827EA0107C2
:101160009C6847EA0400286040F60C42C4F2020280
:101170001568F76825EA0705D96845EA010414608F
:1011800041F20C05C4F202052868366920EA06001F
:101190001B6940EA03022A6041F20C47C4F20207CD
:1011A0003968396041F60C04C4F2020425682560F0
:1011B00041F60C40C4F202000668066042F20C03DD
:1011C000C4F202031A681A604CF2D047C0F6030753
:1011D000396840F2140EC4F2020ECEF800107C689A
:1011E00040F21441C4F202010C60BD6840F6140CD8
:1011F000C4F2020CCCF80050FE6840F61440C4F271
:10120000020006603B6941F21402C4F2020213605C
:101210004FF0000341F21447C4F202073B6041F66D
:101220001404C4F20204236041F61445C4F202051A
:101230002B6042F21406C4F20206336040F2000052
:10124000C4F2020007684CF23C54C0F60304226862
:1012500027EA02074CF2CC36C0F60306356847EAA7
:10126000050040F20007C4F20207386040F2004B6C
:10127000C4F2020BDBF80020656822EA0502706800
:1012800042EA0007CBF8007040F6000AC4F2020AF6
:10129000DAF80020A56822EA0502B06842EA0007F1
:1012A000CAF8007040F60049C4F20209D9F80020DB
:1012B000E56822EA0502F06842EA0007C9F8007012
:1012C00041F20008C4F20208D8F80020246922EA9A
:1012D000040236693243C8F8002041F20047C4F2E4
:1012E00002073D683D6041F60006C4F20206306820
:1012F000306041F60045C4F202052A682A6042F2D5
:101300000004C4F20204206820604CF2F442C0F6EB
:1013100003021068CEF80000506808609168CCF8AD
:101320000010D16840F61440C4F202000160126956
:1013300041F21401C4F202010A6041F21440C4F205
:101340000200036041F61402C4F20202136041F687
:101350001441C4F202010B6042F21400C4F2020014
:1013600003604FF0320008F03BFE40F20003C4F28D
:10137000020318684CF2A032C0F60302116820EA9A
:1013800001004CF21853C0F603031968014340F200
:101390000000C4F202000160DBF80000516820EA9E
:1013A000010059680843CBF80000DAF800009168A2
:1013B00020EA010099680843CAF80000D9F8000043
:1013C000D16820EA0100D9680843C9F80000D8F8BC
:1013D0000010126921EA02011B6941EA0300C8F802
:1013E000000039683960326832602B682B602068F1
:1013F00020604FF0010004F0CFFBBDE8F88F00BF84
:1014000008B543F63002C4F2020213686FEA5320B3
:101410006FEA4021116043F62003C4F201031A6809
:1014200042F001001860FFF715FE08BD2DE9F0013C
:101430009DF814709DF81860079D4CF20044C0F6AA
:10144000030454F820004FEA4104FF2F12D0D0F8D3
:101450000C804CF2F83CC0F6030C1CF8077007FA3D
:1014600004FC4FF0030707FA04F728EA07074CEAE1
:101470000707C760FF2B10D0D0F804C04CF21467E8
:10148000C0F60307FF5C07FA01F74FF0010303FA08
:1014900001F32CEA03033B434360FF2E0FD0876820
:1014A0004CF2C433C0F603039E5D06FA04F64FF017
:1014B000030303FA04F327EA030333438360B5F11C
:1014C000FF3F16D04FEAD10303F1080350F8236021
:1014D00001F007014FEA810105F00F0505FA01F55A
:1014E0004FF00F0707FA01F126EA0101294340F8FE
:1014F0002310FF2A10D001684CF2F033C0F603032A
:101500009B5C03FA04F34FF0030202FA04F421EAAD
:10151000040143EA01040460BDE8F001704700BF24
:101520002DE9F007079F089E099D4CF20044C0F684
:10153000030454F820004FEA41044FEAD10801F0B7
:10154000070C4FEA8C0C6FB1D0F80C9029FA04FA12
:101550000AF003094CF2784AC0F6030A1AF8099017
:1015600087F8009053B1476827FA01F101F00101B3
:101570004CF2C837C0F60307795C197056B183681E
:1015800023FA04F303F003034CF2F431C0F6030131
:10159000CB5C337045B108F1080850F8281021FAE7
:1015A0000CFC0CF00F032B6052B1006820FA04F41D
:1015B00004F003044CF2FC31C0F603010B5D137020
:1015C000BDE8F007704700BF4CF29053C0F603032C
:1015D00053F820100A684CF22443C0F6030353F872
:1015E00020100A404CF2C053C0F6030353F8200009
:1015F000824214BF00200120704700BF4CF200431C
:10160000C0F6030353F82000006970474CF22443EE
:10161000C0F6030353F820307BB139B14CF260516E
:10162000C0F6030151F82020136070474CF2A0422D
:10163000C0F6030252F82000036070473A2800F217
:10164000938000EB80004CF21863C0F6030353F85C
:10165000202002F1FF300D2800F28680DFE800F044
:10166000071019222B343D464F58616A737C43F6AC
:101670004400C4F20200036861F300030360704792
:1016800043F64003C4F202031A6861F300021A60D1
:10169000704743F64003C4F20203186861F3410047
:1016A0001860704743F64000C4F20200026861F31C
:1016B00082020260704743F64000C4F202000368F1
:1016C00061F3C3030360704743F64003C4F20203AF
:1016D0001A6861F304121A60704743F64003C4F2BB
:1016E0000203186861F345101860704743F6440020
:1016F000C4F20200026861F341020260704743F6DF
:101700004400C4F20200036861F3104303607047B1
:1017100043F64403C4F202031A6861F351421A60AB
:10172000704743F64403C4F20203186861F3924021
:101730001860704743F64000C4F20200026861F38B
:1017400086120260704743F64000C4F2020003684C
:1017500061F3C7130360704743F64003C4F202030A
:101760001A6861F308221A60704700BF00EB80001E
:101770004CF21863C0F6030353F820204CF638717E
:10178000C0F6030151F82200704700BF2DE9F84F61
:1017900004468A46914698469DF928709DF92C602A
:1017A0009DF930503A2800F2B680FFF7DFFF04EBD6
:1017B00084024CF21863C0F6030303EB82035A68F9
:1017C000022A94BF8369C369016A02F1FF3CBCF13C
:1017D000030F2ED8DFE80CF0021802186FF3010394
:1017E000BAF1000FC8BF6AF38203B9F1000FC8BF96
:1017F00069F3C303B8F1000FC8BF68F30613002FE5
:1018000017DD67F3C71314E06FF30923BAF1000F74
:10181000C8BF6AF38A23B9F1000FC8BF69F3CB23AD
:10182000B8F1000FC8BF68F30E33002FC8BF67F3CD
:10183000CF3302F1FF37032F44D8DFE807F002145B
:101840002638332C04D1002E06DD66F3820103E036
:10185000002EC8BF66F30001002DC8BF65F341012B
:101860006FF3C30130E0362C04D1002E06DD66F3A1
:10187000861103E0002EC8BF66F30411002DC8BF17
:1018800065F345116FF3C7111EE0382C04D1002E0B
:1018900006DD66F38A2103E0002EC8BF66F3082147
:1018A000002DC8BF65F349216FF3CB210EE0002E58
:1018B000C8BF66F30C31002DC8BF65F34D316FF31F
:1018C000CF3103E0022A01D8836100E0C3610162E5
:1018D00004EB84044CF21860C0F6030050F8243086
:1018E000012B02D0082B16D10BE04CF6B423C0F626
:1018F00003031A6840F24401C4F201010A60BDE822
:10190000F88F4CF6B422C0F60302116840F244404E
:10191000C4F201000160BDE8F88F00BF38B504468D
:101920000D46FFF723FF04EB84014CF21863C0F669
:10193000030303EB8104626802F1FF3103290AD833
:10194000DFE801F002040608456338BD856338BD51
:10195000C56338BD056438BD40F22823C2F20003D8
:1019600018684FF000020261016801F01003002BBB
:101970000CBF01204FF0FF3040F22C23C2F20003D5
:101980001A8810FA82F188B2188070472DE9F04F5A
:1019900089B0154640F22823C2F200034FF000023E
:1019A0001A604FEA01104CF6BC24C0F60304245818
:1019B000142900F2F480092C00F2F4804CF6244340
:1019C000C0F6030353F82430002B00F0EE804FEAFA
:1019D00005124CF6BC20C0F603008258944240F039
:1019E000E78004F1FF36072E4DD8DFE806F0340417
:1019F000101C284C4C4043F64007C4F202073868DC
:101A000040F001023A604FF0000605963EE043F6D2
:101A10004007C4F20207386840F002023A604FF013
:101A20000106059632E043F64007C4F20207386823
:101A300040F004023A604FF00106059626E043F6B6
:101A40004007C4F20207386840F008023A604FF0DD
:101A5000000605961AE043F64407C4F20207386808
:101A600040F001023A604FF0010605960EE043F6A1
:101A70004407C4F20207386840F002023A604FF0AF
:101A80000106059602E04FF00107059740F2282075
:101A90008246C2F2000ACAF800304CF6BC29C0F6F1
:101AA000030909EB011898F804B0D8F8081004915C
:101AB0000DF11F0300934FF0000601960296584661
:101AC00032460DF11E03FFF72BFD9DF81E309DF8E9
:101AD0001F2000924FF003070197D8F80C000290E6
:101AE000584604993A46FFF7A1FC09EB051595F80D
:101AF0000490D5F808800DF11F010091019602961F
:101B00004846414632460DF11E03FFF709FD9DF898
:101B10001F3000930197EA680292484641463A46D0
:101B20003346FFF783FCDAF800104CF64C40C0F661
:101B3000030003680B604CF6B822C0F6030210687D
:101B400088604CF62043C0F603031A688A610E626F
:101B50006FF07F40C862059B93B14CF61C42C0F603
:101B600003021068C86041F65910C0F602004FF039
:101B70000F014CF60C43C0F603031A57FEF726FF7D
:101B800040F22821C2F2000108684FF00002826290
:101B9000036843F0010101604FF001000AE04FF0DB
:101BA000000007E04FF0000004E04FF0000001E00B
:101BB0004FF0000009B0BDE8F08F00BF40F22823CD
:101BC000C2F200031B689BB1A8B91A686FF3000248
:101BD0001A604FF00000586240F22C21C2F200015E
:101BE00008801A6842F0010018604FF00100704749
:101BF0004FF0000070474FF00000704710B483B002
:101C000040F22823C2F200031B6803B310BB40F26A
:101C10002C22C2F20002586A148840EA0440019063
:101C200000BF00BF00BF00BF00BF586A148840EA71
:101C300004400090019C00988442ECD1DDED017AD3
:101C4000B8EEE70A81ED000A4FF0010004E04FF022
:101C5000000001E04FF0000003B010BC704700BF6F
:101C600040F22823C2F200031B689BB1A8B91A688E
:101C70006FF300021A6059624FEA114140F22C20C2
:101C8000C2F2000001801A6842F0010119604FF0B1
:101C9000010070474FF0000070474FF000007047A0
:101CA00043F67403C4F20203186847F20402C4F254
:101CB0000002136840F22E22C2F200024FF000012F
:101CC000117013F0010F04D010464FF0040202709F
:101CD0003EE04FEA106212F0600F07D040F22E2172
:101CE000C2F200014FF020030B7031E002F004015A
:101CF000C9B239B140F22E20C2F200004FF04002CA
:101D0000027025E0C3F3400343EAD06010F0010FF6
:101D100007D040F22E21C2F200014FF080030B7079
:101D200016E002F01001CBB23BB140F22E20C2F21D
:101D300000004FF0010202700AE002F00202D0B28D
:101D400030B140F22E21C2F200014FF002030B70BD
:101D500043F67401C4F202010B6843F0807008601E
:101D600047F20001C4F200010A6842F008030B6068
:101D700043F25450C2F20000016840F23022C2F235
:101D800000021160704700BF40F22E23C2F2000330
:101D90001878704708B547F61021C1F6FF714FF06B
:101DA0000C0218F0F9F94FF00C0008BD00B583B033
:101DB00043F64003C4F202031A6842F080501860F0
:101DC00047F20001C4F200010B6843F480720A601C
:101DD0000DF107006946FEF7B3FA43F67001C4F24D
:101DE00002010A684CF67443C0F6030319684A40BE
:101DF0004CF67043C0F6030319680A421FD1F0B1D4
:101E000042F63C00C4F2000002684FEAC2534FEAB7
:101E1000D3510098814212D142F63C02C4F2000232
:101E20001368C3F3C0319DF80700814207D140F227
:101E30003423C2F200034FF001021A700BE04CF69B
:101E40005840C0F603004FF0070142F22D12C0F6D1
:101E5000020206F037F903B000BD00BF70B50646B8
:101E600040F23424C2F2000442F60C05C4F200052C
:101E700003E000F0C9FA06F031F92378002BF8D01E
:101E8000286810F0200FF4D042F60001C4F20001DF
:101E90000A6842F60403C4F200031B68C2F302108E
:101EA00000EB800102F00F0000EB41013160C2F352
:101EB000023000EB8001C2F3032000EB41017160AE
:101EC000C2F3015000EB8001C2F3034202EB410078
:101ED000B060C3F3072101F0E002E02A14BFC3F3AE
:101EE00042320022B261C3F3011000EB800203F022
:101EF0000F0101EB4200F060C3F300324FEA8201B0
:101F00008818C3F3032202EB400101F1FF30306176
:101F1000C3F3035202EB8201C3F3034303EB41001B
:101F200000F16400706170BD70B58AB0014601A80F
:101F30004FF0240218F030F901A817F053FF059C68
:101F400004F10104E4B2019A46F26763C6F26663E3
:101F500083FB02104FEAE271C1EBA0054FF00006CF
:101F600065F3061605EB8500A2EB400262F303065B
:101F7000029D83FB05104FEAE571C1EBA00262F3FD
:101F80000E3602EB8200A5EB400565F30B26039AA3
:101F900083FB02034FEAE271C1EBA30060F3155625
:101FA00000EB8005A2EB450262F31346079B13B1D9
:101FB00003F0070101E04FF007014FF0000561F366
:101FC0004F35049946F26762C6F2666282FB0130C1
:101FD0004FEAE173C3EBA00060F3051500EB80034B
:101FE000A1EB430161F303054CF6CD40CCF6CC40A8
:101FF000A0FB04034FEAD30161F30C3501EB810030
:10200000A4EB400464F30B25069982FB01304FEAF0
:10201000E173C3EBA00382FB03024FEAE370C0EB62
:10202000A20202EB8200A3EB400262F3175503EB1E
:102030008303A1EB430161F3134540F23420C2F264
:102040000000027852B940F23424C2F2000400F0D9
:10205000DBF906F043F82378002BF8D042F6240190
:10206000C4F200014FF0CA0008604FF053020A604A
:1020700042F60C03C4F20003196841F080001860B6
:102080001A46136813F0400FFBD042F60001C4F269
:1020900000010E6042F60400C4F20000056042F642
:1020A0000C03C4F200031A686FF3C7121A6042F6F9
:1020B0002401C4F200014FF0FF0008600AB070BDB7
:1020C00070B506460D46B1F5007F2ED242F60C03E0
:1020D000C4F20003186810F4803F09D042F60C04E3
:1020E000C4F2000405F0FAFF216811F4803FF9D131
:1020F00042F62403C4F200034FF0CA021A604FF004
:10210000530018604FF0000242F61801C4F20001BB
:102110000A6065F3080266F3CF3242F63C00C4F26F
:10212000000002604FF0FF021A6070BD30B583B04E
:102130000DF107006946FEF703F905464CF66C43BE
:10214000C0F603031A6843F67000C4F2020002608E
:102150004CF67441C0F603010B680360026812F08C
:10216000020F09D143F67004C4F2020405F0B6FF71
:10217000206810F0020FF9D042F62401C4F20001E9
:102180004FF0CA030B604FF053020A6042F60C0096
:10219000C4F20000016841F080030360026812F09D
:1021A000400F09D142F60C04C4F2000405F096FF7A
:1021B000206810F0400FF9D04CF65041C0F60301F2
:1021C0000A6842F61003C4F200031A601A604CF663
:1021D0005440C0F60300016842F60802C4F200024F
:1021E000116042F60C03C4F2000318686FF3C710C5
:1021F000186042F62401C4F200014FF0FF020A60A9
:102200002DB19DF807000099FFF75AFF04E04FF049
:1022100000000146FFF754FF40F23423C2F20003EE
:102220004FF00100187003B030BD00BF0000000087
:1022300010B542F20803CEF204031A6842F010000F
:10224000186042F2E920C0F602004FF00F014FF093
:102250003602FEF7BBFB43F64001C4F202010C68F4
:1022600044F010030B6041F20004C4F200044CF689
:102270007842C0F60302106820604CF6FC61C0F69C
:102280000301886915F0D2FF15A3D3E9002316F0E6
:1022900039FA4FF000024FF00003C3F6F07316F066
:1022A000EBF816F057F841F22C03C4F20003188043
:1022B00041F22800C4F200004FF0000202804CF608
:1022C0007C41C0F60301086841F20C03C4F200032C
:1022D0001860228842F00101218010BDAFF3008018
:1022E0002D431CEBE2362A3F684620F007018D465D
:1022F00001B541F21003C4F200034FF000021A606E
:1023000006F0B6FBBDE801408546704770B504464F
:10231000B0F5CC7F2FD940F23233984216D940F233
:102320006560844215D940F6CB418C4214D941F600
:102330009712944213D943F22F36B44212D946F27F
:102340005F639C4298BF06250ED90FE04FF0010550
:102350000AE04FF0020507E04FF0030504E04FF0FC
:10236000040501E04FF00505072D06D1FEF766FADA
:102370004FF0070501E04FF00005FEF7B5FA0646FD
:1023800004EB84044FEAC4004CF68041C0F603011C
:1023900051F83520B0FBF2F39CB2012C05D9B4F50D
:1023A000805F04D3FEF74AFA01E04FF0020443F2E3
:1023B0000000C4F2000045F2555101604CF6804225
:1023C000C0F6030202EBC5052B7943F20401C4F207
:1023D00000010B6043F20802C4F2000214604AF6E6
:1023E000AA2303603046FEF789FA70BD08B543F2B0
:1023F0000003C4F200034CF6CC421A604FF0C80050
:10240000FFF784FF08BD00BF43F20003C4F20003DE
:102410004AF6AA221A60704710B5044643F2100328
:10242000C4F20003186810F0010F74D04FF03200AE
:1024300007F0D6FD43F21001C4F200010A6812F061
:10244000010F68D04FF0320007F0CAFD43F21003CD
:10245000C4F20003186810F0010F5CD04FF0320096
:1024600007F0BEFD43F21001C4F200010A6812F049
:10247000010F50D04FF0320007F0B2FD43F21003CD
:10248000C4F20003186810F0010F44D04FF032007E
:1024900007F0A6FD43F21001C4F200010A6812F031
:1024A000010F38D04FF0320007F09AFD43F21003CD
:1024B000C4F20003186810F0010F2CD04FF0320066
:1024C00007F08EFD43F21001C4F200010A6812F019
:1024D000010F20D04FF0320007F082FD43F21003CD
:1024E000C4F20003186810F0010F14D04FF032004E
:1024F00007F076FD43F21001C4F200010A6812F001
:10250000010F08D04FF0320007F06AFD43F21003CC
:10251000C4F200031B682046FFF7F8FE10BD00BFA1
:1025200002469CF8043043B1DCF8000040B140F2B0
:10253000C021C2F2000141F82200DCF8000050B9CD
:1025400040F2C023C2F2000353F8220049F6404291
:10255000002808BF104670474FF0010303FA00F04F
:1025600010F4E26F0CBF00200120704770B50D46DB
:102570004CF6F043C0F6030353F82040002C45D03E
:1025800000EB800040F23826C2F2000606EBC006DF
:1025900030464FF0000105F08DF9122D07D142F2BF
:1025A0000431C4F201010A6842F480030B60606BDD
:1025B00065F304006063E36C4FF0050007F010FD65
:1025C000A16841F08042A260236813F0020FFBD0A3
:1025D000E46C122D16D142F20430C4F201000168FD
:1025E0006FF39651016042F20002CEF204021368CA
:1025F0004FEA03504FEA105140F2194291420CBF8A
:10260000A4006400304605F063FA01E04FF0FF34A7
:10261000204670BDF8B504460F464CF6BC43C0F6E4
:10262000030303EB80056E88002E53D013F82000BF
:10263000012803D16878FFF799F801E04FF0000016
:102640005FB940F2B023C2F2000303EB84044FF001
:10265000000020604FF000012BE0BE420BD840F29A
:10266000B021C2F2000101EB84044FF07E522260DF
:102670004FF6FF711DE02A78012A0CBFC16A40F6AF
:10268000FF7140F2B023C2F2000303EB840406EEB4
:10269000907AB8EE667A00EE106AF8EE407AC7EEED
:1026A000270AC4ED000A06F1FF3007FB0107B7FB5C
:1026B000F6F12A78012A03D16878FFF72FF9F8BDDF
:1026C000022A07D1687840F6FF73994228BF19465D
:1026D000FEF7AAFCF8BD00BF38B52DED028B04460D
:1026E00008EE101A4CF6BC45C0F6030505EB800554
:1026F000F7EE007AB4EEE78AF1EE10FA09DC08464C
:1027000016F02EFA00289FED260A18BFB0EE408A78
:1027100001E0B7EE008A2B78012B1CD16878FFF717
:1027200025F8D0ED0B1A6D78B8EE612A62EE082A12
:1027300012EE900A15F048FE4FF000024FF0000331
:10274000C3F6E07315F09AFE15F004FE0146284624
:10275000FFF7E4F818E0022B16D16D78DFED110ACF
:1027600028EE201A11EE100A15F02EFE4FF000028E
:102770004FF00003C3F6E07315F080FE15F0EAFD9C
:1027800001462846FEF750FC40F2B020C2F200009D
:1027900000EB840484ED008ABDEC028B38BD00BFE1
:1027A0000000000000F07F4510B54FF000044FF02E
:1027B00000002146FFF790FF4FF001002146FFF790
:1027C0008BFF4FF002002146FFF786FF4FF003001A
:1027D0002146FFF781FF40F20C03C4F202031A689E
:1027E0001A6040F20C40C4F202000168016040F639
:1027F0000C03C4F202031A684CF62850C0F603001A
:10280000816822EA01024CF6CC40C0F603008168E0
:102810000A431A6040F60C43C4F202031A681A60B5
:1028200041F20C00C4F202000168016041F20C4365
:10283000C4F202031A681A6041F60C00C4F20200E6
:102840000168016041F60C43C4F202031A681A6081
:1028500042F20C00C4F202000168016040F2000381
:10286000C4F202031A681A6040F20040C4F2020087
:102870000168016040F60003C4F202031A684CF6D6
:102880006850C0F60300816822EA01024CF6045049
:10289000C0F6030081680A431A6040F60043C4F2A0
:1028A00002031A681A6041F20000C4F202000168D3
:1028B000016041F20043C4F202031A681A6041F653
:1028C0000000C4F202000168016041F60043C4F256
:1028D00002031A681A6042F20000C4F202000168A2
:1028E000016010BD08B502280ED84CF65853C0F64A
:1028F0000303195CFF290AD04CF60052C0F603020C
:10290000105CFFF733FE08BD4FF0FF3008BD4FF0FD
:10291000FF3008BD10B50446FFF7E4FF07EE900A4C
:10292000B8EE677A4CF65853C0F60303185D1128C9
:102930000BD147F62A21C1F6FF710A8801EE102A51
:10294000F8EEC11AC1EE870A03E09FED030AC7EE55
:10295000000A10EE900A10BD00F07F4540F2B0234F
:10296000C2F2000303EB80000068704738B50D46E3
:10297000044600B30E2801D9FDF760FF4CF6FC6356
:10298000C0F6030353F8240055B1B0FBF5F14FEA4C
:10299000114202F10103B0FBF3F0B0FBF5F502E0E8
:1029A0004FF000052A464CF63871C0F6030151F885
:1029B00024309A62DD6238BD10B582B000918DF886
:1029C0000420042840F0E2804FF00000FFF7C4FD2F
:1029D00048B1EC464FF00000FFF7A2FD01464FF072
:1029E0000000FFF7C3FF4FF00100FFF7B5FD48B14E
:1029F000EC464FF00100FFF793FD01464FF0010058
:102A0000FFF7B4FF4FF00200FFF7A6FD48B1EC4618
:102A10004FF00200FFF784FD01464FF00200FFF780
:102A2000A5FF4FF00300FFF797FD48B1EC464FF0CC
:102A30000300FFF775FD01464FF00300FFF796FF17
:102A40004FF00400FFF788FD48B1EC464FF004005A
:102A5000FFF766FD01464FF00400FFF787FF4FF0D8
:102A60000500FFF779FD48B1EC464FF00500FFF790
:102A700057FD01464FF00500FFF778FF4FF00600C5
:102A8000FFF76AFD48B1EC464FF00600FFF748FD3E
:102A900001464FF00600FFF769FF4FF00700FFF710
:102AA0005BFD48B1EC464FF00700FFF739FD0146EA
:102AB0004FF00700FFF75AFF4FF00800FFF74CFDFB
:102AC00048B1EC464FF00800FFF72AFD01464FF0F1
:102AD0000800FFF74BFF4FF00900FFF73DFD48B13D
:102AE000EC464FF00900FFF71BFD01464FF00900CF
:102AF000FFF73CFF4FF00A00FFF72EFD48B1EC4610
:102B00004FF00A00FFF70CFD01464FF00A00FFF7F7
:102B10002DFF4FF00B00FFF71FFD48B1EC464FF0C3
:102B20000B00FFF7FDFC01464FF00B00FFF71EFF07
:102B30004FF00C00FFF710FD48B1EC464FF00C00D1
:102B4000FFF7EEFC01464FF00C00FFF70FFF4FF0D0
:102B50000D00FFF701FD48B1EC464FF00D00FFF707
:102B6000DFFC01464FF00D00FFF700FF4FF00E00B5
:102B7000FFF7F2FC48B3EC464FF00E00FFF7D0FC35
:102B800001464FF00E00FFF7F1FE1EE04CF6BC438D
:102B9000C0F6030313F82010012916D14CF6BC42ED
:102BA000C0F6030202EB8000447804EB84034CF28D
:102BB0001861C0F6030151F82340EC462046FFF7A8
:102BC000AFFC01462046FFF7D1FE02B010BD00BFAA
:102BD00070B584B040F23825C2F200054CF654546A
:102BE000C0F603042846214604F04CFE05F12800F7
:102BF000214604F047FE05F15000214604F042FE54
:102C000043F64403C4F202031A6842F48070186069
:102C1000196841F400761E604CF65C55C0F6030559
:102C20002C6842F20433C4F201031C604CF6FC42EF
:102C3000C0F60302106842F20401C4F20101086008
:102C400042F20416C4F2010630604CF6B845C0F6F4
:102C500003052C6842F20C03C4F201031C6042F22B
:102C60000C12C4F2010214604CF64C50C0F6030082
:102C7000016842F21006C4F20106316042F21015FA
:102C8000C4F2010529604CF66454C0F603042368BD
:102C900042F22C02C4F20102136042F22C10C4F280
:102CA000010003604CF66051C0F603010E6842F269
:102CB0000805C4F201052E6042F20814C4F20104B2
:102CC00026604FF016004FF00101FEF7B7FC4FF001
:102CD00008004FF00101FEF7B1FC4FF00C004FF07F
:102CE0000101FEF7ABFC4FF005004FF00101FEF7CC
:102CF000A5FC4FF0000400944FF0010601960294E9
:102D00004FF01600214632464FF00603FEF73EFD17
:102D10004CF21865C0F6030595F8C401D5F8C81142
:102D200000940194D5F8C03102934FF0030223467A
:102D3000FEF77CFB0094019602944FF008002146B8
:102D400032464FF00603FEF721FD95F8AC00D5F8AA
:102D5000B01000940194D5F8A82002924FF003021D
:102D60002346FEF763FB0094019602944FF00C009B
:102D7000214632464FF00603FEF708FD95F8FC00A9
:102D8000D5F8001100940194D5F8F83002934FF073
:102D900003022346FEF74AFB0094019602944FF08B
:102DA0000500214632464FF00603FEF7EFFC95F88A
:102DB0007000696F00940194ED6E02954FF003026C
:102DC0002346FEF733FB4FF0040021462246FFF76F
:102DD000F3FD4FF0000520462946FFF77DFC304605
:102DE0002946FFF779FC4FF002002946FFF774FCF3
:102DF0004FF003002946FFF76FFC3046FFF7ACFBAE
:102E000050B14CF63870C0F6030041684CF6505291
:102E1000C0F6030213680B604FF00200FFF79CFB43
:102E200050B14CF63870C0F6030081684CF6505231
:102E3000C0F6030213680B604FF00300FFF78CFB32
:102E400050B14CF63870C0F60300C1684CF65052D1
:102E5000C0F6030213680B604FF00400FFF77CFB21
:102E600050B14CF63870C0F6030001694CF6505270
:102E7000C0F6030213680B604FF00500FFF76CFB10
:102E800050B14CF63870C0F6030041694CF6505210
:102E9000C0F6030213680B604FF00600FFF75CFBFF
:102EA00050B14CF63870C0F6030081694CF65052B0
:102EB000C0F6030213680B604FF00700FFF74CFBEE
:102EC00050B14CF63870C0F60300C1694CF6505250
:102ED000C0F6030213680B604FF00800FFF73CFBDD
:102EE00050B14CF63870C0F60300016A4CF65052EF
:102EF000C0F6030213680B604FF00900FFF72CFBCC
:102F000050B14CF63870C0F60300416A4CF650528E
:102F1000C0F6030213680B604FF00A00FFF71CFBBA
:102F200050B14CF63870C0F60300816A4CF650522E
:102F3000C0F6030213680B604FF00B00FFF70CFBA9
:102F400050B14CF63870C0F60300C16A4CF65052CE
:102F5000C0F6030213680B604FF00C00FFF7FCFA99
:102F600050B14CF63870C0F60300016B4CF650526D
:102F7000C0F6030213680B604FF00D00FFF7ECFA88
:102F800050B14CF63870C0F60300416B4CF650520D
:102F9000C0F6030213680B604FF00E00FFF7DCFA77
:102FA00050B14CF63870C0F60300816B4CF65052AD
:102FB000C0F6030213680B60FFF7F6FB04B070BDA8
:102FC00010B504464FF000004FF01101FFF7CEFAA4
:102FD00047F62A23C1F6FF73198807EE901AB8EE58
:102FE000670A06EE900AB8EE667AC0EE070AC4EDEC
:102FF000000A4FF0010010BD10B504464FF000006C
:103000004FF01201FFF7B2FA07EE900AB8EE677AB6
:103010009FED0B0AC7EE000A10EE900A15F0D4F9E6
:1030200005A3D3E9002315F06DFB15F0E9F9206045
:103030004FF0010010BD00BF6666666666660A4016
:1030400000F07F45AFF3008010B504464FF000005C
:103050004FF01001FFF78AFA07EE900AB8EE677A90
:103060009FED1B0AC7EE000A10EE900A15F0ACF9AE
:1030700011A3D3E9002315F045FB15F0C1F915F0B4
:10308000A3F90FA3D3E9002315F0F6F90EA3D3E9B2
:10309000002315F0EDFB4FF000024FF00003C4F2E7
:1030A000390315F0EBF915F0ABF920604FF0010092
:1030B00010BD00BFAFF300806666666666660A40B4
:1030C00052B81E85EB51E83F7B14AE47E17A643F6E
:1030D00000F07F45AFF3008030B472B64CF69453E5
:1030E000C0F603031A684EF63470CEF20000026098
:1030F0004CF69851C0F603010A684EF68853CEF29A
:1031000000031A604CF69C50C0F60300016842F2BE
:103110000802CEF2040211604CF6A853C0F6030375
:10312000186842F20C01CEF20401086043F6000375
:10313000C4F202031A6842F48030186019460B6822
:1031400013F4003FFBD043F64000C4F202000268D3
:1031500042F08051016047F20003C4F20003186896
:1031600040F480421A604CF69051C0F603010868A2
:1031700043F60803C4F2020318604CF6A052C0F6EE
:103180000302116843F60040C4F2020001604CF6ED
:103190008C53C0F603031A6843F60401C4F202011B
:1031A0000A6043F60000C4F20200036843F0807234
:1031B00002600146086810F0007FFBD043F6080368
:1031C000C4F202031A684FF0020161F301021A60AF
:1031D0001846036803F00C02082AFAD143F64401AA
:1031E000C4F20201086840F480430B6043F63000EB
:1031F000C4F20200026842F48011016047F2000349
:10320000C4F200031A6842F48071196047F20403A3
:10321000C4F200031A6842F400711960036843F4B1
:103220008022026043F61440C4F2020001684BF6AB
:103230002863C0F603031B684CF6A452C0F60302D1
:1032400010686FEA000259400A4206D04BF6286027
:10325000C0F603004178CC2904D12A4B2A4999426F
:1032600021D344E043F60841C4F2020142F63B2078
:10327000C0F61900086046F67F60C4F65D4008603D
:10328000134043F61442C4F202021360136843F081
:103290000201116043F60C40C4F20200026812F40D
:1032A000803FFBD1D9E7194C194D281B20F00305AD
:1032B0004FF0000340F20002C1F200024FF2FC01A5
:1032C000C0F6030105F10404C5F380005D589D506C
:1032D00003F10403A3420CD109E05858985003F1BC
:1032E00004035858985003F10403A342F5D130BCAD
:1032F00070470028F1D05858985003F10403A342B6
:10330000EBD1F4E7882D0408FCF0030800F1030872
:103310008B2D040843F63003C4F202031A6842F40A
:1033200000101860196841F480021A60704700BFED
:103330002DE9F0011546002A66D040F65013C2F27E
:10334000000353E8002F02F1010243E80024012C9E
:10335000F7D04CF6B452C0F60302146846F20846A1
:10336000C4F2020634604CF6B057C0F603073A6860
:1033700046F22843C4F202031A604FF6FF7846F281
:10338000304CC4F2020C46F23447C4F2020746F253
:103390002C46C4F202061C46454534BF2B46434624
:1033A000CCF8001038603360226842F001022260DD
:1033B000ED1A4FEA8303C918C018226812F0010FF2
:1033C000FBD1002DE8D140F65013C2F2000353E8C0
:1033D000002FA2F1010243E80024012CF7D053E8AA
:1033E000002FB2F1004F0DD14FF0000243E800244E
:1033F000012CF4D04EF60450CEF20000016841F0EA
:1034000080510160BFF32F8FBDE8F001704700BF0E
:1034100070B41646002A37D046F21045C4F20205B1
:103420002C6814F0010FFBD14CF6AC52C0F603022D
:10343000146846F20842C4F20202146046F21842CE
:10344000C4F20202116046F21C41C4F2020108609B
:1034500046F21440C4F2020006604CF6B852C0F6C0
:103460000302116846F21040C4F2020001600268D3
:1034700042F0010101603BB146F21040C4F202008B
:10348000036813F0010FFBD170BC704743F6104383
:10349000C4F20203186800280DDA43F60441C4F2AE
:1034A000020140F22312C4F267520A6048F6AB13DD
:1034B000CCF6EF530B6043F61040C4F202000168F3
:1034C00001F00042002A14BF02200020704700BF14
:1034D00043F61043C4F202031868002807DB43F6E2
:1034E0001041C4F202010A6842F000430B607047C9
:1034F00000F17840B0F5801F2CBF002001207047FC
:103500002DE9F04F83B006460D46FFF7F1FF002886
:1035100056D02846FFF7ECFF002854D0AE4255D8CD
:10352000FDF7E2F90190FFF7B1FF0446002841D111
:1035300006F178434FEA93304CF6C052C0F60302CE
:1035400012F8008041F28830FEF766FF4FF0020962
:1035500043F6104BC4F2020B43F60C47C4F20207C9
:103560004CF6046AC0F6030AFEF74EFF494668F3BC
:10357000C60169F3092141F48033CBF80030386883
:1035800010F4803FFBD15AF82820B61808F1010842
:103590005FFA88F8B542E7D24FF06400FEF73CFFCF
:1035A0004CF6BC51C0F60301086843F61043C4F260
:1035B00002031860FFF78CFF0198FDF79FF907E001
:1035C0004FF0020404E04FF0020401E04FF0020467
:1035D000204603B0BDE8F08F2DE9F04106460C46C9
:1035E00015460846FFF784FF002861D005F1FF303B
:1035F0002018FFF77DFF00285DD040F65013C2F27F
:10360000000353E8002F02F1010243E800210129E1
:10361000F7D0FFF73BFF074630BB4CF60061C0F622
:1036200003010A6843F61040C4F2020002608DB143
:1036300006F1FF3843F60C46C4F20206336813F471
:10364000803FFBD118F8011F04F8011BFEF7DCFED8
:10365000013DF3D14CF63464C0F60304226843F60E
:103660001040C4F202000260FFF732FF40F6501330
:10367000C2F2000353E8002FA2F1010243E8002444
:10368000012CF7D053E8002FB2F1004F0DD14FF0CD
:10369000000243E80024012CF4D04EF60450CEF290
:1036A0000000016841F080510160BFF32F8F04E0FA
:1036B0004FF0020701E04FF002073846BDE8F08105
:1036C00040F20833C2F2000318684CF6F062C0F60C
:1036D0000302116801604FF0000303604CF6EC62D6
:1036E000C0F60302116841604CF6D863C0F60303CC
:1036F0001A68C2614FF00D0101624CF6E863C0F632
:1037000003031A680260704740F20033C2F20003FC
:103710001868704770B48568C668446806FB054041
:103720004118196040F20030C2F200000068814286
:103730000CD2521890420CD340F20430C2F2000076
:103740000268891819604FF0010004E04FF0000092
:1037500001E04FF0000070BC704700BF2DE9F04160
:103760000546FEF751FE4FF01E044FF0000840F2F0
:103770000836C2F200064FF00107052D26D8DFE813
:1037800005F0030A0F14191E3268936983F00200D2
:10379000C0F340011BE03068416901F0010116E00F
:1037A00032685369C3F3400111E030684169C1F3E5
:1037B000C0110CE032685369C3F3801107E033682D
:1037C000986980F0010101F0010100E0414689B9EA
:1037D00033685A6912F4807F10D1586910F4806FF1
:1037E00010D1384606F0FCFB013CC6D14FF000007A
:1037F000BDE8F0814FF00100BDE8F0814FF000001E
:10380000BDE8F0814FF00000BDE8F0812DE9F04106
:1038100084B014461D46072900F2AD80072A00F245
:10382000AD8001EB81024CF63863C0F6030303EB75
:103830008202137C002B40F0A48004EB84024CF63F
:103840003863C0F6030303EB8202137C012B40F0C4
:103850009B804CF63863C0F6030301EB810653F8F6
:10386000262004EB840653F826309A4240F08F80DD
:1038700040F2FC27C2F200073870022A15D0032A52
:1038800025D0012A34D143F64000C4F20200066874
:1038900046F40012026040F20833C2F2000345F21F
:1038A0000047C4F200071F6022E043F64000C4F264
:1038B0000200066846F48002026040F20833C2F259
:1038C000000345F60007C4F200071F6010E043F64E
:1038D0004000C4F20200066846F40002026040F2B2
:1038E0000833C2F2000345F60047C4F200071F6028
:1038F0004CF63868C0F6030801EB810108EB810241
:10390000107991684FF0000700974FF0010601967B
:10391000D36802934FF003023B46FDF787FD04EBAB
:10392000840408EB84042079A16800970196E2687A
:1039300002924FF003023346FDF778FDFFF7C0FE19
:1039400045B340F20430C2F200000A99016040F22F
:103950000032C2F200020B9B136040F20C30C2F244
:1039600000004CF6DC61C0F603012A463B4608F035
:10397000D5F8304610E04FF000000DE04FF00000A9
:103980000AE04FF0000007E04FF0000004E04FF0C5
:10399000000001E04FF0010004B0BDE8F08100BF7D
:1039A00038B5044640F20833C2F200031D68A86926
:1039B00010F0020F67D0FFF783FEA96911F0020F24
:1039C00061D03FE040F20835C2F200052B684FF0AD
:1039D000A0021A614FF00200FFF7C0FE286881695B
:1039E00011F0010F08D0456915F4806F00F03C829A
:1039F000036843F4007202604FF0050004F0A0FB7E
:103A00004FF000051AE0012901D002290CD140F243
:103A10000833C2F2000318684FEA142202614FF023
:103A20000300FFF79BFE38B140F20831C2F20001FB
:103A30000B68E4B21C6101E04FF00005281C18BFC0
:103A4000012038BD4FF0000038BD4FF0000038BDF8
:103A50004FF0000038BD4FF0000038BD4FF00000BF
:103A600038BD4FF0000038BD4FF0000038BD4FF0BA
:103A7000000038BD4FF0000038BD4FF0000038BDE9
:103A80004FF0000038BD40F20832C2F20002136865
:103A90004FF000005861196860F3492119601A68F5
:103AA00042F4807018604FF00100FFF757FE0028C5
:103AB000CBD040F20835C2F200052B684FF0A001D0
:103AC00019614FF00200FFF749FE2868826912F081
:103AD000010F08D0436913F4806F00F0C8810168BA
:103AE00041F4007202604FF0050004F029FB40F23F
:103AF0000830C2F2000003684FF0000159611A68F3
:103B000061F349221A60186840F4807119604FF01F
:103B10000100FFF723FE00289AD040F20835C2F2D8
:103B200000052B684FF0A0021A614FF00200FFF76A
:103B300015FE2868816911F0010F08D0436913F45C
:103B4000806F00F09781026842F4007101604FF0CD
:103B5000050004F0F5FA40F20830C2F200000368F4
:103B60004FF0000159611A6861F349221A60186820
:103B700040F4807119604FF00100FFF7EFFD00285D
:103B80003FF469AF40F20835C2F200052B684FF0F0
:103B9000A0021A614FF00200FFF7E0FD286881697A
:103BA00011F0010F08D0436913F4806F00F06581B4
:103BB000026842F4007101604FF0050004F0C0FAA1
:103BC00040F20830C2F2000003684FF00001596172
:103BD0001A6861F349221A60186840F4807119600C
:103BE0004FF00100FFF7BAFD00283FF437AF40F275
:103BF0000835C2F200052B684FF0A0021A614FF0A1
:103C00000200FFF7ABFD2868816911F0010F08D0B1
:103C1000436913F4806F00F03381026842F400714D
:103C200001604FF0050004F08BFA40F20830C2F258
:103C3000000003684FF0000159611A6861F34922DE
:103C40001A60186840F4807119604FF00100FFF7A6
:103C500085FD00283FF405AF40F20835C2F20005AB
:103C60002B684FF0A0021A614FF00200FFF776FDBB
:103C70002868816911F0010F08D0436913F4806F3F
:103C800000F00181026842F4007101604FF005000C
:103C900004F056FA40F20830C2F2000003684FF018
:103CA000000159611A6861F349221A60186840F4EA
:103CB000807119604FF00100FFF750FD00283FF4BC
:103CC000D3AE40F20835C2F200052B684FF0A002D7
:103CD0001A614FF00200FFF741FD2868816911F079
:103CE000010F08D0436913F4806F00F0CF800268A1
:103CF00042F4007101604FF0050004F021FA40F237
:103D00000830C2F2000003684FF0000159611A68E0
:103D100061F349221A60186840F4807119604FF00D
:103D20000100FFF71BFD00283FF4A1AE40F208356B
:103D3000C2F200052B684FF0A0021A614FF002009A
:103D4000FFF70CFD2868816911F0010F08D0436965
:103D500013F4806F00F09D80026842F400710160EE
:103D60004FF0050004F0ECF940F20830C2F2000018
:103D700003684FF0000159611A6861F349221A6023
:103D8000186840F4807119604FF00100FFF7E6FCFD
:103D900000283FF46FAE40F20835C2F200052B68F0
:103DA0004FF0A0021A614FF00200FFF7D7FC28681D
:103DB000816911F0010F07D0436913F4806F6BD054
:103DC000026842F4007101604FF0050004F0B8F998
:103DD00040F20830C2F2000003684FF00001596160
:103DE0001A6861F349221A60186840F480711960FA
:103DF0004FF00100FFF7B2FC00283FF43EAE40F266
:103E00000835C2F200052B684FF0A0021A614FF08E
:103E10000200FFF7A3FC2868816911F0010F07D0A9
:103E2000436913F4806F3AD0026842F40071016074
:103E30004FF0050004F084F940F20830C2F20000AF
:103E400003684FF0000159611A6861F349221A6052
:103E5000186840F4807119604FF00100FFF77EFC94
:103E600000287FF4AFAD0BE64FF0010519E04FF0ED
:103E70000A0516E04FF0090513E04FF0080510E0C1
:103E80004FF007050DE04FF006050AE04FF005057D
:103E900007E04FF0040504E04FF0030501E04FF0A8
:103EA000020540F2FC20C2F20000017803297FF4F1
:103EB000AAADACE5F8B50D461446002A6FD080B225
:103EC000FFF76EFD002865D04FF00300FFF746FCBA
:103ED00000285FD040F20833C2F20003186802687D
:103EE00042F4807101604FF00100FFF737FC0028B9
:103EF00050D040F20833C2F20003186814F1FF31C9
:103F000018BF0121026861F38A2202604FF0A10309
:103F100003614FF00200FFF721FC00283AD040F285
:103F20000830C2F2000001688A6912F0010F31D036
:103F30004B6913F4806F2DD14FF0040640F208371F
:103F4000C2F200073046FFF709FC18B304F1FF3452
:103F5000012C27D1FCF7C8FC39680A696FEA020313
:103F600005F8013B0A686FF38A220A60FCF7C6FC79
:103F7000E8E72B681B6902E04FF004060E4D30465F
:103F8000FFF7ECFB0028F4D10B4B1868016841F4F3
:103F900000720260D4F1010038BF0020F8BD4FF07C
:103FA0000100F8BD386801696FEA010205F8012BCC
:103FB000002CC7D1E0E700BF0803002030B583B074
:103FC00015461C461A4601ABFFF7A4FB48B1019801
:103FD00029462246FFF76EFF00280CBF182000205C
:103FE00001E04FF01F0003B030BD00BF2DE9F84FD6
:103FF00093460D4600295DD004464FF0030840F279
:104000000839C2F2000901E0002E40D01FFA8BF0FF
:10401000FFF7C6FC00283DD00BF0070715F0010F95
:104020004CD14046FFF79AFB002836D0072F1AD80C
:10403000DDB13CB1D9F8000014F8011B6FEA0103AF
:10404000036104E0D9F800604FF0FF02326107F12C
:104050000107BA4605F1FF3635464046FFF77EFBBD
:10406000002845D119E02E4600E02E46D9F8000080
:10407000026842F4007101600BF1080B2BF0070B92
:104080004FF00500FFF76AFB0028BDD107E04FF0B5
:10409000010004E04FF0000001E04FF0000040F2AA
:1040A0000833C2F2000319680A6842F400730B6017
:1040B000BDE8F88F4FF00100BDE8F88F4046FFF7EC
:1040C0004DFB0028E9D0072FCDD82CB9D9F8003006
:1040D0004FF0FF021A6106E0D9F8000014F8011B46
:1040E0006FEA0103036107F1010705F1FF3598E766
:1040F000072FB8D82CB9D9F800504FF0FF022A6129
:1041000006E0D9F8000014F8011B6FEA010303610F
:1041100007F1010706F1FF3583E700BF30B583B033
:1041200015461C461A4601ABFFF7F4FA48B128467B
:104130002146019AFFF75AFF00280CBF18200020E3
:1041400001E04FF01F0003B030BD00BF08B543F2DF
:104150005850C2F2000043F65802C2F20002131A8D
:104160004FF0FF314FEAA302FCF778FB43F658000B
:10417000C2F2000044F25801C2F200010A1A4FEAEA
:10418000A2024FF0FF31A2F12002FCF767FB02F020
:1041900087FB40F21C30C2F2000044F20001C4F27E
:1041A00002014FF480524FF0030314F019F8FCF7AA
:1041B00023FF4FF0000008BDBFF36F8F704700BFB3
:1041C0004CF67473C0F60303185C00EB40014DF22B
:1041D000A002C0F6030252F821305B68704700BFAE
:1041E00038B54CF67473C0F603031B5C03EBC304D1
:1041F00040F23432C2F2000202EB840282F8211053
:1042000014693CB140F23435C2F200051346D2695C
:104210009B69A04738BD00BFF8B506460F464CF66F
:104220007473C0F603031D5C05EBC50040F2343423
:10423000C2F2000404EB8004D4F810C0BCF1000FFB
:1042400007D0E2698A4204D030464FF00001A369EA
:10425000E047E76163695BB105EBC50040F23432CA
:10426000C2F2000202EB800230463946926998475A
:1042700094F8201079B127696FB105EBC50540F2BC
:104280003433C2F2000303EB8505304694F8211065
:10429000E269AB69B847F8BD4CF67473C0F6030326
:1042A000185C00EB40014DF2A002C0F6030252F888
:1042B0002130D86840F08001D9607047F8B50446D5
:1042C00000EB40024DF2A003C0F6030353F8226056
:1042D00035686FEA0500306005F0010215F0020F45
:1042E0001CBF42F00202D2B215F0040F18BF42F018
:1042F000080215F0080F18BF42F0040215F4807F81
:1043000005D0316911F4804F18BF42F0100215F04A
:10431000200F00D1E2B104EBC40740F23433C2F203
:10432000000303EB870087688FB1716804EBC4005A
:1043300040F23433C2F2000303EB80034DF250002D
:10434000C0F60300005DC9B29B69B84700E073681E
:10435000F26812F0800F1CD015F0800F19D0F168B0
:104360006FF3C711F16004EBC40040F23433C2F2C2
:10437000000353F8203063B140F23432C2F200023D
:1043800002EB80024DF25000C0F60300005D91691F
:10439000984715F0400F17D004EBC40140F23433B6
:1043A000C2F2000303EB810253686BB1084640F28E
:1043B0003431C2F2000101EB80024DF25000C0F630
:1043C0000300005D91699847F8BD00BF684620F082
:1043D00007018D4601B54FF00600FFF76FFFBDE8FE
:1043E00001408546704700BF684620F007018D46B2
:1043F00001B54FF00500FFF761FFBDE801408546BC
:10440000704700BF684620F007018D4601B54FF0A8
:104410000400FFF753FFBDE801408546704700BF29
:10442000684620F007018D4601B54FF00300FFF705
:1044300045FFBDE801408546704700BF684620F053
:1044400007018D4601B54FF00200FFF737FFBDE8C9
:1044500001408546704700BF684620F007018D4641
:1044600001B54FF00100FFF729FFBDE80140854687
:10447000704700BF10B582B08DF807104CF674730A
:10448000C0F60303185C00EB40024DF2A001C0F639
:10449000030151F82240236813F0800FFBD002A9DA
:1044A00011F8012D626000EBC00040F23434C2F21A
:1044B000000404EB8004608C4FF0010205F0A8FDBD
:1044C000608404F1200402B010BD00BF70B582B05A
:1044D0008DF807104CF67473C0F60303185C00EBFC
:1044E00040014DF2A002C0F6030252F821402568B7
:1044F00015F0800F1DBF9DF807506560012600264E
:1045000000EBC00340F23430C2F2000000EB830540
:10451000688C0DF107014FF0010205F079FD688408
:1045200005F12005E16841F08002E260304602B00A
:1045300070BD00BF2DE9F84F81468B4690461E4660
:104540009DF828A04CF67473C0F603031D5C05EBC0
:1045500045024DF2A000C0F6030050F822409DF83D
:104560002C70012F14BF00270127082E06D0072E1C
:1045700002D1B8F1000F01D1FCF760F90AF1FF3167
:10458000CBB2012B01D9FCF759F94DF27002C0F6FC
:10459000030252F82500B0FBFBF1A1604FF00002CE
:1045A00067F38612BAF1010F04D0002F0CBF02236B
:1045B000002301E04FF0000363F30D3267F38E3206
:1045C00022614FF06C00B8F1020F14BF00230123E9
:1045D00063F3492018F1000818BF4FF0010868F391
:1045E0008A20082E18BF4FF0000868F30C3040F402
:1045F0000051E1604846FFF7E3FDBDE8F88F00BFDA
:10460000F0B585B00D461E464CF67473C0F6030334
:10461000195C01EB41044DF2A007C0F6030757F8FF
:1046200024704DF26C03C0F60303185C00EB4001EC
:104630004CF67874C0F6030404EBC1040AB1FCF72D
:10464000FDF875B9207B21699DF82C2000924FF070
:1046500001030193626902924FF003023346FCF7B3
:10466000E5FE207861689DF8283000934FF0010244
:104670000192A36802934FF003023346FCF7D6FE83
:104680004DF26800C0F603000168012D14BF00253B
:10469000012565F3C301796105B0F0BD2DE9F8434B
:1046A00005464CF67473C0F60303185C00EBC002B9
:1046B00040F23434C2F2000404EB82044DF2A00153
:1046C000C0F6030100EB40064FEA860301EB030846
:1046D00051F80390FCF708F9064694F82000B8B1A9
:1046E0004FF00007C9F80C703846394698F9042095
:1046F000FCF76CF928463946FFF772FDE3681BB1F9
:104700002846E169A26998474FF0000284F820200A
:104710003046FCF7F3F8BDE8F88300BF2DE9F04F11
:1047200085B005468B46924699464CF67473C0F6A2
:1047300003031E5C40F23438C2F2000806EBC607E1
:104740004FEA870708EB070406EB46004DF2A0018D
:10475000C0F6030101EB8006FCF7C6F8039043F6B0
:104760004003C4F2020318684DF26001C0F6030171
:104770000A6820EA020E4DF25802C0F603021068E1
:104780004EEA0000186043F64403C4F202031868BE
:10479000496820EA01005268104318604DF28C010C
:1047A000C0F6030105EB8503C818C95C427883781D
:1047B00090F803C0CDF800C0007901902846FFF7BB
:1047C0001FFF9DF8382000929DF83C10019128466B
:1047D000594652464B46FFF7ADFE109B48F807304E
:1047E0001298A060119A62601399E160149BA36112
:1047F000B0684FF00F0196F90420FCF7E7F84FF08E
:10480000010084F820000398FCF778F805B0BDE8B3
:10481000F08F00BF4CF67473C0F60303185C00EB16
:10482000C00340F23430C2F2000000EB8303196190
:104830005A6170474DF26C03C0F60303185C00EB3D
:1048400040014CF6C072C0F6030202EB0110704743
:10485000FA2884BF0530C0B2032812D84CF674730E
:10486000C0F60303185C00EBC00140F23432C2F220
:10487000000202EB81034FF6FF7058844FF00100F5
:1048800070474FF000007047FA2884BF0530C0B26F
:1048900003280ED84CF67473C0F60303185C00EBC3
:1048A000C00140F23432C2F2000202EB8103588CA4
:1048B00070474FF000007047082806D9102807D924
:1048C00020288CBF4020202070474FF00800704700
:1048D0004FF01000704700BF022809D0032804D011
:1048E000012814BF0020012070474FF003007047DB
:1048F0004FF00200704700BF40F60013C5F20003FE
:10490000186840F60802C5F200021168C1F34103BD
:10491000022B12BF6FF30200032363F3020040F483
:1049200000406FF3995040F60012C5F2000210608B
:1049300040F60401C5F200010B6843F48070086082
:10494000704700BF4DF29013C0F603031A6840F69B
:104950001030C5F200000260704700BF10B440F68E
:104960005473C2F200031A5CE0B14FF0000340F64A
:104970000C41C2F200014FF04C0404FB0212D1685A
:1049800021F0030202F1040262F312034FF001016D
:1049900061F3DC434DF20012C0F6030202EB40105B
:1049A00081690B6010BC704770B440F22003C5F2FF
:1049B00000031868C0F34342022A01D0062A29D115
:1049C00000F00F014DF29815C0F6030555F821606F
:1049D000C0F30A1505F1030398081BD041F200014A
:1049E000C5F2000100F1FF3404F001040A68334607
:1049F00072604FF0010282420ED10AE00C6803F1AE
:104A0000040343F8044F0C685C6002F10202824226
:104A1000F4D1356070BC7047002CEFD00C6803F106
:104A200004035C6002F101028242E7D1F1E700BFBA
:104A300070B44DF28013C0F6030353F8206032685F
:104A4000002A3CD04DF20011C0F6030101EB4011E9
:104A500002F103024FEA9202CB691B689A420CD919
:104A600040F63402C5F2000211684FF0010303FA68
:104A700000F008431060184623E006F10403C2B1B9
:104A800002F1FF3000F00105086953F8044B04609F
:104A9000501E18D10DE00C691A4652F8045B2560CF
:104AA00000F1FF300C695B68236002F104030138F8
:104AB000F1D14FF0000131604FF0010001E04FF003
:104AC000000070BC7047002DE5D00A6953F8044B14
:104AD00014600138DFD1ECE708B54FF0010303FAA9
:104AE00000F040F23242C2F200021388184210D0A5
:104AF00023EA000340F23240C2F200000380CA6B96
:104B000052B1086A4FF0000104F0C0FC4FF0000001
:104B100008BD4FF0000008BD4FF0010008BD00BF08
:104B200070B540F21403C5F200031C684DF2F800A2
:104B3000C0F6030001680C4200F0BB8140F65072E1
:104B4000C2F200021378012B40F2B38140F2180048
:104B5000C5F2000001684DF2AC12C0F60302136802
:104B6000194200F0A68140F61800C5F20000016865
:104B700011F0010F56D040F60815C5F200052A685D
:104B800040F60830C5F2000003682A60036040F672
:104B90005471C2F20001087840F60C41C2F20001E3
:104BA0004FF04C0505FB001503F00100E96A0143D5
:104BB000E962C3F3C000296B0143296303F00803D2
:104BC000D8B258BBD2B212F0010F0ED01DE0EA6A83
:104BD00022B105F1100000F087FF2BE02B6B002BBA
:104BE000F7D1686B0028F4D124E012F0900FEED0DA
:104BF00040F63403C5F20003186820F00101196083
:104C00004FF00000FFF714FFE1E76E6B4FF000007C
:104C10002946FFF761FF30436863D8E74FF0000192
:104C2000E963CFE740F61802C5F20002136813F4F7
:104C3000803FA0D140F61801C5F200010A6802F0D9
:104C4000020398B2002856D040F62815C5F2000598
:104C50002A6840F62830C5F2000003682A60036025
:104C600040F65471C2F20001487840F60C41C2F29D
:104C700000014FF04C0505FB001503F00100E96A47
:104C80000143E962C3F3C000296B0143296303F0C8
:104C90000803D8B258BBD2B212F0010F0ED01DE0FB
:104CA000EA6A22B105F1100000F01EFF2FE02B6B25
:104CB000002BF7D1686B0028F4D128E012F0900F98
:104CC000EED040F63403C5F20003186820F002016C
:104CD00019604FF00100FFF7ABFEE1E76E6B4FF09C
:104CE00001002946FFF7F8FE30436863D8E74FF02C
:104CF0000001E963CFE740F61801C5F200010A6838
:104D00004FEA124303F0020081B200299CD140F621
:104D10001801C5F200010A6802F0040398B20028E5
:104D200056D040F64815C5F200052A6840F64830CE
:104D3000C5F2000003682A60036040F65471C2F2B5
:104D40000001887840F60C41C2F200014FF04C059A
:104D500005FB001503F00100E96A0143E962C3F3B2
:104D6000C000296B0143296303F00803D8B258BB84
:104D7000D2B212F0010F0ED01DE0EA6A22B105F1A5
:104D8000100000F0B1FE2FE02B6B002BF7D1686B09
:104D90000028F4D128E012F0900FEED040F6340352
:104DA000C5F20003186820F0040119604FF00200FA
:104DB000FFF73EFEE1E76E6B4FF002002946FFF77A
:104DC0008BFE30436863D8E74FF00001E963CFE71B
:104DD00040F61801C5F200010A684FEA124303F0D9
:104DE000040081B200299CD140F61801C5F20001EF
:104DF0000A6802F0080398B258B940F61801C5F2E3
:104E000000010A684FEA124303F0080081B200294A
:104E10004FD040F66815C5F200052A6840F66830A4
:104E2000C5F2000003682A60036040F65471C2F2C4
:104E30000001C87840F60C41C2F200014FF04C0569
:104E400005FB001503F00100E96A0143E962C3F3C1
:104E5000C000296B0143296303F00803D8B210B1E5
:104E60004FF00001E963D2B212F0010F08D06E6B6F
:104E70004FF003002946FFF72FFE304368630EE032
:104E800012F0900F0BD040F63403C5F200031868FF
:104E900020F0080119604FF00300FFF7C9FDEA6A2E
:104EA0001AB92B6B0BB9686B18B105F1100000F043
:104EB0001BFE14F0100F01D0FFF776FD14F4805F95
:104EC0000DD040F62171C2F200014FF001020A70CC
:104ED00040F61873C2F20003186802F09BFF14F446
:104EE000005F01D0FFF708FD14F4006F14D040F606
:104EF0006C60C2F200004FF00101017040F6447393
:104F0000C2F200034FF000021A7040F61870C2F2AD
:104F10000000006802F07EFF002C14DA40F66C619D
:104F2000C2F200014FF000030B7040F64470C2F271
:104F300000004FF00102027040F61871C2F2000149
:104F4000086802F067FF40F21403C5F200031C601A
:104F500070BD00BF684620F007018D4689B500AFDF
:104F6000FFF7DEFDBD46BDE889408546704700BFBE
:104F70002DE9F04140F60C46C2F200064FF04C031A
:104F800003FB0066304650F8205F4DF20018C0F673
:104F900003084FEA451708EB07044FF000014FF0F4
:104FA0001C0215F01DF935624FF00100B06258F88F
:104FB00007204FF00003136061690B60A0684FF099
:104FC000FF02026061680B60A0690360E1680A602B
:104FD0004DF29812C0F6030252F8250003604DF21C
:104FE0008011C0F6030151F825201360BDE8F0815F
:104FF00000B583B04FF00003019340F21001C5F2F9
:1050000000010A68B0F1FF3F08BF102060F3891269
:1050100042F0200040F21003C5F200031860194668
:1050200040F63F52C0F20302019800F101000190E6
:105030000B6813F0200F02D001989042F4D94FF082
:10504000030004F0CDFF03B000BD00BF2DE9F8431D
:105050004FF04C0303FB00F040F60C41C2F200019C
:105060004418256A4FF0010606FA05F64DF20012C3
:10507000C0F6030202EB45174058002867D0A3682A
:10508000FBB1D7F80080D8F8001011F4004F18D108
:10509000D8F80020914663F30A09007AFFF71CFC58
:1050A00060F3934949F4004965F3995949F08050F8
:1050B000C0F3404363F39A60C8F800002846FFF746
:1050C00097FFE168F1B17A68106810F4004F19D1C8
:1050D0002846FFF743FCD7F80480D8F80070E3684F
:1050E00063F30A072168087AFFF7F6FB60F393473A
:1050F00047F4004242F01047C7F3404060F39A671C
:10510000C8F800704DF29813C0F6030353F8251049
:105110004FF000020A60A06858B140F61C03C5F2C7
:105120000003196846EA010290B2196860F30F01A2
:105130001960E3685BB140F61C00C5F2000002682C
:1051400046EA1246B6B2016866F31F410160BDE847
:10515000F88300BF70B582B04FF00002019240F2B8
:105160001003C5F20003196841F0010018600192B4
:105170001A6812F0010F19D0019940F63F53C0F29E
:105180000303994212D840F21000C5F2000040F625
:105190003F52C0F20302019901F10101019103683C
:1051A00013F0010F02D001999142F4D94FF003009E
:1051B00004F016FF4FF00000019040F21002C5F21B
:1051C00000021368002B1DDB019940F63F50C0F22E
:1051D0000300814216D84FF0030640F21005C5F2D5
:1051E000000540F63F54C0F20304304604F0F8FED8
:1051F000019A02F1010201922B68002B02DB019956
:10520000A142F2D902B070BD00B583B04FF00003E7
:10521000019340F21000C5F20000026842F0100154
:10522000016040F63F52C0F20302019B03F101030B
:105230000193016811F0100F02D0019B9342F4D941
:105240004FF0030004F0CCFE03B000BD50B14DF2AE
:10525000A811C0F603010A6840F21803C5F2000362
:105260001A6070474DF2F403C0F603031A6840F267
:105270001800C5F200000260704700BF38B54FF05B
:10528000000440F60063C5F200031C6040F6000213
:10529000C5F20002106840F0030164F3820164F378
:1052A0000A11116040F22405C5F200052B684FF089
:1052B000400262F30F032B60204662F31F40214639
:1052C00062F31F4162F30F0140F22805C5F20005A9
:1052D00029604FF0800363F30F0040F20412C5F21F
:1052E000000210604FF0C00161F30F0040F208159A
:1052F000C5F2000528604FF4807363F30F0040F29D
:105300000C12C5F2000210604FF0FF30FFF770FE84
:10531000FFF77AFF40F61000C5F20000046040F687
:105320001401C5F200010C604FF0FF3540F6180380
:10533000C5F200031D6040F61C02C5F200021460B5
:105340002046FFF715FE4FF00100FFF711FE4FF06A
:105350000200FFF70DFE4FF00300FFF709FE4FF0CC
:105360000400FFF705FE4FF00500FFF701FE4FF0C8
:105370000600FFF7FDFD4FF00700FFF7F9FD40F2D3
:105380001800C5F20000046040F21401C5F20001EB
:105390000D604FF00100FFF759FF38BD40F2324376
:1053A000C2F2000319884FF0010202FA00F008402F
:1053B00000280CBF02200320704700BF40F60013F6
:1053C000C5F200031B68C3F3076202F08000C1B29C
:1053D00009B143F0804343F4001040F60012C5F2D7
:1053E00000021060704700BF2DE9F84305461646DD
:1053F0004DF20018C0F6030808EB40184DF2801378
:10540000C0F6030353F820704FF0010909FA00F9C0
:105410000C46A9B9386840B940F23243C2F20003E1
:10542000188819EA000F5AD10AE040F23241C2F25C
:1054300000010A8819EA020F02D02846FFF7D8FDBA
:1054400006F1030107F1040388081CD000F1FF32C4
:1054500002F0010CA4F1040151F8042F43F8042BCD
:1054600001383ED10FE001F1040249681C4644F8BE
:10547000041B00F1FF3002F1040152685A6004F18C
:1054800004030138EFD13E6040F23243C2F2000320
:10549000198849EA0109A3F8009065B940F610108F
:1054A000C5F2000002684FF0010161F3D44266F3D7
:1054B0000602026009E0D8F8140002684FF0010308
:1054C00063F3DC4266F312020260D8F80030186819
:1054D00040F004421A6016B12846FFF7A9FABDE869
:1054E000F883BCF1000FBED051F8042F43F8042B11
:1054F0000138B8D1C7E700BF70B504464DF2981324
:10550000C0F6030353F82060334653F8045BAA4205
:1055100038BF1546084619462A4614F03DFE4FF09E
:10552000000030602046FFF719FA4DF20011C0F676
:10553000030101EB441463681A6842F004401860E8
:10554000284670BDF8B5054640F60C43C2F200038C
:105550001868002871D040F60C41C2F20001CA6CF4
:10556000002A71D040F60C44C2F20004D4F89860CE
:10557000002E6DD040F60C47C2F20007D7F8E43099
:10558000002B69D040F60C40C2F20000D0F8301178
:10559000002965D040F60C42C2F20002D2F87C41EC
:1055A000002C61D040F60C46C2F20006D6F8C87155
:1055B000002F5DD040F60C43C2F20003D3F8140272
:1055C000002859D040F60C41C2F20001D1F8602207
:1055D000002A55D0464E4FF00807FBF72FF92C7ADA
:1055E000002C53D040F23042C2F200021088014633
:1055F00010F0020F55D04FF0010404F1010441FAFC
:1056000004F212F0010FF8D14FF0010101FA04F198
:10561000084340F23043C2F20003188044B968895D
:10562000FFF74AF9B060A889FFF746F9F06042E059
:105630006A89B260A989F1603DE040F60C46C2F289
:1056400000064FF000071EE02A4E4FF001071AE057
:10565000294E4FF0020716E0284E4FF0030712E0E4
:10566000274E4FF004070EE0264E4FF005070AE0E4
:10567000254E4FF0060706E0244E4FF0070702E0E4
:105680001B4E4FF00807072FA9D9A6E740F2304379
:10569000C2F20003188840F0010119804FF00004A5
:1056A000BDE740F0020440F23043C2F200031C8028
:1056B0004FF00104BCE740F65470C2F200000755F9
:1056C000374647F8205B38464FF000014FF01C0288
:1056D00014F086FD34626B68B36306F110004FF07E
:1056E00006012A683B4600F0DFF92046F8BD00BFFE
:1056F0006C0E0020580C0020A40C0020F00C0020A0
:105700003C0D0020880D0020D40D0020200E00202C
:10571000022907D140F60003C5F200031A6860F3BE
:105720000A121A60704700BF10B54FF0000440F62F
:105730003403C5F200031C6040F60400C5F200000B
:10574000026842F0010101602046FFF711FC4FF0B2
:105750000100FFF70DFC4FF00200FFF709FC4FF0CE
:105760000300FFF705FC4FF00400FFF701FC4FF0CA
:105770000500FFF7FDFB4FF00600FFF7F9FB4FF0C8
:105780000700FFF7F5FB4FF0FF30FFF731FC40F269
:105790003243C2F200031C8040F61800C5F200003C
:1057A0004FF0FF3202604DF2B011C0F603010868FD
:1057B00040F61C03C5F2000318604DF2FC02C0F66F
:1057C0000302116840F61400C5F2000001604DF2BA
:1057D0009413C0F603031A6840F61001C5F20001E5
:1057E0000A6020464FF00201FFF792FFFFF7AAF888
:1057F0002046FFF72BFC4FF00100FFF727FC4FF08E
:105800000200FFF723FC4FF00300FFF71FFC4FF0EF
:105810000400FFF71BFC4FF00500FFF717FC4FF0EB
:105820000600FFF713FC4FF00700FFF70FFC10BD59
:1058300008B5FFF779FF08BD704700BFF0B585B028
:10584000054641F28830FCF7E7FD002D62D043F6B3
:105850003401C4F202010C6844F080060E604FF07F
:10586000000400944FF0030601964FF00A070297D8
:1058700020464FF00B0132462346FBF7D7FD00943C
:105880000196029720464FF00C0132462346FBF763
:10589000CDFD40F20C06C5F20006336843F040022D
:1058A0003260FFF757FC40F23800C5F200004FF4B9
:1058B0000411016044F6206004F092FBFCF7A4FDA3
:1058C000336843F0400064F3082064F349204FF04C
:1058D000050262F38D2064F35D7040F08041316019
:1058E00044F6206004F07CFBFCF78EFDFFF7C6FC5D
:1058F00040F20803C5F2000340F28110186044F63C
:105900005570C0F602004FF00F014FF04302FBF755
:105910005DF813E04FF000004FF00F014FF043022D
:10592000FBF754F84FF0000340F23802C5F20002D2
:10593000136040F21800C5F2000003602846FFF72C
:105940007BFF4FF06400FCF767FD05B0F0BD00BFC2
:105950002DE9F04182B04DF2B417C0F6030745F6C9
:105960003126C0F6020640F28C15C2F200054FF057
:105970000408CDF8008038464FF0800132462B46AF
:1059800002F094FB40F26444C2F200042060CDF8BF
:10599000008038464FF08101324605EB080302F0E3
:1059A00085FB6060CDF8008038464FF082013246BA
:1059B00005F1080302F07AFBA060CDF800803846BC
:1059C0004FF08301324605F10C0302F06FFBE060FB
:1059D000CDF8008038464FF08401324605F11003BF
:1059E00002F064FB2061CDF8008038464FF085015D
:1059F000324605F1140302F059FB6061CDF80080D6
:105A000038464FF08601324605F1180302F04EFB8E
:105A1000A061CDF8008038464FF08701324605F18D
:105A20001C0302F043FBE06102B0BDE8F08100BF5F
:105A300080B505464FF0000640F23C49C2F200092D
:105A400040F28448C2F2000840F23847C2F2000730
:105A50001FE0FAF749FF2C68616829604FF00002E7
:105A60006260237B062B0ED1216849F82610092E8F
:105A70009CBF0136F6B2012E03D93A8802F1010229
:105A80003A8088F80060FAF739FF23680BB1A06804
:105A900098472B6803F1FF3010F1030FD9D902F0BA
:105AA00087F94FF00006F4E70260B3F1FF3F18BF3B
:105AB0008360FF290ED143F25453C2F200031A68E7
:105AC00022B192F829304FEA530101E04FF007016B
:105AD0000173704701F07F010173704710B14FF0FF
:105AE00000020260704700BF38B50446FAF7FCFEBA
:105AF000054640F28643C2F200031A8802F1010211
:105B00001A80002C35D06368EBB940F28840C2F2AD
:105B10000000028802F101020280207B40F28C1317
:105B2000C2F2000353F82010616043F82040247B48
:105B300040F26442C2F2000252F8240002F06AF914
:105B40004FF0010422E040F23440C2F2000002882B
:105B500002F101020280247B062C15D140F23A4169
:105B6000C2F200010B8803F101030B804FF0000427
:105B70000CE040F23640C2F20000018801F1010160
:105B800001804FF0000401E04FF000042846FAF7CE
:105B9000B5FE204638BD00BF10B5044640F2946003
:105BA000C2F200004FF000014FF0240214F018FB85
:105BB000D4B140F2D440C2F200004FF000014FF0E7
:105BC000480214F00DFB40F26450C2F200004FF0A6
:105BD00000014FF0240214F003FB40F25C53C2F2C8
:105BE00000034FF002021A7010BD00BF38B54DF22D
:105BF0001C23C0F6030353F8205040F22051C2F298
:105C0000000151F820404DF26022C0F60302105C02
:105C1000FBF7F4FC2840A04214BF0020012038BD4F
:105C20004DF26023C0F603031A5C40F26451C2F2E5
:105C3000000151F822204DF21C23C0F6030353F853
:105C4000200002420CBF00200120704770B440F6D3
:105C50005013C2F2000353E8002F02F1010243E89F
:105C600000210129F7D04DF26022C0F60302155C35
:105C700040F29461C2F2000151F825404DF21C2619
:105C8000C0F6030656F8202024EA020041F8250059
:105C900053E8005FA5F1010543E80056012EF7D057
:105CA00053E8005FB5F1004F0DD14FF0000543E818
:105CB0000056012EF4D04EF60450CEF200000168DA
:105CC00041F080510160BFF32F8F14420CBF0020C0
:105CD000012070BC704700BF4DF27023C0F6030373
:105CE000185C704708B54FF0000040F25851C2F2FE
:105CF0000001FAF7A7FD003018BF012008BD00BF62
:105D000010B50446FBF77AFC40F2AC13C2F2000374
:105D100053F82410484010BD10B504464FF0010060
:105D2000FFF73AFF4DF2FC13C0F6030353F834209B
:105D300040F26051C2F200010A6003EBC4046068E3
:105D400040F28853C2F20003186010BD00B585B060
:105D50004FF00000FFF7E0FF4FF00003009340F228
:105D60008C52C2F2000201924FF0400002904DF2BC
:105D70005420C0F603004FF0020145F62162C0F640
:105D8000020202F07FF840F29063C2F20003186052
:105D900005B000BD2DE9F001804600283CD04FF051
:105DA00000034FEA8302086850F823404D6855F815
:105DB000236086EA0407886850F8235084EA050CBB
:105DC0004CEA07076FEA070CC86850F8235026EA28
:105DD000050707EA0C0705EA0C0C66EA0C063540D5
:105DE00040F82350CD6855F82300384345F8230088
:105DF0000D6955F82300384345F823004D690DB16E
:105E000045F82370486885588868855048688450EC
:105E100003F101034345C4D1BDE8F001704700BF61
:105E20002DE9F84340F26058C2F2000840F28C6657
:105E3000C2F2000640F28C44C2F200044FF00005AA
:105E400040F28857C2F20007D8F8000000EB80004B
:105E500002F076F93368002B40F00B822046294689
:105E60004FF0240214F0BCF903E24FF009004DF2A8
:105E7000C011C0F60301FFF78DFF40F25C53C2F280
:105E80000003197859B101F1FF3040F25C52C2F2BF
:105E90000002107040F29463C2F200031D6040F2F1
:105EA0005851C2F200010868E8B940F25852C2F2F3
:105EB0000002156040F21C53C2F20003197849B980
:105EC00040F25851C2F20001086860B1284606F05D
:105ED000E7FC08E040F25850C2F20000026842F0CD
:105EE00000630360ECE740F25C52C2F200021378F8
:105EF0005BB103F1FF3140F25C50C2F2000001706F
:105F000040F29462C2F20002556040F25853C2F26D
:105F10000003196841BB4DF2D810C0F60300426877
:105F200040F2B043C2F2000359680A4040F25850B0
:105F3000C2F20000026040F21C52C2F2000213786A
:105F40004BB940F25853C2F20003196861B12846B8
:105F500006F0A6FC08E040F25851C2F200010868C1
:105F600040F000620A60ECE740F25C50C2F20000D0
:105F700002785AB102F1FF3340F25C51C2F20001E3
:105F80000B7040F29460C2F20000856040F25852FB
:105F9000C2F200021368EBB940F25851C2F200019C
:105FA0000D6040F21C50C2F2000002784AB940F283
:105FB0005852C2F20002136863B1284606F070FC22
:105FC00008E040F25853C2F20003196841F0006043
:105FD0001860ECE740F25C51C2F20001087858B159
:105FE00000F1FF3340F25C52C2F20002137040F243
:105FF0009461C2F20001CD6040F25850C2F200003C
:106000000368EBB940F25852C2F20002156040F248
:106010001C51C2F20001087848B940F25850C2F24F
:106020000000036863B1284606F03AFC08E040F23D
:106030005853C2F200031A6842F000611960ECE79D
:1060400040F25C52C2F20002117859B101F1FF3006
:1060500040F25C53C2F20003187040F29462C2F244
:106060000002156140F25851C2F20001086840BBBD
:106070004DF2D813C0F603031A6940F2B041C2F2E0
:1060800000010869024040F25853C2F200031A604E
:1060900040F21C52C2F20002117849B940F2585144
:1060A000C2F20001086860B1284606F0F9FB08E07A
:1060B00040F25850C2F20000036843F000620260F0
:1060C000ECE740F25C53C2F200031A785AB102F1D5
:1060D000FF3140F25C50C2F20000017040F2946364
:1060E000C2F200035D6140F25852C2F20002116830
:1060F000E9B940F25850C2F20000056040F21C536A
:10610000C2F200031A784AB940F25852C2F20002B1
:10611000116861B1284606F0C3FB08E040F258510F
:10612000C2F20001086840F000630B60ECE740F247
:106130005C50C2F2000003785BB103F1FF3140F222
:106140005C52C2F20002117040F29460C2F2000090
:10615000856140F25853C2F200031968E9B940F270
:106160005852C2F20002156040F21C50C2F2000008
:1061700003784BB940F25853C2F20003196861B179
:10618000284606F08DFB08E040F25851C2F20001AB
:106190000A6842F000600860ECE740F25C52C2F22C
:1061A0000002107858B100F1FF3340F25C51C2F2A6
:1061B00000010B7040F29462C2F20002D56140F21D
:1061C0005850C2F200000368EBB940F25851C2F2D5
:1061D00000010D6040F21C52C2F20002107848B972
:1061E00040F25850C2F20000036863B1284606F03E
:1061F00057FB08E040F25853C2F20003196841F01F
:1062000000621A60ECE740F25C51C2F200010A78C9
:106210005AB102F1FF3040F25C53C2F20003187031
:1062200040F29461C2F200010D6240F25852C2F293
:1062300000021068D8B940F25853C2F200031D6042
:1062400040F21C51C2F200010A783AB140F25850B3
:10625000C2F20000036843F00061016040F258524E
:10626000C2F20002106810B1284606F019FB356032
:10627000EAE5D4F800902846FFF742FD40EA09011C
:106280002160D4F804904FF00100FFF739FD40EA97
:1062900009026260D4F808904FF00200FFF730FD69
:1062A00040EA0900A060D4F80C904FF00300FFF71B
:1062B00027FD40EA0903E360D4F810904FF0040092
:1062C000FFF71EFD40EA09012161D4F814904FF058
:1062D0000500FFF715FD40EA09026261D4F8189045
:1062E0004FF00600FFF70CFD40EA0900A061D4F86A
:1062F0001C904FF00700FFF703FD40EA0903E3613C
:10630000D4F820904FF00800FFF7FAFC40EA0901AA
:106310002162306800F1010030603A689042FFF479
:1063200093ADA2E500B585B04FF00003009340F2B5
:10633000FC62C2F2000201924FF0400002904DF266
:106340008030C0F603004FF0060146F26532C0F619
:10635000020201F097FD40F2B863C2F20003186038
:1063600005B000BD2DE9F04F85B040F66C031E4628
:10637000C2F2000640F624000746C2F2000740F2CF
:10638000D861C2F20001019101F012FD3268002AC9
:10639000FAD061E1E359002B53D02846FFF7B0FC57
:1063A00001996258605090434BD0E35910EA0302C0
:1063B00047D0039991F800E04DF28839C0F60309FF
:1063C0004FEA451840F2BC61C2F200014FF6FF7C73
:1063D0004DF2802AC0F6030A40F6000BC2F2000B11
:1063E00000957046C2F10003134022EA030218B977
:1063F00054F80B502B4221D15FEA136E04D01AF8E7
:106400000E3003F118030EE01D0C04D01AF805300D
:1064100003F1100307E05FEA132E1ABF1AF80E30DB
:1064200008331AF80330434419F8035031F815E0E3
:10643000E6451CBF0EF1010E21F815E0002AD1D16E
:10644000009D05F1010504F10404092DA2D1029C6F
:10645000621E029240F0F7800399087800F1010073
:10646000C3B20B700B2B03D14FF000040C7002E091
:10647000002B40F0E58040F64802C2F200021168AD
:1064800091B16FEA01003B6803403B6040F60005B4
:10649000C2F200052C682040286040F64801C2F294
:1064A00000014FF000020A6040F64800C2F200000E
:1064B000436893B16FEA03057C682C407C6040F62A
:1064C0000002C2F2000251680D40556040F64800DB
:1064D000C2F200004FF00003436040F64805C2F2EC
:1064E0000005AC6894B16FEA0400BA680240BA6073
:1064F00040F60003C2F2000399680840986040F635
:106500004805C2F200054FF00004AC6040F64800B8
:10651000C2F20000C26892B16FEA0203F968194042
:10652000F96040F60005C2F20005EC682340EB601C
:1065300040F64800C2F200004FF00002C26040F690
:106540004803C2F20003196991B16FEA01053C6981
:106550002C403C6140F60000C2F200000269154088
:10656000056140F64803C2F200034FF000011961D3
:1065700040F64805C2F200056C6994B16FEA040068
:106580007A6902407A6140F60003C2F20003596959
:106590000840586140F64805C2F200054FF000047B
:1065A0006C6140F64800C2F20000826992B16FEA65
:1065B0000203B9691940B96140F60005C2F200054D
:1065C000AC692340AB6140F64800C2F200004FF0D6
:1065D0000002826140F64803C2F20003D96991B11A
:1065E0006FEA0105FC692C40FC6140F60000C2F234
:1065F0000000C2691540C56140F64803C2F20003BD
:106600004FF00001D96140F64805C2F200052C6A3E
:1066100094B16FEA04003A6A02403A6240F600031D
:10662000C2F20003196A0840186240F64805C2F237
:1066300000054FF000042C624FF4FA70029002E063
:106640004FF4FA7502954FF0010001F079FD3268C0
:10665000002A3FF499AE07E04FF4FA75029540F234
:10666000FC74C2F2000403944FF00004254691E646
:1066700010B54FF0000440F66C03C2F200031C603A
:1066800040F60000C2F2000021464FF00902FAF77E
:10669000E5F840F62400C2F2000021464FF009025E
:1066A000FAF7DCF840F64800C2F2000021464FF04D
:1066B0000902FAF7D3F840F2D860C2F2000021468E
:1066C0004FF00902FAF7CAF840F2BC60C2F20000CB
:1066D00021464FF01A0213F083FD40F2FC70C2F223
:1066E0000000047010BD00BF70B54DF26023C0F60D
:1066F00003031B5C4DF21C22C0F6030252F820205B
:1067000040F66C00C2F20000046840F62405C2F2B4
:10671000000555F82300104206D104F1010640F6A9
:106720006C05C2F200052E6049B140F60001C2F2CC
:10673000000151F82350154341F8235009E040F679
:106740000001C2F2000151F8235025EA020541F888
:106750002350104340F62401C2F2000141F8230007
:1067600040F64801C2F2000151F8230020EA02027B
:1067700041F8232034B940F2B863C2F2000318682C
:1067800001F048FB70BD00BF30B44DF26023C0F68D
:1067900003031B5C4DF21C22C0F6030252F82020BA
:1067A00040F62400C2F2000050F82300104229D025
:1067B00040F66C04C2F20004256805F1010525606D
:1067C00071B140F64801C2F2000151F82340144370
:1067D00041F8234040F2FC71C2F20001097889B906
:1067E0006FEA020240F60001C2F2000151F82340B4
:1067F000144041F82340024040F62400C2F2000059
:1068000040F8232030BC704730B4034640F65012A5
:10681000C2F2000252E8000F00F1010042E8000459
:10682000012CF7D040F2BC60C2F2000030F8132017
:1068300039B140F2BC61C2F200014FF0000421F80E
:10684000134040F65013C2F2000353E8004FA4F186
:10685000010443E80045012DF7D053E8004FB4F19F
:10686000004F0DD14FF0000443E80045012DF4D056
:106870004EF60450CEF20000016841F080510160F4
:10688000BFF32F8F104630BC704700BF40F2FC733F
:10689000C2F200031878D0F1010038BF0020704721
:1068A0002DE9F84FDFF834814B4FC8EB07004FEA72
:1068B000D00707F101074FF0000540F2982AC0F613
:1068C000000A40F28039C0F6000931E044464FF03A
:1068D00000066FEA060B0BEB070101F0010B58F8FD
:1068E000043CAB4229D135E054F8043CAB4205D11D
:1068F00054F8080C8047FBF787FD0BE0FF2B09D904
:10690000FF2D07D154F8040C4FF0070154F8082C60
:1069100001F0D8FB06F1010604F1080454F8041C48
:10692000A94240D14CE005F10105B5F5807F02D0C8
:10693000CA45CBD3F7E7BDE8F88FFF2B0FD9FF2D62
:106940000DD158F8040C4FF0070158F8082C01F04D
:10695000B9FB04E058F8082C9047FBF755FD06F109
:10696000010604F10804BE42DDD0BBF1000FBBD02C
:1069700054F8040CA8420AD0FF280DD9FF2D0BD1E2
:106980004FF0070154F8082C01F09CFB04E054F888
:10699000081C8847FBF738FD06F1010604F10804DE
:1069A000BE42A1D1BFE7FF290FD9FF2D0DD154F869
:1069B000040C4FF0070154F8082C01F083FB04E0AD
:1069C00054F8082C9047FBF71FFD06F1010604F16F
:1069D0000804BE4288D1A6E787030008A002000889
:1069E000027840F6E903C2F200031B789A4206D30C
:1069F0004FF000020270087800F1010008700A7878
:106A000040F6EA03C2F200031878824224BF002055
:106A10000870704738B140F61840C4F202004FF0D9
:106A200002010180704740F61A43C4F202034FF09E
:106A300002021A80704700BF08B540F61843C4F23E
:106A400002034FF008021A8000EA0201CBB23BB108
:106A500040F61843C4F202034FF08001198006E0AB
:106A600040F61A41C4F202014FF080020A8000F0A1
:106A70000402D3B23BB140F61841C4F202014FF018
:106A800040030B8006E040F61A41C4F202014FF0C9
:106A900040020A8010F0010F19BF40F61841C4F2FD
:106AA000020140F61A41C4F202014FF010020A80BE
:106AB00000F00200C1B239B140F61840C4F2020041
:106AC0004FF02001018006E040F61A43C4F20203B1
:106AD0004FF020021A804FF0010003F081FA40F6D7
:106AE0001A43C4F202034FF008021A8008BD00BF27
:106AF00010B50C46FFF78EFF40F61843C4F20203B0
:106B00004FF008021A8014F0800F19BF40F61843A6
:106B1000C4F2020340F61A43C4F202034FF08000AD
:106B2000188004F04001CBB23BB140F61841C4F2EA
:106B300002014FF040030B8006E040F61A40C4F219
:106B400002004FF04002028004F01000C2B23AB1DD
:106B500040F61840C4F202004FF01002028006E036
:106B600040F61A41C4F202014FF010030B8004F00A
:106B70002001CBB23BB140F61841C4F202014FF004
:106B800020030B8006E040F61A40C4F202004FF0EA
:106B9000200202804FF0010003F022FA40F61A4072
:106BA000C4F202004FF0080202802046FFF744FFC3
:106BB0004FF0320003F014FA10BD00BF08B50329EE
:106BC00014D8DFE801F0020B05084FF0800107E060
:106BD0004FF0940104E04FF0D40101E04FF0C00108
:106BE0000A184FF00000D1B2FFF782FF08BD00BFC6
:106BF00008B540F6FB03C2F20003187830B940F63E
:106C0000F001C2F20001086801F004F940F6FB034C
:106C1000C2F200034FF002021A7008BD10B5A0F1D5
:106C20000803052B3DD8DFE803F01F3C2C3C03850F
:106C300040F68400C2F200004FF020014FF05402F1
:106C400013F0CEFA40F6DC00C2F200004FF0FF3144
:106C50004FF00C0213F0C4FA40F6F400C2F2000048
:106C6000026802F1010202604FF0000140F6780371
:106C7000C2F20003197040F67900C2F20000017000
:106C800056E040F67801C2F200014FF000030B70AD
:106C900040F67900C2F20000027802F101020270AF
:106CA0003CE040F67802C2F20002127840F6790128
:106CB000C2F200010B7840F6E901C2F20001097846
:106CC00001FB032340F68401C2F20001C95C81424A
:106CD0001DD040F68404C2F20004E0544FEA531081
:106CE00040F6DC01C2F2000103F01F034FF0010483
:106CF00004FA03F351F820401C4341F8204040F6C9
:106D0000F400C2F20000016801F10101016002F12A
:106D1000010240F67803C2F200031A7040F67800D0
:106D2000C2F2000040F67901C2F20001FFF758FEFE
:106D3000FFF75EFF4FF0000010BD00BF70B4039D71
:106D4000049C064628B140F6EB00C2F20000007831
:106D5000307029B140F6F900C2F2000000780870E6
:106D60002AB140F6E801C2F20001087810702BB198
:106D700040F6FA02C2F20002117819702DB140F605
:106D80007803C2F20003187828702CB140F679021B
:106D9000C2F200021178217070BC704707281DD81C
:106DA000002808BF022040F6EB03C2F2000318706F
:106DB0004DF2AC43C0F6030313F8101040F6E9029D
:106DC000C2F20002117003EB4000417840F6EA0382
:106DD000C2F2000319704FF0010070474FF000003D
:106DE000704700BF10B540F6F903C2F200034FF040
:106DF00001021A704FF00200FFF7D0FF4FF00004BD
:106E000040F67C00C2F20000046040F6EC01C2F2E1
:106E100000010C604DF2A840C0F603004FF087015E
:106E200047F28932C0F6020201F04CF940F6F00355
:106E3000C2F2000318604FF00C002146FFF7EEFE8F
:106E400010BD00BF034628B140F6E900C2F20000C1
:106E50000078187029B140F6EA03C2F200031878EE
:106E600008702AB140F6F401C2F200010B68136009
:106E700040F68400C2F20000704700BF2DE9F041E7
:106E800040F68407C2F200073F1853284DD8002A65
:106E90004BD03B4607F1010702F1FF3257FA82F768
:106EA0004FF0000640F6DC04C2F200044FF001058A
:106EB0006FEA030C0CEB070202EA050C13F8018BD6
:106EC00001F1FF3111F8012F904530D13EE013F868
:106ED00001CB01F1010049788C450ED003F8011C6B
:106EE0004FEA521102F01F0605FA06FC54F8216021
:106EF0004CEA060644F821602E4602F10102D2B2A5
:106F0000542A07D013F801CB00F1010140788445E1
:106F100043D151E04EB140F6F403C2F200031968C8
:106F200001F101011960FFF763FEBDE8F08103F88C
:106F3000012C4FEA501600F01F0805FA08F854F823
:106F4000262048EA020244F826202E4600F10100DD
:106F5000C2B2542ADED0BB42DCD0BCF1000FB6D0A6
:106F600013F801CB11F8010F84450ED003F8010C82
:106F70004FEA521002F01F0605FA06FC54F8206092
:106F80004CEA060644F820602E4602F10102D2B215
:106F9000542ABFD0BB429AD1BCE703F8010C4FEA98
:106FA000521002F01F0605FA06FC54F820604CEA65
:106FB000060644F820602E4602F10102D2B2542A9D
:106FC000A8D0BB4283D1A5E740F6D803C2F20003A4
:106FD0004FF000021A7070474FF05400704700BF26
:106FE00038B540F6D803C2F20003187868B14FF004
:106FF000050540F6D804C2F20004FBF705FA28465E
:1070000001F09EF821780029F7D140F6D803C2F2AA
:1070100000034FF001021A7038BD00BF38B54FF0C1
:10702000000240F6EC03C2F200031868B0F1FF3F23
:1070300000F0CE8010B140F001010847FFF7D0FF0B
:1070400040F6FB00C2F200004FF0010202704FF068
:10705000000340F67401C2F200010B6040F6F80034
:10706000C2F20000037089E040F67003C2F2000330
:107070004FF000021A704FF001026BE040F6740509
:10708000C2F200052B684FF0010103F01F0401FA62
:1070900004F44FEA531340F6DC05C2F2000555F83C
:1070A00023301C4245D0AAB140F6F801C2F20001DB
:1070B0000978FFF783FD40F6EC00C2F20000494B6F
:1070C00003604FF0010038BD40F6EC04C2F200044A
:1070D000444A226040F67404C2F2000421684FF072
:1070E000010040F68402C2F20002515CFFF700FD8D
:1070F00020684FEA501240F6DC03C2F2000300F0B1
:107100001F044FF0010000FA04F153F8224024EA72
:10711000010443F8224040F6EC03C2F20003324A75
:107120001A6038BD40F6EC03C2F200032E48186026
:1071300000E00A4640F67003C2F20003197801F13C
:107140000101197040F67400C2F20000036803F1F7
:107150000103036040F67001C2F20001087840F6B6
:10716000E903C2F200031978814287D840F6F8009B
:10717000C2F20000027802F10102027040F6F80348
:10718000C2F20003197840F6EA00C2F20000027869
:107190009142FFF469AF40F6FB03C2F20003197895
:1071A00001297FF44DAF40F6FB00C2F200004FF022
:1071B0000002027040F67803C2F20003187840F62D
:1071C0007901C2F200010978FFF7F8FCFFF7FCFE35
:1071D00040F6EC01C2F200014FF000020A604FF0ED
:1071E000030038BDC87002082471020808B50030D9
:1071F00018BF012040F6F903C2F2000318700031F5
:1072000018BF012140F6E800C2F200000170003210
:1072100018BF012240F6FA03C2F200031A70FFF70A
:10722000DFFE40F68001C2F20001087800B340F6AC
:10723000F902C2F200021378002B14BF04200020D0
:1072400040F6E801C2F200010A78002A14BF0223C6
:10725000002340F6FA01C2F200010A78002A14BFA6
:107260000921082101434FF000001943FFF740FCBA
:10727000FFF7AAFE08BD00BF10B540F60043C4F2F8
:1072800002031A684FF0010464F387121A60186849
:1072900064F383001860196864F3092119601A689F
:1072A00064F38B221A60186864F30D301860196853
:1072B00064F38F3119604FF00000FFF7ABFB4FF024
:1072C0000300FFF7B9FB41F2040002F089FE4FF022
:1072D0000300FFF7B1FB4FF0640002F081FE4FF0B6
:1072E0000300FFF7A9FB4FF0320002F079FE4FF0E8
:1072F0000200FFF7A1FB4FF0320002F071FEFFF732
:107300006FFE4FF000004FF02801FFF7F1FB4FF048
:1073100000004FF00601FFF7EBFBFFF755FE40F6CC
:107320008003C2F200031C7040F6F902C2F20002B0
:10733000107840F6E801C2F20001097840F6FA033D
:10734000C2F200031A78FFF751FFFFF749FE4FF032
:1073500000002146FFF7CCFB40F2A46002F040FEA3
:10736000FFF732FEFFF73CFE40F67800C2F2000065
:10737000007840F67902C2F200021178FFF71EFC95
:10738000FFF722FE10BD00BF10B540F6FB03C2F2AE
:1073900000034FF001021A704FF47A7000F0D0FE33
:1073A000FFF76AFF4FF0020402E0204600F0C8FE3B
:1073B000FFF734FE0128F8D000F0FAFCF8E700BF30
:1073C0002DE9F04180460C46174640F68003C2F294
:1073D0000003187868B94FF0320640F68005C2F213
:1073E0000005FBF711F8304600F0AAFE29780029C5
:1073F000F7D04FF4FA6002F0F3FDFFF7F1FD4FF024
:10740000000048F04001FFF773FB4FF0320002F03C
:10741000E7FD4FEAC702D3B203F1FF37FFB2FBB17A
:1074200007F10107E7194FF001066FEA0405781923
:1074300000EA0605304614F8011BFFF759FBBC4271
:1074400022D10DE0254615F8011B3046FFF750FB11
:10745000617805F101043046FFF74AFBBC42F1D1E7
:1074600040F67001C2F20001087840F6F802C2F25C
:1074700000021178FFF7A2FB4FF0320002F0B0FDDE
:10748000FFF7A2FDBDE8F081002DDBD0304614F8F7
:10749000011BFFF72DFBBC42D4D1E1E708B540F654
:1074A0007802C2F20002107040F67903C2F20003C3
:1074B000197010461946FFF793FA40F6E800C2F239
:1074C0000000017879B1FFF78BFD40F67802C2F237
:1074D0000002107840F67903C2F200031978FFF732
:1074E0006DFBFFF771FD08BD10B5044640F6FC00CA
:1074F000C2F2000001F0C2F92CB140F62B10C2F22A
:107500000000017804E040F62A13C2F20003197863
:1075100040F62812C2F20002117040F62913C2F29E
:1075200000031C704FF00300FBF774F810BD00BFA0
:1075300010B582B040F62414C2F200042068003076
:1075400018BF0120FFF7D0FF216879B14FF0000389
:107550000093019340F6FC00C2F200004FF0FF02DE
:1075600047F2E943C0F6020301F02EFA02B010BD63
:1075700010B5082824DC082925DC002804DB40F6A7
:107580002A14C2F200042070002904DB40F62B10FC
:10759000C2F200000170002A08DBC2EB02124FEABF
:1075A000820040F62411C2F20001086040F6201269
:1075B000C2F200021370FFF7BBFF4FF0010010BDD5
:1075C0004FF0000010BD4FF0000010BD40F6281332
:1075D000C2F2000318787047034628B10868834256
:1075E00014BF0020012070474FF00000704700BF1B
:1075F00010B440F65013C2F2000353E8002F02F11A
:10760000010243E800210129F7D00468C4B162688F
:10761000824202D19268626002E0436881689960A8
:107620002368834202D15B68236002E0826841687C
:107630005160A26802F1FF31A1604FF000040460C4
:1076400040F65013C2F2000353E8002FA2F10102EA
:1076500043E80024012CF7D053E8002FB2F1004F8B
:107660000DD14FF0000243E80024012CF4D04EF677
:107670000450CEF20000016841F080510160BFF378
:107680002F8F10BC704700BF38B504460D464FF031
:1076900000014FF0100212F0A3FDE56038BD00BFFD
:1076A000F8B504460F46C6688D192946FFF794FFC2
:1076B00000283CD140F65013C2F2000353E8002FDB
:1076C00002F1010243E800210129F7D04FF0000048
:1076D00068606168A96001B14D60226802B92560E7
:1076E0006560BC51A36803F10103A36040F6501329
:1076F000C2F2000353E8002FA2F1010243E8002484
:10770000012CF7D053E8002FB2F1004F0DD14FF00C
:10771000000243E80024012CF4D04EF60450CEF2CF
:107720000000016841F080510160BFF32F8FF8BD68
:107730002DE9F04104468846C6688D199719C2B9EB
:1077400040F65013C2F2000353E8002F02F1010289
:1077500043E800210129F7D002686A6005604FF014
:107760000000A860616809B9656020E06B689D60F1
:107770001DE03946FFF730FF00283FD02846FFF7CD
:1077800037FF40F65013C2F2000353E8002F02F116
:10779000010243E800210129F7D0B868A8606F60B2
:1077A000BD602168B9420EBF2560A9684D6048F8E8
:1077B0000640A26802F10102A26040F65013C2F234
:1077C000000353E8002FA2F1010243E80024012C3A
:1077D000F7D053E8002FB2F1004F0DD14FF0000267
:1077E00043E80024012CF4D04EF60450CEF2000001
:1077F000016841F080510160BFF32F8FBDE8F08137
:10780000C368C918486808B1C01A70474FF0000033
:10781000704700BF036813B1C068181A70474FF073
:107820000000704708B5C368C918FFF7D5FE08BD4A
:1078300008B5C0680818FFF7DBFE08BD08B540F6BC
:107840002C10C2F200004FF01C01FFF71DFF08BD15
:1078500070B5054600F108063046FFF7DBFF044629
:10786000686050B130462146FFF7E2FF4FF001005B
:10787000A861204600F0CEFA70BD4FF00003AB6166
:1078800070BD00BF38B504460D464FF000014FF003
:10789000280212F0A5FC204640F8085B4FF01C01BE
:1078A000FFF7F2FE40F62C10C2F200002146FFF76F
:1078B000F7FE38BD2DE9F0410746884643F25453A0
:1078C000C2F200031868002800F0FE8040F6501451
:1078D000C2F2000454E8002F02F1010244E8002142
:1078E0000129F7D0796831B143F25452C2F2000253
:1078F000136899422ED143F25450C2F2000004683A
:107900007C60B96901F10101B96140F65013C2F21E
:10791000000353E8002FA2F1010243E80024012CE8
:10792000F7D053E8002FB2F1004F0DD14FF0000215
:1079300043E80024012CF4D04EF60450CEF20000AF
:10794000016841F080510160BFF32F8F4FF00100BB
:10795000BDE8F081B8F1FF3F24D140F65013C2F2E8
:10796000000353E8002FA2F1010243E80024012C98
:10797000F7D053E8002FB2F1004F0DD14FF00002C5
:1079800043E80024012CF4D04EF60450CEF200005F
:10799000016841F080510160BFF32F8F4FF000006C
:1079A000BDE8F08107F108052846FFF733FF0246DE
:1079B000F0B143F25456C2F20006306892F8294002
:1079C00090F829108C4208D912E0336892F8290007
:1079D00093F82940A04204D90AE043F25456C2F277
:1079E000000628461146FFF70BFF02460028ECD19F
:1079F000284643F25451C2F200010968FFF798FE8D
:107A000040F65016C2F2000656E8002FA2F101021D
:107A100046E80024012CF7D056E8002FB2F1004FC1
:107A20000DD14FF0000246E80024012CF4D04EF6B0
:107A30000450CEF20000016841F080510160BFF3B4
:107A40002F8FB8F1000F04D008EB880000F078FB0E
:107A500001E000F0ADF940F65014C2F2000454E821
:107A6000003F03F1010344E80032012AF7D043F25A
:107A70005456C2F2000628463168FFF7D9FE54E892
:107A8000003FA3F1010344E80032012AF7D054E893
:107A9000003FB3F1004F0DD14FF0000344E8003236
:107AA000012AF4D04EF60450CEF20000016841F0F5
:107AB00080510160BFF32F8F78683268904214BF05
:107AC00000200120BDE8F0814FF00100BDE8F08109
:107AD00010B5044643F25453C2F20003186800285C
:107AE00060D06268904201D0F8F7A8FE40F65013CB
:107AF000C2F2000353E8002F02F1010243E8002123
:107B00000129F7D0A16901F1FF30A06118B340F657
:107B10005013C2F2000353E8002FA2F1010243E820
:107B20000024012CF7D053E8002FB2F1004F0DD103
:107B30004FF0000243E80024012CF4D04EF604502C
:107B4000CEF20000016841F080510160BFF32F8F39
:107B50004FF0000010BD2046FFF77AFE40F65013AC
:107B6000C2F2000353E8002FA2F1010243E800240F
:107B7000012CF7D053E8002FB2F1004F0DD14FF098
:107B8000000243E80024012CF4D04EF60450CEF25B
:107B90000000016841F080510160BFF32F8F4FF06A
:107BA000010010BD4FF0010010BD00BFF8B5054643
:107BB00040F65013C2F2000353E8002F02F1010215
:107BC00043E800210129F7D040F62C10C2F2000052
:107BD000FFF720FE0446E0B140F62C17C2F2000782
:107BE0006068A84203D12046FFF732FE0AE004F1A4
:107BF000080630462946FFF715FE18B130462946DB
:107C0000FFF716FE38462146FFF7FAFD0446002826
:107C1000E6D140F65013C2F2000353E8002FA2F160
:107C2000010243E80024012CF7D053E8002FB2F101
:107C3000004F0DD14FF0000243E80024012CF4D096
:107C40004EF60450CEF20000016841F08051016010
:107C5000BFF32F8FF8BD00BF02282BD111F0030F07
:107C60001FD148F21F52C5F2EB12A2FB01204FEACE
:107C700050134FF0640202FB131083B2A3B948F211
:107C80001F52C5F2EB12A2FB01204FEAD0134FF4B2
:107C9000C87202FB131188B2D0F1010338BF002370
:107CA00004E04FF0000301E04FF0010303F11C0377
:107CB000D8B2704700F1FF3042F29343C9F2492332
:107CC00083FB00210B184FEAE072C2EBA301C1EB6A
:107CD000C103C21A4FF00101C8F20001114000298E
:107CE00005DA01F1FF3060F0010101F10101C1F19C
:107CF0001F03D8B2704700BF08B54DF2BC43C0F6B1
:107D00000303195C012906D011B102290BD105E04A
:107D1000FCF790FD08BD02F023F908BDF8F78EFDD1
:107D20004FF0000008BD4FF0000008BD4EF60453B0
:107D3000CEF200031A6842F080501860704700BF0E
:107D40004FF0010280F8282040F64C13C2F20003E5
:107D500090F8291002FA01F2188802431A8070473D
:107D600010B440F64813C2F200031A68C2B1904240
:107D700013D104E088420FD102F1140203E040F66F
:107D80004812C2F2000243691BB19C698169611803
:107D900099614369136003E00A4651690029E9D1FA
:107DA0004FF0000282614FF0FF31416110BC70471B
:107DB00010B5F8F799FD044643F25453C2F200039C
:107DC000186890F82820032A1BD0F8F78DFD43F29D
:107DD0005453C2F2000319684FF0000281F82820C2
:107DE00091F82920096940F63C23C2F2000343F8C8
:107DF0002210F8F783FD2046F8F780FDFFF796FF85
:107E000010BD4FF0020180F828102046F8F776FDEB
:107E100010BD00BF38B5044690B3036883B3F8F7CC
:107E200063FD054694F8280010BB2046FFF788FF45
:107E300043F25451C2F200010B6843B194F8292077
:107E400093F8290020F00101531A002B15DA40F6AF
:107E50005012C2F20002106838B140F0004140F602
:107E60005013C2F20003196007E0FFF75FFF04E060
:107E7000022804BF032084F828002846F8F73EFDB6
:107E800038BD00BF2DE9F04F85B006460F4693463A
:107E900098460F9DDDF84090F8F726FD824640F6A3
:107EA0009413C2F200031968504881420FD240F285
:107EB0000002C2F2020252F82C4C54B14C4B1C4648
:107EC0008B4207D953F82C090028F8D102E0474C1F
:107ED00000E0464CA14206D1A1F12C0140F69412DB
:107EE000C2F20002116020464FF000014FF02C0258
:107EF00012F076F94FF0FF3161611EB94DF2C046C4
:107F0000C0F603062660B8F1000F08D00E9B042BC4
:107F100008D9184600F103004FEA900604E04FF03C
:107F2000000601E04FF000060DBB44F25809C2F212
:107F3000000940F63C15C2F20005296848F2A1305C
:107F4000C0F602000090CDF80480029648464FF03B
:107F500000025B46F9F700F82A68A260E0604FEA89
:107F6000800153182B60C1EB0900606020E02846B7
:107F70004FF0FF314A46F8F771FC4AF2ED52CDF668
:107F8000CE622A60E56005EB8905656048F2A131A3
:107F9000C0F602010091CDF80480029628462946D9
:107FA0004FF001025B46F8F7D7FFA5EB8003636053
:107FB0006FEA0702C2F3C01101EB470707F0FF07A2
:107FC00084F8297040F65413C2F2000353F82700D6
:107FD000206143F827405046F8F790FC2046FFF711
:107FE00019FF204605B0BDE8F08F00BFD4FF012087
:107FF000A8FF012030B585B04FF0000143F2545383
:10800000C2F200031960284C40F20005C2F20205DA
:108010002A1B20464FEAA202F8F720FC40F63C104B
:10802000C2F200000460A5F12C0540F69411C2F2E2
:1080300000010D6043F65803C2F200034FF0B5048F
:10804000CBF26B141C6003F14C004FF0FF3243F88D
:10805000042F43F8042F43F8042F8342F9D14FF043
:108060000004009440F69811C2F2000101914FF013
:10807000280302934DF2CC40C0F603004FF00701F5
:1080800048F22112C0F602022346FFF7FBFE40F63B
:108090003822C2F20002106040F65410C2F2000012
:1080A000C46305B030BD00BF5C40002010B584B093
:1080B000069C00944FF0000401940294FFF7E2FE46
:1080C00004B010BD00B585B04FF0000300930193DC
:1080D0000293FFF7D7FE05B000BD00BF38B543F2ED
:1080E0005453C2F200031868C0B1F8F7FDFB05460F
:1080F00043F25454C2F200042068FFF721FE2168C5
:1081000091F82920086940F63C23C2F2000343F8A5
:1081100022002846F8F7F2FBFFF708FE38BD00BF43
:1081200038B543F25455C2F2000540F65414C2F279
:1081300000042B6822681A61FFF7D0FFF9E700BF3F
:1081400038B543F25453C2F200031968002900F015
:10815000918020B9FFF7C2FF4FF001029AE0B0F121
:10816000FF3F04D1FFF724FE4FF0000292E040F6FB
:108170005014C2F2000454E8002F02F1010244E856
:1081800000210129F7D040F64812C2F2000215681A
:10819000002D7AD0AB6998426FD3C01A05F1140153
:1081A0006D691DB1AB698342F7D96AE043F254555A
:1081B000C2F200052B689861086858611846F8F704
:1081C00041FB40F65014C2F2000454E8003FA3F112
:1081D000010344E80032012AF7D054E8003FB3F12C
:1081E000004F0DD14FF0000344E80032012AF4D0D3
:1081F0004EF60450CEF20000016841F0805101605B
:10820000BFF32F8FFFF7D4FD54E8003F03F10103C4
:1082100044E80032012AF7D028684169B1F1FF3FF4
:1082200004D0FFF79DFD4FF0000201E04FF0010286
:1082300040F65013C2F2000353E8004FA4F10104CA
:1082400043E80045012DF7D053E8004FB4F1004F4B
:108250000DD14FF0000443E80045012DF4D04EF657
:108260000450CEF20000016841F080510160BFF37C
:108270002F8F0FE04FF001020CE040F64811C2F2E0
:108280000001AC69221AAA6190E740F64811C2F2D7
:1082900000018BE7104638BDF8B5044600287AD0B7
:1082A000F8F722FB064640F69413C2F20003196861
:1082B0003948814211D240F20002C2F2020252F861
:1082C0001C5CA54263D0354B1D468B4205D9A3F1FA
:1082D0002C03D86BA042F7D15AE094F8293040F62D
:1082E0005412C2F2000252F82300A04206D10169E2
:1082F00040F65412C2F2000242F823102046FFF763
:108300002FFD2046FFF752FC94F82900236940F620
:108310003C21C2F2000141F8203043F25452C2F233
:1083200000021068A04229D0A06838B3E76800EBCB
:10833000870540F63C17C2F200073B685A1B2946E6
:108340004FEAA2024FF00003FBF762F8E1683868D9
:10835000A0EB81033B6040F69412C2F20002116868
:108360000D4B99420AD29A68954203D8E068A2EB75
:1083700080029A60A3F12C038B42F4D84FF00001E5
:10838000216084F828103046F8F7B8FAF8BD024D9D
:1083900021692961A1E7F8BDD4FF0120A8FF0120D0
:1083A00000BFF04772B643F25454C2F20004206892
:1083B000FFF772FF4FF000032360F8F71DFE00BFC8
:1083C00040F64813C2F20003196849B1886950B1F8
:1083D00000F1FF328A61D2F1010038BF00207047FE
:1083E0004FF0000070474FF00000704770B540F646
:1083F0004813C2F200031C68A4B1A06990B940F60A
:108400004815C2F200054FF0FF3660692946F8F7BB
:1084100019FA66612046FFF7FDFC2C6814B1A169CA
:108420000029F2D070BD00BFF0B472B640F64C1314
:10843000C2F200031C882CB940F63823C2F20003B4
:1084400018685FE04DF2D44CC0F6030C40F63C25B2
:10845000C2F2000540F65416C2F20006C4F1000351
:1084600023401A0A1ABF1CF8021008311CF8031026
:1084700011F0010F0AD141F0010055F8200038B188
:1084800090F82820012A38D81F4602E01F4600E055
:108490001F4655F82120B2B192F828307BB140F642
:1084A0004C10C2F20000048010462BE090F82830F7
:1084B00033B140F64C12C2F20002148022E01046A2
:1084C00000690028F2D156F82100824207D1BC434E
:1084D000C4D140F64C11C2F200010C80ACE745F863
:1084E000210011F0010FD4D114EA4703D1D04FEA93
:1084F0004707BFB241F00101CBE740F64C11C2F291
:1085000000010C8062B6F0BC704700BF70B543F24A
:108510005453C2F200031B6883420FD193F8282002
:10852000012A9CBF022283F8282093F8291040F6E4
:108530003C20C2F2000040F8213070BD40F64012ED
:10854000C2F20002136043F25451C2F2000108600B
:1085500090F8292040F63C23C2F2000343F82200A1
:1085600090F8281001299CBF022180F82810826809
:10857000AAB9C1684AF2ED53CDF6CE6308689842B5
:1085800001D0F8F75BF943F25452C2F200021168CD
:108590004868CB6898427ED2F8F750F970BD40F633
:1085A0004413C2F200031B68984274D093B3586816
:1085B00044F25804C2F20004251A4FEAA501D9601A
:1085C00043F65802C2F2000290420AD34FF0B503BC
:1085D000CBF26B1343F65800C2F2000004689C42D1
:1085E00001D0F8F72BF940F64415C2F200052A68CD
:1085F00040F63C14C2F2000420685168D2684FF083
:108600000003FAF705FF296823688B60C86803EB4D
:108610008002226043F25451C2F200010B6840F61E
:108620004410C2F200000360DA68002A33D05868B0
:1086300099684FF00103FAF7EBFE43F25456C2F289
:1086400000063568A868EC6800EB840440F63C1628
:10865000C2F200063268131B21464FEAA3024FF014
:108660000003FAF7D5FEE9683068A0EB81023260BA
:1086700040F69413C2F200031968074B99420AD2DC
:108680009A68944203D8E868A2EB80029A60A3F14A
:108690002C038B42F4D870BDD4FF012000B585B007
:1086A00040F6D830C2F200004FF00001FEF7ECFFB8
:1086B00040F68020C2F200004FF00001FEF7E4FF18
:1086C0004FF00003009340F69822C2F2000201929C
:1086D0004FF0500002904DF2D450C0F603001946FE
:1086E00048F61922C0F60202FFF7CCFB40F67C23C5
:1086F000C2F20003186005B000BD00BF08B5FFF767
:1087000089F8034648B1C06850B100F1FF31D96023
:10871000D1F1010038BF002008BD4FF0000008BDB6
:108720004FF0000008BD00BF70B505460E46144668
:1087300040F65013C2F2000353E8002F02F1010289
:1087400043E800210129F7D0FFF764F8024600282A
:1087500039D0C06884422DD3241A28461146FFF729
:108760004FF8024600282ED0C068A042F4D921E07C
:1087700040F65013C2F2000353E8002FA2F10102A9
:1087800043E80024012CF7D053E8002FB2F1004F4A
:108790000DD14FF0000243E80024012CF4D04EF636
:1087A0000450CEF20000016841F080510160BFF337
:1087B0002F8F70BDF460D1680B1BD3602846314603
:1087C000FEF7B6FFD4E7F46028463146FEF768FFAF
:1087D000CEE700BFF8B50646FFF71CF80446F8B12F
:1087E000C368EBB930462146FFF70AF80546F8F7AB
:1087F0007BF8074630462146FFF71AF83846F8F767
:108800007DF822691AB130462146FFF78DFF04F149
:108810001400FDF769F91DB12C46E8680028E1D085
:10882000F8BD00BF08B540F69423C2F200031A68F1
:1088300002F101021A6040F68020C2F20000FFF748
:108840005DFF28B140F68020C2F20000FFF7C2FFB2
:1088500008BD00BF08B5014640F6D830C2F200009E
:10886000FEF7E0FF20B140F6D830C2F2000008BDAC
:1088700040F68020C2F2000008BD00BF70B504467B
:1088800040F65013C2F2000353E8002F02F1010238
:1088900043E800210129F7D0FFF7DCFF0546214618
:1088A000FEF7C0FF002845D040F65010C2F200008D
:1088B00050E8002F02F1010240E800210129F7D021
:1088C00028462146FEF79CFF18B1C168E2688B1864
:1088D000C360F8F709F8064628462146FEF7A8FFC8
:1088E0003046F8F70BF84FF0FF35E56040F65013CF
:1088F000C2F2000353E8002FA2F1010243E8002571
:10890000012DF7D053E8002FB2F1004F0DD14FF0F9
:10891000000243E80025012DF4D04EF60450CEF2BB
:108920000000016841F080510160BFF32F8F4FF0CC
:10893000010501E04FF0000504F11400FDF7CEF849
:1089400040F65013C2F2000353E8002FA2F10102D7
:1089500043E80024012CF7D053E8002FB2F1004F78
:108960000DD14FF0000243E80024012CF4D04EF664
:108970000450CEF20000016841F080510160BFF365
:108980002F8F284670BD00BF2DE9F04105460F46E8
:1089900014469846FFF772FF064694B19DF82030C2
:1089A000002B14BF20460020286105F11400414629
:1089B000069A079BFDF778F8384629462246FFF7C6
:1089C000B3FE3046BDE8F08170B584B00E46154662
:1089D0000093089C01949DF82430029340F6802176
:1089E000C2F2000132462B46FFF7CEFF04B070BD45
:1089F00070B584B00E4615460093089C01949DF80E
:108A00002430029340F6D831C2F2000132462B46A0
:108A1000FFF7BAFF04B070BD00B583B04FF000039C
:108A200000934FF00100019040F6E830C2F20000E0
:108A300041F288314FF0FF0248F62503C0F60203E9
:108A4000FFF7D6FF40F6D834C2F20004FFF7CEFCA1
:108A50002046FFF7BFFEFFF7ABF9F7E740F690239C
:108A6000C2F2000318681A689042FBD1704700BF39
:108A700010B540F69023C2F200031A6802F1010219
:108A80001A60FFF79DFC044640F6D830C2F20000A1
:108A9000FFF734FE204310F0FF0F06D040F67C2095
:108AA000C2F200000068FFF7B5F910BD08B54DF23D
:108AB0008860C0F603004FF0060148F6E962C0F690
:108AC0000202FFF7FFFA40F61873C2F200031860C3
:108AD00008BD00BF38B504460D4640F60C43C2F24F
:108AE0000003586AA0420AD040F60C41C2F20001CD
:108AF0004C620A681AB115B14948FCF7F5FF40F617
:108B00000C43C2F20003186F84420AD040F60C41B5
:108B1000C2F200010C67CA6C1AB115B14148FCF7EA
:108B2000E3FF40F60C43C2F20003D3F8BC008442DA
:108B30000CD040F60C41C2F20001C1F8BC40D1F8A3
:108B400098201AB115B13848FCF7CEFF40F60C4317
:108B5000C2F20003D3F8080184420CD040F60C4165
:108B6000C2F20001C1F80841D1F8E4201AB115B1F0
:108B70002E48FCF7B9FF40F60C43C2F20003D3F8CD
:108B8000540184420CD040F60C41C2F20001C1F8FD
:108B90005441D1F830211AB115B12548FCF7A4FF92
:108BA00040F60C43C2F20003D3F8A00184420CD07B
:108BB00040F60C41C2F20001C1F8A041D1F87C217D
:108BC0001AB115B11B48FCF78FFF40F60C43C2F2F7
:108BD0000003D3F8EC0184420CD040F60C41C2F201
:108BE0000001C1F8EC41D1F8C8211AB115B1124801
:108BF000FCF77AFF40F60C43C2F20003D3F83802C8
:108C0000A0420CD040F60C41C2F20001C1F838423B
:108C1000D1F814221AB115B10848FCF765FF38BD28
:108C20001C0C0020680C0020B40C0020000D00205B
:108C30004C0D0020980D0020E40D0020300E002087
:108C40002DE9F04707460D4691460898DDF8288043
:108C50000C683E68D8F800108A19944202D80219AC
:108C6000964203D304192C60BDE8F087341B061B21
:108C7000B14234BF8A46B246099931B1D9F80000F1
:108C800008181919524611F087FAD8F80030CAEBC3
:108C90000302C8F800203E6806EB0A013960D9F8E3
:108CA000000000EB0A03C9F800302E68A4195444F0
:108CB0002C60BDE8F08700BF70B584B09CF81960E7
:108CC000157A947B4FF007038CF810304FF00502B3
:108CD0008CF8112006F00F0260F3C7128CF81220F6
:108CE0004FF0000065F301008CF813004FF0000214
:108CF00061F30A02ACF814208CF81640DCF80C1072
:108D00000093DCF804300193CDF808C001F10400B1
:108D10000CF108020CF11003FFF792FF04B070BDD4
:108D20002DE9F04F8FB00746059114464FF0000330
:108D30000793136012896068131A8B4238BF05933A
:108D40000599002900F0AA8040F61C75C2F20005C2
:108D50002D6815B34FEAC5054FF000024FF0FF0133
:108D6000134640F62470C2F20000A5F10806C6F3CF
:108D7000C00E1658F6798E4240F0958096E016584F
:108D8000F6798E421CBF0133314602F10802865843
:108D9000F6798E4240F09F80A0E04FF0000303EB95
:108DA00043024FEAC20000F1100008904FF48071B6
:108DB000ADF824104FF00402ADF826208DF82830CD
:108DC0000DF129004FF000014FF0070211F008FAF1
:108DD00004F1040B04944FF010030093019705A8CD
:108DE00002905846214607AA08ABFFF729FF0599CC
:108DF000002951D04FF001028DF821200DF13200F1
:108E00004FF000014FF0060211F0EAF940F61C7332
:108E1000C2F20003186800283ED04FF0FF014FF067
:108E2000000440F62479C2F200094DF2E058C0F681
:108E3000030840F61C7AC2F2000A59F83450ED7962
:108E40008D4223D08DF820404FEA05160DF1220007
:108E500008EB06014FF0080211F09EF906F1080137
:108E60000DF12A0041444FF0080211F095F94FF03E
:108E700018020092019705AB02935846049907AA7D
:108E800008ABFFF7DDFE059830B1294604F1010477
:108E9000DAF80020A242D0D8079801E04FF0FF3066
:108EA0000FB0BDE8F08F03F10103314602F1080273
:108EB000AA423FF474AFBEF1000F3FF460AF165802
:108EC000F6798E421CBF0133314602F10802AA42F4
:108ED0007FF455AF63E703F10103314602F1080265
:108EE000AA427FF44CAF5AE72DE9F0414FF0010060
:108EF000FCF7A4FC4DF26060C0F60300FCF722FB17
:108F000040F65073C2F200034FF001021A7040F6AF
:108F1000D460C2F20000016841B940F6D464C2F2E4
:108F20000004FEF745FF2568002DFAD040F62177B2
:108F3000C2F2000740F65074C2F2000440F66C66BC
:108F4000C2F2000640F64475C2F2000540F6D06851
:108F5000C2F200083B783BB14FF000023A704FF08C
:108F600002002070FCF764FC317859B14FF0000327
:108F70003370227862F07F0020704FF001000146CC
:108F8000FFF7A8FD297851B14FF000002870237831
:108F900003F07F0222704FF00101FFF79BFD98F86C
:108FA000000010B9FEF704FFD4E740F65071C2F29A
:108FB00000014FF002030B704FF00000FCF73EFC85
:108FC000BDE8F08108B540F6D463C2F20003186032
:108FD00040F61870C2F200000068FEF71BFF08BDE3
:108FE00070B505460E4640F67473C2F20003186869
:108FF000032801D9F7F722FC40F67472C2F200028E
:10900000116840F6B064C2F2000444F8316004EB29
:10901000C104656001F10101116070BD70B50546C4
:109020000C461646032801D9F7F708FC40F62473CE
:10903000C2F2000353F8350008B1F7F7FFFB40F622
:109040002471C2F2000141F8354001EBC5056E60A4
:1090500040F61C73C2F200031A6802F101021A60A2
:10906000206930B1FCF76EFA04F10404206900288D
:10907000F8D170BD08B540F60C43C2F20003196880
:1090800081425AD040F60C42C2F20002D36C8342B5
:1090900034D040F60C41C2F20001D1F8982082424F
:1090A0002FD040F60C43C2F20003D3F8E410814203
:1090B0002AD040F60C42C2F20002D2F8303183428C
:1090C00025D040F60C41C2F20001D1F87C21824249
:1090D00020D040F60C43C2F20003D3F8C8118142FD
:1090E0001BD040F60C42C2F20002D2F81432834286
:1090F00016D0F7F7A3FB4FF0080013E04FF0010084
:1091000010E04FF002000DE04FF003000AE04FF0D6
:10911000040007E04FF0050004E04FF0060001E016
:109120004FF0070040F60C41C2F200014FF04C0234
:1091300002FB001090F8200008BD4FF00000F1E79E
:109140002DE9F04F8FB0089007910A924FF000037D
:1091500009931360546813891B1B8B4238BF079314
:109160000799002900F04A81082C69D840F61C7440
:10917000C2F20004D4F800E040F67475C2F20005B3
:109180002E680EEBCE0707EBC60404F109044FF07E
:10919000000140F62477C2F20007CB598BB1DD689D
:1091A000641903F110051B695BB15E890EB104F10E
:1091B00007049B890BB104F1070455F8043F002B09
:1091C000F3D101F108012029E7D140F6D461C2F2C0
:1091D00000010D682F7E6E7EEB8A03F10103C3F35D
:1091E00047054FF000010C914FF009038DF82C302A
:1091F0004FF002018DF82D10ADF82E408DF830E0C3
:109200004FF001018DF831104FF0000167F3451167
:1092100066F3861161F07F018DF833108DF83450BC
:109220000093019007A8029002F10400114609AAD8
:109230000BABFFF705FD079A002A00F0DD80E0E0A8
:109240004FF009001060DCE05BF83640002C00F0C5
:10925000CE80059D286800284BD07A68B2420CD099
:109260004FF0000310F0010F3ED1DFE007EBC30227
:109270005268B24240F0E38001E04FF0000357F83B
:109280003300D2B290F8048090F805C090F806E060
:10929000C579016819B143F01000C3B201E04FF085
:1092A00000034FF008008DF82C004FF00B018DF8F3
:1092B0002D108DF82E208DF82F808DF830C08DF870
:1092C00031E08DF832508DF833300A990090089AC9
:1092D000019207AB029301F1040009AA0BABFFF75F
:1092E000AFFC079828B987E003F101052B468542BA
:1092F000BCD104F1100523697BB129464FF000026F
:10930000588908B102F101029B890BB102F10102F7
:1093100051F8043F002BF3D101E04FF000025FFA57
:1093200086FCD2B294F804E06079A17923681BB17D
:1093300046F02003DBB201E04FF000038DF82CA0D3
:109340004FF004088DF82D808DF82EC04FF0000CE2
:109350008DF82FC08DF830208DF831E08DF8320077
:109360008DF833108DF834300A99CDF800A0089AA2
:10937000019207A8029001EB080009AA0BABFFF7C6
:109380005FFC0799002937D0A3686BB10A99E2689E
:1093900000920898019007AA029201EB080009AA1E
:1093A000FFF74EFC079B3BB3246904B34FF0010861
:1093B0004FF000092046FFF75DFE8DF8350061890A
:1093C00039B10DF11C0C40462246FFF775FC079998
:1093D00091B1A18939B10DF11C0C48462246FFF725
:1093E0006BFC079840B155F8044F002CE2D106F110
:1093F0000106042E7FF428AF099814E04FF0FF30E7
:1094000011E04FF0000640F6247BC2F2000B40F65C
:109410007474C2F2000405944FF0090A40F6B06774
:10942000C2F2000710E70FB0BDE8F08F03F10103AF
:1094300007EBC3014A68B2427FF456AF1FE705F15C
:10944000010307EBC3014A68B2427FF44DAF16E750
:1094500008B540F65473C2F200031A5C40F60C41A2
:10946000C2F200014FF04C0000FB0210436AD3F13E
:10947000010238BF002242634FF00001C163016462
:10948000416400F11000FCF72FFB08BD2DE9F84FF7
:1094900081468A4640F65473C2F200031A5C40F6D5
:1094A0000C40C2F200004FF04C0404FB020404F133
:1094B00048064FF001084FF0000740F6D86BC2F2A3
:1094C000000B354640463146F7F7BCF930B14FF056
:1094D00002003146F7F7B6F9BDE8F88FBAF1000F90
:1094E00005D148464146FBF759FF032827D0256C94
:1094F00075B15846A168E26BA8470546B0F1FF3F39
:1095000014D06064484659462A46FBF76DFF0EE0CA
:10951000616CA5688D4228BF0D464846E16B2A461E
:10952000FBF762FFE36B5A19E26300E03D46606CB3
:10953000A16888423CBFE7632764451B65643846E1
:109540003146F7F77FF90228BBD0BDE8F88F00BF9E
:10955000F8B505460E46174640F65473C2F20003AE
:109560001A5C40F60C40C2F200004FF04C0404FBC1
:1095700002044FF00000FBF769FEE76326644FF03A
:109580000001616428464FF00101FFF77FFF4FF0B3
:109590000100FBF75BFEF8BDF8B505460F46164621
:1095A00040F65473C2F200031A5C40F60C40C2F25B
:1095B00000004FF04C0404FB0204A168B1420DD23C
:1095C00043F65803C2F200039F4207D344F2580205
:1095D000C2F20002974201D2F7F730F94FF00000D3
:1095E000FBF734FEE7634FF0000020646664284612
:1095F0004FF00101FFF74AFF4FF00100FBF726FE95
:10960000F8BD00BF08B5FBF777FF08BD70B586B0A1
:1096100005460C46164602A8F8F7BCFB01462EB1DB
:1096200002A82A46234600F0A5FD07E04FF00103FB
:10963000009302A82A46234600F04EFE06B070BDF5
:1096400070B58AB00378212B00F0938004D86BB1F9
:10965000012B40F0D88186E0A12B00F0A781C02B20
:1096600000F0B481802B40F0CE8195E0417805294F
:1096700003D0092940F0CA8146E0408840F6507284
:10968000C2F200021378022B02D0032B33D118E070
:1096900000F1FF318AB27E2A30D8C0B240F664733E
:1096A000C2F2000318704FF00201FCF731F840F6E7
:1096B0005070C2F200004FF0030101704FF0010042
:1096C000C3E170B940F66472C2F20002107040F655
:1096D0005070C2F200004FF0020303704FF001001F
:1096E000B3E17F280DD840F66471C2F20001087022
:1096F0004FF00100A9E14FF00200A6E14FF0020097
:10970000A3E14FF00200A0E1827840F65073C2F26C
:1097100000031978022923D972B940F65073C2F2B6
:1097200000034FF0030119704FF001000146FFF7ED
:10973000D1F94FF0010088E1012A18BF022040F062
:10974000848140F65070C2F200004FF004020270B3
:109750004FF000000146FFF7BDF94FF0010074E142
:109760004FF0020071E140780B280CBF012002206D
:109770006BE18388032B00F24C8140F62474C2F223
:10978000000404EBC3035B68002B00F0458198479D
:10979000002808BF022058E142781AB1062A40F09A
:1097A0003E8121E0C18802291BD14FF00000ADF8B5
:1097B000040040F6D462C2F2000212680346517EF1
:1097C00061F30003ADF80430127E62F341030AA98D
:1097D00021F8243D4FF00202FFF7DEFE4FF00300B8
:1097E00033E14FF0020030E18278C1888CB2C37857
:1097F000022B2ED0032B3DD0012B40F0D48040F61D
:109800007065C2F2000528464DF27461C0F603018E
:109810004FF0120210F0C0FC40F6D460C2F200001B
:1098200001688A892A81CB896B81088AA8818A7C10
:109830002A71CB7C6B71097DA9714FF0000029461C
:10984000122C34BF22461222FFF7A6FE4FF003006F
:10985000FBE040F66872C2F2000211814FF0000096
:10986000506049F24111C0F60201FFF771FE4FF05E
:109870000300EAE0D2B940F67064C2F2000404F1D9
:1098800002004DF27061C0F603014FF0020210F0C9
:1098900083FC4FF0040222704FF0030565704FF017
:1098A00000002146FFF778FE2846CEE0012A06D1C7
:1098B00040F6D463C2F20003196809682FE0022A57
:1098C00006D140F6D462C2F200021068416826E078
:1098D000032A06D140F6D463C2F2000319688968EE
:1098E0001DE002F00F0022F00F03102B08D15A4B9D
:1098F000196888420EDA594A52F8300001680EE0C1
:10990000202B07D1032805D8554951F8300008B15C
:10991000016804E0EE2A04D04FF0020095E009B996
:109920003EE05049B1F1FF3F40F0888001A84FF080
:1099300020014FF00102FFF769FE0AAD2A184FF02F
:10994000000002F8240C01A978E000F10206428030
:1099500003F10102134611F8015F5DB100F104004B
:10996000758002F1010311F8012F002A6FD101E087
:109970004FF0000340F67061C2F200014FF00305A2
:109980004D7003F101034FEA4303DAB20A704FF05E
:109990000000A24228BF2246FFF7FEFD284654E001
:1099A0004FF0020051E04FF002004EE08388032B9D
:1099B00038D840F62474C2F2000404EBC3035B6899
:1099C0009BB39847002808BF02203EE04378212B34
:1099D0002ED1C18840F66873C2F2000319814FF09E
:1099E00000025A608088042825D1104648F621518B
:1099F000C0F6020140F66872C2F20002FFF7A8FD4D
:109A00004FF0030021E04FF002001EE04FF0020093
:109A10001BE04FF0020018E04FF0020015E04FF09D
:109A2000020012E04FF002000FE04FF002000CE0E5
:109A30004FF0020009E04FF0020006E00A78002A29
:109A400096D009484FF000037FE70AB070BD1E2B87
:109A50007FF47BAF8EE700BF740F0020B00E0020B4
:109A6000240F00208CD60308700E002010B5044689
:109A7000436993B14FF00000606140F65071C2F24B
:109A800000010A78032A08D140F66473C2F2000389
:109A900018784FF00301FBF73BFE206958B34FF0F5
:109AA00000002061E06040F62071C2F20001087001
:109AB00040F64871C2F200014FF00802FFF7A2FD24
:109AC000082853D140F64872C2F20002137813F00E
:109AD000800F06D140F64870C2F20000C18800290C
:109AE00044D140F64870C2F200004FF000010A462F
:109AF000FFF7A6FD2DE0E168002937D04FF0000008
:109B0000E06040F62072C2F20002137840F6706105
:109B1000C2F20001C3F14002FFF774FD034628B30F
:109B200040F62070C2F2000001785A18D2B20270DA
:109B300040F64873C2F20003D888904216D140F62E
:109B40004870C2F2000040F67061C2F20001FFF7F7
:109B500077FD012804D0022808D1FBF72FFC10BDA7
:109B60004FF0000001460246FFF716FD10BD00BF92
:109B700008B540F67873C2F200031B693BB14FF0A1
:109B8000000140F67872C2F200025269984740F62E
:109B90007870C2F200004FF00001017041608160F6
:109BA000C1600161416108BD40F67870C2F20000F9
:109BB00081614DF2E061C0F603018A5C42778377F0
:109BC000037F6FF3070303774FF000014162704793
:109BD00030B583B040F67874C2F200042070089D5E
:109BE0006560099DA5600A9DE5600B9D25610C9D42
:109BF00065619DF8184000949DF81C400194FFF7A2
:109C0000D3FF03B030BD00BF40F67873C2F200034B
:109C10005B6AB3F1FF3F09D140F67871C2F20001EF
:109C20004FF000034B624FF0010070473F2B0BD801
:109C300040F67872C2F20002106AC15403F10103C7
:109C400053624FF0010070474FF00000704700BFB3
:109C5000704700BF70B540F67874C2F2000404F19A
:109C600018004DF29861C0F603014FF0070210F0A2
:109C700093FA4FF000004DF24471C0F60301FFF774
:109C8000AFF949F6C966C0F602064FF000004DF282
:109C9000E461C0F603013246FFF7C0F94DF24C759E
:109CA000C0F603054FF0010029463246FFF7B6F92A
:109CB0002869FFF7DFF984F8280040F6A470C2F2A3
:109CC00000004FF0070149F6D942C0F602024FF0FA
:109CD0000003FBF7E9FE70BD38B541F25803C2F24C
:109CE00000034FF001021A7040F67874C2F20004CB
:109CF00094F828004FF000010A46FFF74DFC606819
:109D000068B140F67874C2F200044FF0FF35656226
:109D10006368207861699847616A0029F7D040F646
:109D20007870C2F200004FF000024262836833B1E3
:109D300040F67871C2F2000108784969984738BD49
:109D40002DE9F04F83B0804643680BB9806828B195
:109D50004FF00001C8F80810FFF7BEFFD8F80C203C
:109D6000002A45D04FF00003C8F80C30D8F80000A6
:109D700041F21801C2F200014FF04002FFF742FC2D
:109D8000814640F67870C2F20000C16800292FD0E9
:109D9000B9F1000F2CD040F67874C2F2000441F201
:109DA0001806C2F200064FF0000509F1FF3B0BF068
:109DB000010B2078715D2A466369E768B84705F1B1
:109DC000010AD14570D113E0207816F80A102A460E
:109DD0006369E768B8470AF1010A207816F80A10A3
:109DE0002A466369E768B8470AF1010AD145EBD111
:109DF000D8F81420002A54D04FF0000441F2580340
:109E0000C2F200031C70C8F8144040F6F470C2F2AD
:109E10000000FEF733FD40F67870C2F200004462A5
:109E20004168002936D040F67875C2F2000540F648
:109E3000B474C2F200042C622C46656A6268207811
:109E400061699047636A9D42F7D11DB3D8F800005D
:109E500040F6B471C2F200012A46FFF79DFB4FF0B5
:109E600000000090019040F6F470C2F200004FF044
:109E70004B014FF0FF0249F6D943C0F60203FEF74B
:109E8000B7FD0EE040F67872C2F200021078516918
:109E9000984706E040F67871C2F200018B68002B0B
:109EA000F0D103B0BDE8F08FBBF1000F8CD020786B
:109EB00016F80A102A466369E768B8470AF1010AEA
:109EC000D14581D194E700BF10B544780378212BA8
:109ED00002D0A12B1BD10EE0202C04D0222C14BFC9
:109EE0000020012010BD072A14D10D4810F054F9AC
:109EF0004FF0010010BD212C0FD14FF00000084998
:109F00004FF00702FFF748FB4FF0030010BD4FF082
:109F1000000010BD4FF0020010BD4FF0000010BD5A
:109F2000900F002008B541F25803C2F200031878E0
:109F300070B940F67871C2F200014A6A72B940F60F
:109F40007873C2F2000393F82800FFF781FA08BD86
:109F500040F6A470C2F20000FBF7C6FD08BD00BFCA
:109F60004DF2B060C0F60300704700BF70B40378D4
:109F700001298CBF4478002402298CBF85780025F4
:109F8000DCF8000048B34FEA93064DF67800C0F6BF
:109F90000300365C16704FEA031343EA141303F010
:109FA0003F031B5C5370012907D94FEA840444EA3C
:109FB000951303F03F04205C01E04FF03D009070EA
:109FC000022907D905F03F054DF67803C0F60303D3
:109FD000E95C01E04FF03D01D17070BC704700BFFB
:109FE00082B04FF015010CE00191019B03F1FF32AB
:109FF000019233B100BF019B03F1FF320192002BAC
:10A00000F8D100F1FF30B0F1FF3FEDD102B0704761
:10A0100070B4C4B24FEA10204DF60C16C0F6030619
:10A020004DF27875C0F6030511F8013B1AB94BB92A
:10A0300044EA00200BE06340F45C4440E85C013AF1
:10A04000F2D1F5E76340F45C4440E85CECE770BCB7
:10A05000704700BF10B444F6FB43C0F2861311F8FA
:10A06000014B02B9ACB380EA04404FEA400010F063
:10A07000807F18BF58404FEA400010F0807F18BF23
:10A0800058404FEA400010F0807F18BF58404FEA18
:10A09000400010F0807F18BF58404FEA400010F099
:10A0A000807F18BF58404FEA400010F0807F18BFF3
:10A0B00058404FEA400010F0807F18BF58404FEAE8
:10A0C000400010F0807F18BF5840002AC7D0013AE6
:10A0D000C5D120F07F4010BC704700BF82B0019016
:10A0E0009DF806304FF0000063F307009DF805204F
:10A0F00062F30F209DF8042062F317409DF80720BB
:10A1000012F0800F14BF63F07F0103F07F0161F351
:10A1100007004FEA4201CAB262F31F6013F0800FDA
:10A1200018BF42F0010262F31F6002B0704700BF27
:10A1300084B0C0F307438DF80C30C0F307228DF8CC
:10A140000D20C3B24FEA10604FEA500210F0010F29
:10A1500014BF63F07F0103F07F018DF80E1013F040
:10A16000800F18BF62F07F028DF80F20039804B0B3
:10A17000704700BF2DE9F04F83B005460F461446E7
:10A180001E46019201F1FF3313F1050F44D8032E4F
:10A1900043D9A6F10400C0F380080DF1040C284651
:10A1A000FFF7E4FE05F10305A7F1030104F1040440
:10A1B000A6F10406A7F1040717F1050F67D92CE0F3
:10A1C0000DF1040C284639462246FFF7CFFE05F173
:10A1D000030B5D46A7F1030104F1040A5446A6F1FE
:10A1E00004094E46A7F1040717F1050F15D80F46CD
:10A1F0000DF1040C58465246FFF7B8FE0BF103056B
:10A20000A7F103010AF10404A9F10406A7F1040867
:10A2100018F1050F59D900E0FFE799B396B30DF196
:10A22000040C28466A46FFF7A1FE022E11D0032E29
:10A2300002D0012E26D11AE0019929B19DF8002003
:10A2400022704FF0010301E04FF0000304F101041C
:10A2500001E04FF00003019830B102A9CA1812F8CA
:10A26000080C207003F1010304F1010401E04FF038
:10A270000003019921B102AAD31813F8080C207029
:10A2800004F101040199601A03B0BDE8F08F0F4694
:10A29000032EC2D9B8F1000F92D00DF1040C28465C
:10A2A0002246FFF763FE05F10305A7F1030104F160
:10A2B0000404A6F10406A7F1040717F1050FACD8B2
:10A2C0000F46032E3FF67CAFA7E7A7F10307032E47
:10A2D0003FF676AFA1E700BFF0B49DF81040ECB1B7
:10A2E0004FEA41079F421CD2DD1B1DD056194FF08B
:10A2F00030046FEA0203F31803F0010302F8014B84
:10A30000B24240F0928007E0134603F8014B5470CC
:10A3100003F10102B242F7D13B4607E04FF00005DE
:10A3200004E04FF0000501E04FF0000500293CD0AB
:10A3300003F1FF34002B3AD000F101034118284605
:10A34000521B04F1FF3515F0020F10D032E0A4F1DA
:10A35000020603F101031F46012C29D03446B446FE
:10A3600013F8016C4FEA1616092E42D944E01E4636
:10A3700013F8015C4FEA1515092D8CBF37353035C0
:10A38000155414B900F1010012E013F8016C06F045
:10A390000F05092D8CBF373530351618757000F153
:10A3A000020528468B42D2D102E0284600E028462A
:10A3B000F0BC70471E4613F8015C4FEA1515092DD5
:10A3C00094BF303537351554002CDBD013F8016CB1
:10A3D00006F00F05092D94BF303537351618757006
:10A3E00000F102008B42E3D003F10103A4F1020467
:10A3F000BDE706F1300601E006F137065655BCF11F
:10A40000000FBFD013F8016C06F00F06092E94BFA1
:10A41000303637361018467005F102008F42C7D02B
:10A4200003F10103A4F10204A1E7002B3FF46CAF98
:10A4300002F8014BB2427FF467AF6DE7DCF81430ED
:10A4400093F8452083F84420DCF8141091F8463046
:10A4500081F84530DCF8141091F8472081F8462047
:10A46000DCF8143083F84700704700BFDCF8143084
:10A4700093F8470093F8462083F84720DCF814103F
:10A4800091F8453081F84630DCF8141091F84420FA
:10A4900081F84520704700BF43F2E012C2F200028B
:10A4A000136840F20001C0F60101C85CC918497880
:10A4B00003F10203136041EA00207047DCF8043026
:10A4C000DCF8082002EBD300CCF8080003F0070109
:10A4D0004FF0010303FA01F2CCF80420704700BFEB
:10A4E0002DE9F04F83B004468A4693461E46CDF8C8
:10A4F00004C04FF00007B846B9463DE02546304657
:10A50000D047034600283DD0B9F1000F0CD12028D8
:10A5100029D0092829D00A2829D00D2829D0022D90
:10A520004FF0010988BF0225A3F13002D1B20929F9
:10A5300010D9A3F14100C1B2052903D8A3F1370313
:10A54000D9B207E0A3F16102D0B205281AD8A3F16D
:10A550005703D9B24FEA0717FCB241EA040708F1E2
:10A5600001082C4606E02C4604E02C4602E02C466E
:10A5700000E02C463046D847FF2CBFD004F1FF3511
:10A58000002CBCD1DDF804C03846FFF757FF019B13
:10A590005A69D8F1010838BF4FF0000882F850809E
:10A5A00003B0BDE8F08F00BF43F2D803C2F200034E
:10A5B0001B684B634BB19A68824209D0DB684B63DE
:10A5C0001BB19A688242F9D102E04FF01E00704739
:10A5D0004FF00000704700BF884204D8884234BF63
:10A5E0000220002070474FF001007047D0F804317E
:10A5F000D0F80021934214BFC05C0020704700BF18
:10A60000D0F80431FF2B14BF01330023C0F804310C
:10A61000704700BF10B4DCF81420D16C0B46044620
:10A6200058B14FEA016343EA116301F47F4043EA02
:10A63000002301F47F0143EA1123DCF8040030B168
:10A6400099B24FEA134060F30F0361F31F435CB903
:10A650004FEA036141EA136103F47F4041EA0021BC
:10A6600003F47F0341EA1323D36410BC704700BF97
:10A67000DCF80030FA2B05D841F25C02C2F200028D
:10A68000D05C70474FF00000704700BFDCF800302E
:10A6900003F10103CCF80030DCF8140090F85120ED
:10A6A00002F1010280F85120704700BF70B40446E7
:10A6B0000846A1B199188C4211D22518AA420ED28F
:10A6C00094423ABFC4EB0206F6B20026A94205D274
:10A6D0000019821AD31AF118C8B200E0304670BCD3
:10A6E000704700BFF0B583B043F2B003C2F200037D
:10A6F0004FF00C021A7043F29800C2F20000046896
:10A700003CB3154643F2B007C2F200074FF0000613
:10A7100021680B6873B10DF107000DF10601984730
:10A720009DF807009DF8061032463B78FFF7BEFF04
:10A730004519EDB26468002CEAD143F2B002C2F2CE
:10A7400000021078A84204D243F2B001C2F2000124
:10A750000D7043F2B003C2F200034FF00A025A70C8
:10A7600043F2C804C2F2000424683CB3154643F225
:10A77000B007C2F200074FF000062068036873B10B
:10A780000DF107000DF1060198479DF807009DF8AF
:10A79000061032467B78FFF789FF4519EDB26468F1
:10A7A000002CEAD143F2B001C2F200014A78AA4279
:10A7B00004D243F2B000C2F20000457043F2B0038D
:10A7C000C2F200034FF00201997043F2A804C2F2F2
:10A7D000000424683CB30D4643F2B007C2F2000700
:10A7E0004FF000062268136873B10DF107000DF1F8
:10A7F000060198479DF807009DF806103246BB7881
:10A80000FFF754FF4519EDB26468002CEAD143F21A
:10A81000B000C2F200008178A94204D243F2B00233
:10A82000C2F20002957043F2B003C2F200034FF08F
:10A830000100D87043F2F414C2F2000424683CB35F
:10A84000054643F2B007C2F200074FF00006216848
:10A850000A6872B10DF107000DF1060190479DF8ED
:10A8600007009DF806103246FB78FFF71FFF4519D9
:10A87000EDB26468002CEAD143F2B003C2F20003E7
:10A88000D878A84204D243F2B001C2F20001CD70E0
:10A8900003B0F0BD43F2DC13C2F20003196840F2CA
:10A8A0000000C0F60200401A704700BF034610B116
:10A8B00082688A4218D043F2AC03C2F200031868DF
:10A8C00060B182688A4203D10BE083688B420AD070
:10A8D00040680028F9D14FF0000305E04FF0000375
:10A8E00002E0034600E003461846704710B540F208
:10A8F000A064C1F200044FF4117303FB0044D4F8C8
:10A900000811B1F1FF3F03D0D4F8042191420DD1D9
:10A9100023689A6A4FF0FF019047002834D0D4F89A
:10A92000080100F10100C4F8080110BD91422BD8C4
:10A930006318197943F2B502C2F2000213787BB9A9
:10A94000FD290FD923689A6A4FF0FE019047D8B1CC
:10A9500043F2B500C2F200004FF00101017010BDDA
:10A960006FEA01012268936AC9B2984760B1D4F8CE
:10A97000080100F10100C4F8080143F2B501C2F278
:10A9800000014FF000020A7010BD00BF70B506460E
:10A9900040F2A065C1F200054FF4117404FB00F40D
:10A9A0002B194FF00101C3F80C112A5993699847EC
:10A9B0002859016A3046884770BD00BF38B540F25B
:10A9C000A061C1F200014FF4117202FB00F28C1879
:10A9D000D4F80831D4F80451AB420DD08958E318AB
:10A9E0008A6A1979904738B1D4F80801FF2814BF52
:10A9F00001300020C4F8080138BD00BF38B540F26E
:10AA0000A064C1F200044FF4117202FB00F2A3181B
:10AA1000D3F80451D3F808118D4206D14FF000014C
:10AA2000C3F80C11A2589369984738BD10B440F28E
:10AA3000A063C1F200034FF4117202FB003000F575
:10AA40008870D0F80031FF2B14BF5A1C0022D0F8B8
:10AA50000441A2421CBFC154C0F8002110BC704781
:10AA6000F8B543F2DC14C2F2000424688568C768B4
:10AA7000466807FB05604518611911D2CE180B48CE
:10AA8000864210D8012B04D1635D13704FF0000093
:10AA9000F8BD10461A460FF07FFB4FF00000F8BDDE
:10AAA0004FF01F00F8BD4FF01F00F8BD0100020875
:10AAB00010B543F29C03C2F200031A8840F2A06072
:10AAC000C1F200004FF4117404FB0204F5F70CFF0F
:10AAD0004FF0FF31C4F810124FF00003C4F81832E1
:10AAE00004F58874F5F70AFF10BD00BFF8B50646F7
:10AAF0004FF00203037044F20000C0F60000C28B66
:10AB00004FF6FF718A4221D03F4C404BA34222D2E4
:10AB100003F110033E4DEF1A4FEA17124FF6FF757F
:10AB200002F1010002F001071C46D98BA9424FD166
:10AB300015E01C46D98BA94211D002F1010203F1A4
:10AB400010031C46D98BA94257D108E044F20004F7
:10AB5000C0F6000403E044F20004C0F600044FF61F
:10AB6000FF7021464FF00D02FFF752FA4FF6FF73C8
:10AB7000984208BF0020E28982421BD0A4F1100550
:10AB800044F20000C0F6000085421AD34FF6FF7071
:10AB900029464FF00D02FFF73BFA4FF6FF7188424E
:10ABA00008BF002034F8024C84420AD12C464FF0F2
:10ABB000010201E04FF00002607BFF2806D13270F5
:10ABC00004E04FF0020333704FF000042046F8BD5C
:10ABD0004FF0000202F1010203F110038242BED0E5
:10ABE000002FA6D01C46D98BA942B8D002F1010291
:10ABF00003F1100382429CD1B1E702F1010203F19B
:10AC00001003824295D1AAE70080000800400008A6
:10AC10000F80000870B5C0B005460E4620F0FF0456
:10AC2000684621464FF04002F8F782FB00AB53FA2A
:10AC300085F031464FF010020FF0AEFA684621461B
:10AC40004FF48072F8F7C8FC40B070BD38B50546C7
:10AC500040F2A064C1F200044FF4117303FB0044FE
:10AC6000D4F81C02FDF718FB43F29C00C2F200006E
:10AC70000188A94206D143F29C03C2F200034FF6B9
:10AC8000FF721A804FF00000C4F81C0238BD00BFEC
:10AC900010B54FF00000FAF77FFF43F29803C2F2BD
:10ACA00000031C6834B12068016901B188476468F9
:10ACB000002CF8D110BD00BF10B50446072827D8D6
:10ACC000032894BF4FF4FA73322303FB01F140F2DF
:10ACD000A063C1F2000303EBC000C0F8141969B10E
:10ACE000FDF7BCFE002808BF012040F2A063C1F2BE
:10ACF000000303EBC404C4F8100910BD40F2A061C6
:10AD0000C1F2000101EBC4044FF00002C4F81029A5
:10AD100010BD00BF38B50446072851D840F2A063E3
:10AD2000C1F2000303EBC000D0F8145935B340F270
:10AD3000A061C1F2000101EBC402D2F81039EBB1FD
:10AD4000FDF78CFE002808BF012040F2A061C1F28F
:10AD5000000101EBC402D2F81039C01A85420CD2AE
:10AD600040F2A065C1F2000505EBC4014FF00005FB
:10AD7000C1F81459C1F8105900E02D1A05F1040565
:10AD80004CF6CD42CCF6CC42A2FB05234FEA930011
:10AD9000032C0AD800F1630348F21F51C5F2EB11EE
:10ADA000A1FB03324FEA521038BD00F109014CF605
:10ADB000CD42CCF6CC42A2FB01304FEAD00038BDE8
:10ADC0004FF0000038BD00BF70B506466446DCF8A1
:10ADD00014305D6AFDF742FE6169CA6A0AB9C86249
:10ADE00008E0801A05EB850506FB05F6B04224BF96
:10ADF0000020C8626369D96AD1F1010038BF002020
:10AE000070BD00BF10B540F2A063C1F200034FF463
:10AE1000117404FB003303F58873D3F80841002C48
:10AE20005FD15AB14FF0FF31C3F8001143F25C0318
:10AE3000C2F200034FF00000187010BDD3F80021DB
:10AE4000B2F1FF3F06D1FF294BD14FF00002C3F80A
:10AE5000002110BDFF291ED143F25C01C2F20001A6
:10AE60004FF000040C70012A10D94FF00102C3F812
:10AE7000082140F2A063C1F200034FF4117101FBFD
:10AE80000030D0F81C02FCF7C5FF10BD4FF00000E9
:10AE9000C3F8000110BDFE2907D143F25C03C2F2E2
:10AEA00000034FF00101197010BD43F25C00C2F2C3
:10AEB0000000007848B16FEA0101C9B243F25C00BA
:10AEC000C2F200004FF000040470FF2A05D8995424
:10AED00002F10102C3F8002110BD4FF0FF32C3F8A8
:10AEE000002110BD08B540F2A063C1F200034FF489
:10AEF000117202FB0030D0F80811D0F8043100F1D3
:10AF0000040099420AD94FF00002C0F8002143F230
:10AF1000F810C2F200004068FCF77CFF08BD00BFDB
:10AF2000F8B5654643F2DC03C2F200031A7802F07A
:10AF30000804E7B227B1DCF8146096F8516007E026
:10AF400012F0110F06BFDCF8147097F8526000265B
:10AF500001EB800411F8203003F0070302F0200217
:10AF6000D7B23FB111F8202002F00807FAB20AB1B7
:10AF70004FEA430311F820704FEA9712012A08D0D4
:10AF8000022A10D111F82000C0F3011101FB06675D
:10AF90000BE06F6997F8517011F82020C2F301108F
:10AFA00000FB077701E04FF00007042B50D8DFE8E3
:10AFB00013F0C60140003B002200050043F2E011FF
:10AFC000C2F200010B6840F20007C0F60107FA1850
:10AFD00092F802E0D0784FEA006040EA0E405278E2
:10AFE00040EA0220FF5C03F104030B603843FFF7E3
:10AFF0009FF868602CE043F2E012C2F2000213688E
:10B0000040F20000C0F60100C11891F801C0C05C18
:10B010004FEA004040EA0C208978084303F103031B
:10B0200013603F186F6013E0FFF736FAC2196A60C9
:10B030000EE043F2E013C2F20003186840F2000190
:10B04000C0F601010A5CBF186F6000F101001860D2
:10B05000637803F0070343F2DC00C2F200000178DA
:10B0600001F02002D7B237B1607800F00801CAB20F
:10B070000AB14FEA430367784FEA9710012807D0D7
:10B0800002280ED16178C1F3011202FB06670AE0C3
:10B090006F6997F851006178C1F3011202FB000754
:10B0A00001E04FF00007042B50D8DFE813F048010F
:10B0B00040003B002200050043F2E011C2F2000113
:10B0C0000B6840F20007C0F60107FA1892F802E098
:10B0D000D0784FEA006040EA0E40527840EA022001
:10B0E000FF5C03F104030B603843FFF721F8A8600D
:10B0F0002CE043F2E012C2F20002136840F20000BA
:10B10000C0F60100C11891F801C0C05C4FEA0040D0
:10B1100040EA0C208978084303F1030313603F18C9
:10B12000AF6013E0FFF7B8F9C219AA600EE043F26E
:10B13000E013C2F20003186840F20001C0F60101FA
:10B140000A5CBF18AF6000F101001860A37803F03B
:10B15000070343F2DC00C2F20000017801F0200294
:10B16000D7B237B1A07800F00801CAB20AB14FEAED
:10B170004303A7784FEA9710012807D002280ED181
:10B18000A178C1F3011202FB06670AE06F6997F824
:10B190005100A178C1F3011202FB000701E04FF05A
:10B1A0000007042B50D8DFE813F0CA0040003B0032
:10B1B0002200050043F2E011C2F200010B6840F2E8
:10B1C0000007C0F60107FA1892F802E0D0784FEABB
:10B1D000006040EA0E40527840EA0220FA5C03F137
:10B1E00004030B601043FEF7A3FFE8602CE043F27A
:10B1F000E012C2F20002136840F20000C0F6010043
:10B20000C11891F801C0C05C4FEA004040EA0C2030
:10B210008978084303F1030313603F18EF6013E0DC
:10B22000FFF73AF9C219EA600EE043F2E013C2F206
:10B230000003186840F20001C0F601010A5CBF1863
:10B24000EF6000F101001860E37803F0070343F2B8
:10B25000DC00C2F20000017801F02002D0B230B16F
:10B26000E17801F00802D0B208B14FEA4303E17877
:10B270004FEA9112012A02D0022A0FD108E06E692A
:10B2800096F85100E278C2F3011101FB000607E0D5
:10B29000E078C0F3011101FB066601E04FF0000603
:10B2A000042B4CD8DFE803F04B031318300043F2B3
:10B2B000E013C2F20003186840F20001C0F6010179
:10B2C0000A5CB6182E6100F101001860F8BDFFF7A6
:10B2D000E3F882192A61F8BD43F2E012C2F20002DB
:10B2E000136840F20000C0F60100C1184C78C05C41
:10B2F0004FEA004040EA04208978084303F1030341
:10B30000136036182E61F8BD43F2E011C2F200015D
:10B310000B6840F20004C0F60104E2189678D07879
:10B320004FEA006040EA0640527840EA0220E25CC0
:10B3300003F104030B601043FEF7FAFE2861F8BD29
:10B3400010B58AB0044601A8F6F788FD039B237068
:10B35000029860700199A170079A1AB102F1FF304A
:10B36000C3B201E04FF00603E3704FF0010101FAB0
:10B3700003F222710AB010BD70B582B00546124CBE
:10B3800004EB80066846FFF7DBFF9DF8002014F809
:10B3900025309A4212D19DF80100717888420DD172
:10B3A000B2789DF804301A4208D0F078D0F101004C
:10B3B00038BF00204FF00101F17002E04FF00000B3
:10B3C000F07002B070BD00BFF00F001008B5032888
:10B3D0001ED8DFE800F0020910174EF2C820C0F6B0
:10B3E000030010F0C9FC08BD4EF2CC20C0F60300EB
:10B3F00010F0C2FC08BD4EF2E020C0F6030010F0D1
:10B40000BBFC08BD4EF2F820C0F6030010F0B4FCFF
:10B4100008BD00BF2DE9F8430546884616461F467D
:10B4200043F29C03C2F20003B3F8009043F254507D
:10B43000C2F20000016843F29402C2F200021368F3
:10B44000994201D0FFF734FB072D6ED81F2E6CD820
:10B4500040F2A064C1F200044FF4117000FB0944F3
:10B4600043F2F810C2F200004FF00001FCF722FA9C
:10B47000217965F34711072D14BF00250125AA196D
:10B4800062F304012171CBB22DB184F805804344ED
:10B490004FF0020001E04FF0010006F1FF3E5FFABD
:10B4A0008EFE46B302463F1A0EF0010C3D5C04F1DD
:10B4B000040635545B1902F101020EF1FF31C9B2E5
:10B4C000FF2934D114E0BD5C04F10406B5545B19C6
:10B4D00002F1010201F1FF3101F0FF01BD5CB55441
:10B4E0005B1902F1010201F1FF31C9B2FF29EAD172
:10B4F00000F1010070442218137100F10100C4F83A
:10B5000004014FF0FF33C4F8083121680B6A43F29D
:10B510009C00C2F2000000789847FCF749FC43F217
:10B52000F810C2F20000FCF7D3FABDE8F8834FFA36
:10B530008CF5002DC7D0BD5C04F10406B5545B1931
:10B5400002F1010201F1FF31C9B2FF29BBD1CFE7FE
:10B5500000B583B04FF0040241F25A03C2F2000377
:10B560001A704FF001008DF8040043F2CC01C2F2D2
:10B5700000010B88ADF805304FF007004FF0410196
:10B580000DEB0203FFF746FF03B000BD08B541F223
:10B590005A03C2F20003197889B198B1042814D073
:10B5A000042904D1FFF7D4FF4FF0010008BD41F298
:10B5B0005A02C2F2000210704FF0000008BD4FF0B6
:10B5C000000008BD4FF0000008BD4FF0000008BDAE
:10B5D00010B586B00DF10700FFF788FA044618B1E0
:10B5E0009DF8073023B90FE044F20004C0F60004D0
:10B5F000E2894FF6FF7082422BD048F20001C0F67C
:10B6000000018C4209D32AE0304821464FF00D0258
:10B610000EF06CF9002848D0EAE74FF6FF7248F2C6
:10B620000000C0F600006FEA0403C118C1F3001166
:10B6300004F11004E389934239D10AE004F11003C4
:10B640001C46D989914204D003F11004E389934246
:10B6500039D148F20002C0F60002944207D344F206
:10B660000004C0F6000420462146F7F749FF02A86F
:10B6700016494FF00D020EF08FFD4FF0FF008DF8D0
:10B6800015004FF6FF7002A94FF00D02FEF7C0FC47
:10B690004FF6FF71884212BFADF816000021ADF8D9
:10B6A0001610204602A9FFF7B5FA06B010BD844275
:10B6B000D5D20029C2D004F11004E1899142C8D04A
:10B6C0008442BBD3CBE78442B8D3C8E762100020E2
:10B6D0002DE9F04F85B0884691461D46E2464FF071
:10B6E000000426464FF0020B2DE007462846C047CF
:10B6F000034670B324B9202822D0092802D11FE0C4
:10B70000012C05D12B2B0DD02D2B0DD05C4601E04B
:10B71000022C01D12E2B09D0A3F13002D0B209287E
:10B7200017D805E05C4603E05C4601E04FF00304F7
:10B730000E2E05D804A98A1902F8103C06F101065C
:10B740002846C8473846FF28CFD000F1FF370028E9
:10B75000CCD1012C12D98EB104ACA6194FF0000443
:10B7600006F8104C684621460EF01AF9DAF8141063
:10B77000C864DAF8142082F8504005E0DAF8143092
:10B780004FF0010083F8500005B0BDE8F08F00BF16
:10B7900010B5044643F26800C2F20000FCF798F9C5
:10B7A000F6F732FEFAF79EFA08B1FBF7C1FE204623
:10B7B000FCF7C6FC43F26800C2F200004FF0000143
:10B7C000FCF778F810BD00BF10B586B040F200005D
:10B7D000C0F601003449F7F793FE00284BD1334BF4
:10B7E000334A9A421DD240F20001C0F601010B68B3
:10B7F000B3F1FF3F42D102F104032E4AD01A20F0E8
:10B800000302991812F0040F3FD118468B420CD056
:10B8100003F104021B68B3F1FF3F3ED04FF000007C
:10B8200031E040F20000C0F6010040F20003C0F633
:10B830000203984225D10DF10700FFF757F904469E
:10B84000B0B19DF80710022912D002A821464FF08E
:10B8500010020EF0A1FC9DF815006FF307008DF8A3
:10B860001500204602A9FFF7D5F94FF001000AE0C4
:10B870004FF0010007E04FF0000004E04FF000003F
:10B8800001E04FF0000006B010BD184603F10403BC
:10B890000268B2F1FF3FB8D0C0E702F104031068BC
:10B8A000B0F1FF3FB1D0B9E7FFFF01080000020887
:10B8B00000000108030002082DE9F00703460028F4
:10B8C0004ED040F20022C0F6000292F8469092F864
:10B8D000470043F2B004C2F2000494F8018092F8E9
:10B8E00048C0257843F2CC02C2F200021468177AED
:10B8F000567AD2F804A04FF000021A7083F8019033
:10B900009870DA704FF0FB0018714FF0060983F859
:10B9100005909D7183F807804FF0040883F8088034
:10B9200083F8098083F80AC0DD721A734FEA142580
:10B930005D739C73DF731E745A744FF01D029A740A
:10B940004FF00202DA744FF0FE021A755A754FEA90
:10B950001A229A7583F817A018764FF01F005876B0
:10B9600029B143F2B003C2F200031A680A60BDE8CD
:10B97000F0077047034628B143F2CC02C2F200023E
:10B980001068186043F2CC01C2F20001087A7047D7
:10B9900070B505460E4614464FF000002946FEF7E6
:10B9A00085FF08B1F4F74AFF43F2AC03C2F200038B
:10B9B0001A686260A56026601C6070BD08B539B168
:10B9C00043F29803C2F200031A68426018601EE056
:10B9D00043F29803C2F200031B6883420FD15868F8
:10B9E00043F29801C2F20001086010E042685A6018
:10B9F00041605A688242F9D013461BB907E033B15F
:10BA00004FF000015A688242F0D01346F5E7FEF786
:10BA100069FE08BD08B539B143F2C803C2F200039C
:10BA20001A68426018601EE043F2C803C2F20003C5
:10BA30001B6883420FD1586843F2C801C2F200016B
:10BA4000086010E042685A6041605A688242F9D04A
:10BA500013461BB907E033B14FF000015A68824228
:10BA6000F0D01346F5E7FEF73DFE08BD08B539B145
:10BA700043F2A803C2F200031A68426018601EE095
:10BA800043F2A803C2F200031B6883420FD1586837
:10BA900043F2A801C2F20001086010E042685A6057
:10BAA00041605A688242F9D013461BB907E033B1AE
:10BAB0004FF000015A688242F0D01346F5E7FEF7D6
:10BAC00011FE08BD08B539B143F2F413C2F2000308
:10BAD0001A68426018601EE043F2F413C2F20003D9
:10BAE0001B6883420FD1586843F2F411C2F200017F
:10BAF000086010E042685A6041605A688242F9D09A
:10BB000013461BB907E033B14FF000015A68824277
:10BB1000F0D01346F5E7FEF7E5FD08BD0160436090
:10BB2000826043F2D803C2F200031A68C260186050
:10BB3000704700BF70B582B006464FF000038DF825
:10BB400007300D4601B10B7043F29800C2F20000BD
:10BB5000046874B121684B6843B130460DF10701A8
:10BB60002A46984710B19DF8070013E06468002C3E
:10BB7000F0D10B2E05DC0C2E03D83046FAF750F826
:10BB800008E02DB14FF005022A704FF0000001E0EF
:10BB90004FF0000002B070BD70B582B006464FF0A5
:10BBA00000038DF807300D4601B10B7043F2980089
:10BBB000C2F20000046874B121688B6843B130465A
:10BBC0000DF107012A46984710B19DF807001BE0C8
:10BBD0006468002CF0D10B2E0DDC0C2E0BD83046F7
:10BBE000FAF734F88DF8070010B13046FAF774F818
:10BBF0009DF8070008E02DB14FF005022A704FF0C4
:10BC0000000001E04FF0000002B070BD70B582B0DE
:10BC100006464FF000038DF807300D4601B10B705A
:10BC200043F29800C2F20000046874B12168CB6846
:10BC300043B130460DF107012A46984710B19DF8EF
:10BC4000070013E06468002CF0D10B2E05DC0C2EED
:10BC500003D83046F9F7CAFF08E02DB14FF00502CE
:10BC60002A704FF0000001E04FF0000002B070BDFC
:10BC700070B582B006464FF000038DF807300D46D0
:10BC800001B10B7043F2C800C2F2000004685CB15D
:10BC900021688B682BB130460DF107012A46984781
:10BCA00058B96468002CF3D1092E0CDC0A2E0AD88E
:10BCB0003046F5F789FC8DF807009DF80700003045
:10BCC00018BF012008E02DB14FF006022A704FF096
:10BCD000000001E04FF0000002B070BDF0B583B08D
:10BCE00005460E464FF000038DF8073043F2C800BA
:10BCF000C2F200000468E4B14FF000072168CA688E
:10BD00001AB1284631469047F0B923689B6833B191
:10BD100028460DF106010DF10702984700E038466C
:10BD20009DF8071099B9646814B10028E6D004E0C2
:10BD300018B9092D0DDC0A2D0ED82846314607F01A
:10BD40007DF94FF0000009E04FF0000006E00846E2
:10BD500004E04FF0060001E04FF0060003B0F0BD34
:10BD600070B582B005460E464FF000038DF80730DF
:10BD700012B11946FFF7B2FF43F2C800C2F2000049
:10BD800004686CB121684B68284631460DF1070202
:10BD9000984710B19DF8070012E06468002CF1D1BB
:10BDA000092D08DC0A2D09D828463146F5F72EFC66
:10BDB0004FF0000004E04FF0060001E04FF00600F5
:10BDC00002B070BD08B54FF0000001464FF001020F
:10BDD000FFF7C6FF08BD00BF70B582B005460E462E
:10BDE0004FF000038DF8073043F2A800C2F20000C4
:10BDF00004689CB121684B68284669460DF107022A
:10BE0000984728B10EB1009830609DF8070014E003
:10BE100064681CB19DF80720002AEBD0012D07D8DB
:10BE20004EB12846F6F776FD30604FF0000004E092
:10BE30004FF00F0001E04FF0000002B070BD00BFF6
:10BE400070B582B005460E464FF000038DF80730FE
:10BE500043F2F410C2F20000046884B121684B6818
:10BE6000284631460DF10702984710B19DF80700AA
:10BE700010E064681CB19DF80720002AEED03DB99F
:10BE80004FF000003146F6F727FC4FF0000001E0CC
:10BE90004FF00E0002B070BD70B582B005460E4680
:10BEA0004FF000038DF8073043F2F410C2F20000A7
:10BEB0000468A4B121688B685BB1284669460DF11E
:10BEC0000702984728B10EB1009830609DF807002E
:10BED00014E064681CB19DF80720002AEAD045B937
:10BEE00056B14FF00000F6F739FD30604FF000001A
:10BEF00004E04FF0060001E04FF0000002B070BD1A
:10BF00002DE9F04F2DED048B8BB083469246914284
:10BF100064D289464FF000089FED379A9FED328B2F
:10BF2000DFED369A32A7D7E900674FF000044FF0F3
:10BF30000005C3F6E0758DED019ABBF1020F05D146
:10BF40005FFA89F001A9FFF7A7FF04E05FFA89F023
:10BF500001A9FFF741FF08EB48030AAAD01800F82F
:10BF6000209C01980CF030FA53EC182B0CF0A4FD37
:10BF700008B1CDED019A01980CF026FA32463B4605
:10BF80000CF0C0FB22462B460CF078FA0CF0E2F9DC
:10BF900081B208EB48030AAAD31803F81E1C4FEA23
:10BFA000112003F81F0C08F10108B8F10A0F06D0A0
:10BFB0000AF1FF3149450DD1B8F1000F0AD008EB65
:10BFC00048024FF007005946D2B202ABFFF722FAFF
:10BFD0004FF0000809F10109CA45ACD80BB0BDEC1F
:10BFE000048BBDE8F08F00BF9831CB64FE0F70402A
:10BFF0000000000000E06F4000000000F37F80437D
:10C000002DE9F04F9FB040F6C410FCF799F84FF0BF
:10C0100002004FF0000143F2B003C2F20003DA78ED
:10C02000FFF76EFF4FF0010002904FF0000BDA4671
:10C03000D94607464CF6CD41CCF6CC4103914FF0A2
:10C040007D00FCF77DF88DF83790C8464E464C468B
:10C0500013E045F0800504F10804E4B216A9725C0F
:10C06000AA4202D016ABF554B84606F101069DF877
:10C070003750002D50D1202E4ED020460DF13701E3
:10C08000FFF758FD051C18BF012504F10102D0B2CD
:10C090000DF13701FFF74EFD10B145F00205EDB28D
:10C0A00004F10203D8B20DF13701FFF743FD08B1E7
:10C0B00045F0040504F10300C0B20DF13701FFF7AC
:10C0C00039FD08B145F0080504F10401C8B20DF1CD
:10C0D0003701FFF72FFD08B145F0100504F1050207
:10C0E000D0B20DF13701FFF725FD08B145F020056D
:10C0F00004F10603D8B20DF13701FFF71BFD08B1BB
:10C1000045F0400504F10700C0B20DF13701FFF71B
:10C1100011FD00289DD19EE7B8F1000F02D1BAF1C0
:10C12000000F0CD14FF002004946F2B216ABFFF7F8
:10C1300071F94FF03200FCF703F8019701E0CDF8F8
:10C1400004908DF83790C8464E464C4613E045F0B3
:10C15000800504F10804E4B20EA8315CA94202D0C3
:10C160000EAAB554B84606F101069DF83750002DC9
:10C1700050D1202E4ED020460DF13701FFF778FD2B
:10C18000051C18BF012504F10100C0B20DF13701F3
:10C19000FFF76EFD10B145F00201CDB204F10202CD
:10C1A000D0B20DF13701FFF763FD08B145F004058A
:10C1B00004F10303D8B20DF13701FFF759FD08B1BF
:10C1C00045F0080504F10400C0B20DF13701FFF796
:10C1D0004FFD08B145F0100504F10501C8B20DF19D
:10C1E0003701FFF745FD08B145F0200504F10602CF
:10C1F000D0B20DF13701FFF73BFD08B145F0400526
:10C2000004F10703D8B20DF13701FFF731FD002823
:10C210009DD19EE7B8F1000F02D1BAF1010F0AD10A
:10C2200048464946F2B20EABFFF7F4F84FF0320041
:10C23000FBF786FF019743F2B003C2F200039A783E
:10C24000B2B1039EA6FB0A044FEA141000EB800172
:10C25000BAEB810F0CD138464946FFF751FE4FF03B
:10C260003200FBF76DFFBBF1000F40F0B88003E038
:10C27000BBF1000F40F09C8005A849464FF020021A
:10C280000DF0AEFF43F2B006C2F20006B478ACB3D4
:10C290004D466FEA0900011901F0010209F0070398
:10C2A00007FA03F69DF8140046EA00018DF8141011
:10C2B00005F10105A542C0F2B3801FE01EAB03EB00
:10C2C000D50605F0070007FA00F216F8641C42EAEA
:10C2D000010306F8643C05F101051EA800EBD50238
:10C2E00005F0070107FA01F312F8646C43EA06004F
:10C2F00002F8640C05F10105A542DFDB4FF00700F1
:10C300004FF011014FF01E0205ABFFF783F84FF01D
:10C310003200FBF715FF05A849464FF020020DF04B
:10C320005FFF43F2B004C2F20004E578A5B34B46C8
:10C330006FEA0902511901F0010609F0070007FA36
:10C3400000F49DF8142044EA02018DF8141003F162
:10C3500001039D4250DC1FE01EAC04EBD30203F04E
:10C36000070007FA00F612F8641C46EA010402F816
:10C37000644C03F101031EAA02EBD30403F007008F
:10C3800007FA00F614F8641C46EA010204F8642C6B
:10C3900003F101039D42DFDC4FF007004FF0120173
:10C3A0004FF01E0205ABFFF735F84FF0060B16E015
:10C3B000019AA2B9BBF1020F11D1029D7DB943F2DE
:10C3C000B003C2F20003DA784AB14FF002004946E6
:10C3D000FFF796FD4FF03200FBF7B2FE0297BAF17D
:10C3E000000F06D10BF1FF3BCDF808904FF0280A63
:10C3F00025E60AF1FF3A22E6002EADD01EAE06EB8E
:10C40000D30403F0070007FA00F214F8641C42EAB0
:10C41000010604F8646C03F101039D429CDCBBE758
:10C42000002A3FF44BAF1EAA02EBD50305F0070626
:10C4300007FA06F013F8641C40EA010203F8642CC2
:10C4400005F10105A542FFF639AF57E72DE9F04F99
:10C450002DED028B87B008EE100A0C461746994660
:10C46000129E1399B5EEC08AF1EE10FA54BF002562
:10C470000125A84604F1FF33D8B2082807D8092AB5
:10C4800005D8A24601F1FF32944205D808E001F137
:10C49000FF339C4240F2CD8001F1FF34E4B2C8E0AA
:10C4A00018EE100A0CF080FB48B930464FF03F01FF
:10C4B00022460DF095FE4FF000013155C4E018EE14
:10C4C000100A0DF075F806EE900AF2EE047AF4EE1A
:10C4D000E76AF1EE10FA0DDB4FF00100B0EE677A7B
:10C4E00000F1010067EE877AF4EEE76AF1EE10FAE8
:10C4F000F6DA03E04FF00100F2EE047A2146431928
:10C50000A34200F39680C0EB040EC5EB0E0202F1CD
:10C51000FF3E4EF21C7AC0F6030ADFED9C4AF6EEAF
:10C52000003AB2EE044AC0EB040CC5EB0C0303F076
:10C53000010BBEF1000F00F38F808AE0BEF1000F07
:10C5400004DDBE45B4BF72463A4601E04FF000023A
:10C550005AF8223003EE103AB8EE430A20EE027A7F
:10C56000B4EEE47AF1EE10FA48BF37EE237ABDEE6E
:10C57000C73A13EE10CABCFBF3FB06EE10BAB8EED6
:10C58000C65AB4EEE75AF1EE10FA0DDB00F1010CD9
:10C5900087EE006A67EE847A0EF1FF3E6046BEF1D8
:10C5A000000200F3C380BEE013EE105AB5FBF3F4B3
:10C5B00003FB14542CB916EE107A002F08BF4FF06D
:10C5C0000008B9F1000F07D0C8EB0103181A002AC0
:10C5D00018BF0138831A01E04FF0000301F1010197
:10C5E000B8F1000F04D04EF21C37C0F6030703E089
:10C5F0004BF60077C0F6030722B14EF22030C0F6AA
:10C60000030003E04BF60070C0F603004EF2343531
:10C61000C0F60305009501978DED026A0390049220
:10C62000059430464EF22432C0F603020DF0A2F912
:10C630000AE03046002D0CBF2B212D2122460DF0A3
:10C64000CFFD4FF00000305507B0BDEC028BBDE8C8
:10C65000F08F4FF0000203E0BE45B4BF72463A4689
:10C660005AF8223000EE103AB8EE405A65EE260A2B
:10C67000F4EEE40AF1EE10FA48BF70EEA30ABDEE44
:10C68000E03A13EE10CABCFBF3FC06EE10CAF8EE5B
:10C69000C65AF4EEE75AF1EE10FA85DB00F101001C
:10C6A00080EE852A67EE847A0EF1FF3E42199142B0
:10C6B000BFDBBBF1000F3FF441AFBEF1000F02DC66
:10C6C0004FF0000203E0BE45B4BF72463A465AF846
:10C6D000223001EE103AF8EE411A21EE822AB4EE31
:10C6E000E42AF1EE10FA48BF32EE232ABDEEC23A38
:10C6F00013EE10BABBFBF3FB06EE10BAF8EEC62A37
:10C70000F4EEE72AF1EE10FAFFF64EAF00F1010069
:10C7100082EE212A67EE847A0EF1FF3E4319994298
:10C72000BFF60CAF85E74FF0000202E0BA42A8BFA7
:10C730003A465AF8223006EE903AF8EE660A20EEB3
:10C74000861AB4EEE41AF1EE10FA48BF31EE231A5D
:10C75000BDEEC13A13EE10BABBFBF3FB06EE10BA06
:10C76000F8EEC65AF4EEE75AF1EE10FAFFF61CAFF7
:10C770000CF1010081EE202A67EE847A0EF1FF3E73
:10C7800042199142BFF6DAAE53E700BF0000004BFA
:10C79000F8B505460F46F4F7A7F8064640F2A06242
:10C7A000C1F200024FF4117303FB05F01418115885
:10C7B00011B18A682846904784F820724FF000052E
:10C7C000C4F81052C4F81452C4F80451C4F8085103
:10C7D0003046F4F793F804F5097029464FF0080243
:10C7E000F4F73CF8F8BD00BF70B588B0054640F2DC
:10C7F000A064C1F200044FF4117303FB004494F8E9
:10C80000200200284AD043F29C01C2F200010A88AB
:10C810004FF6FF76B24204D0D0B24FF00401FFF7DA
:10C82000B7FF28464FF00001FFF7B2FF43F29C0626
:10C83000C2F2000635804EF24030C0F603004FF0E1
:10C84000070142F24932C0F60302FBF73BFCC4F891
:10C850001C02246830784FF0010300934FF000026F
:10C8600001924AF6ED01C0F6020102914AF6E56333
:10C87000C0F6020303934AF60561C0F60201049173
:10C880004AF64D43C0F602030593069264684FF4DE
:10C8900016514FF00803A047FEF70AF908B070BD23
:10C8A000704700BF08B5B0F1FF3F04D040B9024661
:10C8B000F6F782F808BD4FF000000246F6F77CF864
:10C8C00008BD00BF38B506F0ADFB43F2B403C2F2B9
:10C8D00000034FF001021A704FF000042546E0B249
:10C8E00029462A46FFF73CFA40B904F10104E0B2B8
:10C8F00029462A46FFF734FA002867D04FF0FF3068
:10C900004FF00001FFF7CEFF4FF000004FF00001A5
:10C91000FFF796FA43F2F411C2F200010C6834B149
:10C920002368DA6802B190476468002CF8D143F2BA
:10C93000AC00C2F2000004683CB121680B680BB186
:10C94000A06898476468002CF7D1F9F791FEFEF7CC
:10C950009FF940F2A062C1F2000292F8200204287E
:10C9600006D028B14FF000004FF00401FFF710FF90
:10C9700040F2A061C1F2000191F86434042B06D0AA
:10C980002BB14FF001004FF00401FFF701FF40F21F
:10C99000A062C1F2000292F8A806042806D028B1CD
:10C9A0004FF002004FF00401FFF7F2FE40F2A061E9
:10C9B000C1F2000191F8EC38042B06D02BB14FF0F6
:10C9C00003004FF00401FFF7E3FE38BD04F101045A
:10C9D000B4F5807F83D191E738B5054643F29404DE
:10C9E000C2F200042068FBF757FC4FF000032360FD
:10C9F0008DB14EF25030C0F603004FF007014CF6F7
:10CA00001D32C0F60202FBF75DFB43F2A002C2F248
:10CA10000002106038BD43F2A004C2F20004206896
:10CA2000FBF73AFC4FF00000206041F25A02C2F2DC
:10CA300000021070FAF7C8FAFFF744FF0AF036FE5A
:10CA400043F29C01C2F2000108884FF6FF7398423E
:10CA500004D0C0B24FF00401FFF79AFE38BD00BF0A
:10CA600070B543F2F810C2F200004EF26031C0F629
:10CA70000301FAF707FF43F29C03C2F200034FF6EB
:10CA8000FF721A8040F2A064C1F200044FF0040665
:10CA900084F820624FF00005C4F81C522846FBF7CA
:10CAA0002BF9206084F86464C4F860544FF00100EE
:10CAB000FBF722F9C4F8440284F8A866C4F8A45627
:10CAC0004FF00200FBF718F9C4F8880484F8EC680A
:10CAD000C4F8E8584FF00300FBF70EF9C4F8CC0691
:10CAE00043F26800C2F200004EF26C31C0F603015E
:10CAF000FAF7C8FE43F2B800C2F200004EF210711D
:10CB0000C0F603012A462B46FFF708F8FDF7EAFDB9
:10CB10004FF00100FFF760FF70BD00BF2DE9F04F3F
:10CB20002DED048BABB01CAF26AC4DF60C25C0F63A
:10CB3000030595E80F0084E80F00A7604AF27163CF
:10CB4000C0F60203E36020462AA9F7F735FB22AEC0
:10CB500095E80F0086E80F00B7604AF28D60C0F6D6
:10CB60000200F06030462146F7F726FB4FF0000444
:10CB70001B9443F26800C2F200002146FAF79AFEC5
:10CB800043F2CC01C2F200010C72FFF79BFE0AF0E7
:10CB90008DFD4FF00200FFF727FE43F2E012C2F2D4
:10CBA000000215680DBB0FF0D7F8F0B9F5F7ECF8F7
:10CBB00010F0C20F19D14FF00300FEF707FC4FF43D
:10CBC0007A754FF032063046FBF7BAFAF5F71CFCDF
:10CBD00005F1FF343046FBF7B3FAF5F715FC651E97
:10CBE000F1D14FF00000FEF7F1FB43F2DC03C2F29B
:10CBF00000034FF000041C604FF00100187040F279
:10CC0000A066C1F2000606F519652846214642F6DF
:10CC100054220DF0E5FA41F25C00C2F20000214618
:10CC20004FF400520DF0DCFA06F5116021464FF08A
:10CC300040020DF0D5FA43F2E000C2F200002146B6
:10CC40004FF0FC020DF0CCFA21954FF00A01C6F826
:10CC5000B41920462946FDF7A7FC43F29002C2F220
:10CC60000002146043F2A403C2F200031C6043F20A
:10CC7000E015C2F200054FF030042C6040F20004D1
:10CC8000C0F6010494F82F0000F1010094F82E1072
:10CC900000EB0122101943F2DC13C2F2000318600A
:10CCA000FBF7DCFE0A902B68E15CFF2930D143F2F0
:10CCB000CC02C2F200024FF0010111721360219800
:10CCC000026A1AB102F1010250F8223043F2CC019B
:10CCD000C2F200014B604FF0FF00487243F2A00324
:10CCE000C2F200034FF000021A6043F29C01C2F24C
:10CCF0000001088840F2A062C1F200024FF41173F3
:10CD000003FB0021D1F81C02FBF784F805F0E6BA1A
:10CD100006F066F94FF000070997BA463C4601E075
:10CD20004FF000042CB94FF00000FEF731FD4FF03A
:10CD3000640404F1FF3441F25A06C2F20006357869
:10CD4000032D27D14FF000038DF8443043F2E0115A
:10CD5000C2F200010F88ADF845704FF007004FF0A8
:10CD600041014FF0040211ABFEF754FB41F25A06A9
:10CD7000C2F200063578032D15D14FF0000741F2BD
:10CD80005A06C2F200063846FEF702FD3078032844
:10CD9000F9D008E0022D06D141F25A00C2F200009B
:10CDA0004FF00302027043F2DC03C2F200031A7870
:10CDB00002F0E7016FF34511197043F2E015C2F27A
:10CDC00000052F68089743F2E016C2F2000640F211
:10CDD0000007C0F6010743F2DC08C2F200084EF279
:10CDE0004479C0F6030930683D5C00F10100306011
:10CDF00098F8003013F0010F0ED10AF1010A40F249
:10CE0000FF32924508D943F2CC06C2F200064FF039
:10CE10003600307205F0FCB90DF1700C2846494619
:10CE2000FEF77EF84DF6A051C0F6030151F825300B
:10CE30004DF6205BC0F6030B43F00100004733685A
:10CE4000FA5C0B9203F1010333600F2A05F2D881DB
:10CE50000DF1700C10465946FEF762F84EF6C831D7
:10CE6000C0F603010B9851F82030E5E73368FA5C0F
:10CE70000B9203F101033360102A02D9154605F025
:10CE8000C0B90DF1700C0B984EF64431C0F6030199
:10CE9000FEF746F84EF2AC41C0F603010B9851F88C
:10CEA0002030C9E73368FA5C0B9203F10103336069
:10CEB0000F2A02D9154605F0A4B90DF1700C0B9894
:10CEC0004EF68831C0F60301FEF72AF84DF66050A1
:10CED000C0F603000B9950F82130ADE73368FA5CD7
:10CEE0000B9203F1010333602F2A02D9154605F096
:10CEF00088B90DF1700C0B984EF60841C0F603018D
:10CF0000FEF70EF84EF2EC31C0F603010B9851F823
:10CF1000203091E73368FA5C0B9203F10103336030
:10CF20003B2A02D9154605F06CB90DF1700C0B982F
:10CF30004DF63021C0F60301FDF7F2FF4EF2A011CD
:10CF4000C0F603010B9851F8203075E73368FA5C9E
:10CF50000B9203F1010333603F2A02D9154605F015
:10CF600050B90DF1700C0B984DF62041C0F603013D
:10CF7000FDF7D6FF4DF62030C0F603000B9950F8B0
:10CF8000213059E73368FA5C0B9203F101033360F7
:10CF9000432A02D9154605F034B90DF1700C0B98EF
:10CFA0004EF2F041C0F60301FDF7BAFF4EF2006108
:10CFB000C0F603010B9851F820303DE7219E96F80A
:10CFC00046500DF1700CFDF751FA219F291897F882
:10CFD000502002F001000B181C9387F84730FF2BFC
:10CFE00094BF0023012387F850309BE6219E96F8DA
:10CFF00046500DF1700CFDF739FA2F181C97219946
:10D0000081F84770FF2F94BF0027012781F85070E7
:10D0100088E60DF1700CFDF729FA30B1219A92F8EB
:10D020004730181C18BF012001E04FF00000219E7E
:10D0300086F8470076E60DF1700CFDF717FA219D92
:10D0400095F84770384085F847006BE61D99A1F1C7
:10D05000FB011C9119E11D98A0F1FB001C90A1E1BE
:10D060001D9AA2F1FB021C92D2E11D9BA3F1FB03CE
:10D070001C936FE21D9EA6F1FB061C964FF0020169
:10D080001B9106E21D98A0F1FB001C901E9A1B92BA
:10D0900030E21D9BA3F1FB031C932AE11D9EA6F128
:10D0A000FB061C96ADE21D99A1F1FB011C91E9E282
:10D0B0001D9FA7F1FB071C971E981B9026E31D9A46
:10D0C000A2F1FB021C921E9B1B934FF000068DF8F1
:10D0D0006A60D4E31D99A1F1FB011C911E981B907D
:10D0E0004FF001028DF86A20C9E31D9BA3F1FB03F9
:10D0F0001C9300F061BC1D9DA5F1FB051C9500F083
:10D10000B6BC9DF874004FF00101FEF7E7FD8DF805
:10D110006B0000283FF406AE43F2CC04C2F20004D8
:10D12000207205F075B81D9E1C964FF001028DF817
:10D130006A201646219991F84700024205D09DF8D1
:10D1400070003146FEF7CAFD68B99DF86A204FEAC3
:10D1500042038DF86A301C9901F101011C9113F012
:10D16000FE02E7D10CE09DF86A60012E08D19DF81F
:10D170006B4043F2CC00C2F20000047205F048B8E4
:10D180000DF1700CFDF772F9CCE59DF8740005F017
:10D1900019FFC7E50DF1700CFDF768F91C9043F21B
:10D1A000E016C2F2000632681C9902EB41003060C2
:10D1B000FDF772F91C9001F0DDBE43F2DC03C2F210
:10D1C0000003197811F0280F06D01D9AB2F5005F00
:10D1D00034BF0022012204E01D9AFA2A94BF0022E3
:10D1E000012242B143F2CC04C2F200044FF0130119
:10D1F000217205F00DB841F25C06C2F200061D98DE
:10D20000335C1C93CBE7219A92F852601C96C6E7D8
:10D21000219890F850301C93C1E74FF0000A81E547
:10D220000DF1700CFDF722F91C90219F97F8471023
:10D230001B91FDF7D1F987F8470073E5219D95F81B
:10D24000470095F84610FDF7C7F985F8500069E5E5
:10D250000DF1700CFDF732F91E9B41F25C06C2F233
:10D260000006F25C1D9922EA0100F0545AE543F2EF
:10D27000E000C2F200004FF000014FF0FB020CF0A2
:10D28000AFFF4FE54FF000031C930DF1A80C1CF805
:10D29000386DFDF7EBF80146304608F0FBFC8DF8E1
:10D2A0006B0000283FF43EAD43F2CC04C2F2000410
:10D2B000207204F0ADBF07F0F3F833E507F0F8F89B
:10D2C0008DF86B0000283FF42DAD43F2CC02C2F282
:10D2D0000002107204F09CBF43F2DC17C2F2000798
:10D2E0003D681D99681807F0CFF81BE54FF0000066
:10D2F0001C901C9B40F2A066C1F200064FF4117115
:10D3000001FB036292F8200203283FD140F2A0679C
:10D31000C1F2000701FB03F303F58876B919FB1886
:10D3200003F104034FF00000D1F80021FE2A94BF5E
:10D33000551C0025D1F80471BD4214BF00250125FC
:10D3400065F30000BA4214BF0022012262F34100DB
:10D35000D3F80051FE2D94BF013500250DF1A80C26
:10D360004CF8385DD3F80461B54214BF002501259F
:10D3700065F38200D3F80811D1F1010338BF00230F
:10D3800063F3C300C0B2FDF759F8CBE443F2CC0419
:10D39000C2F200044FF04803237204F039BF4FF08B
:10D3A00000001C901C9E40F2A062C1F200024FF4EB
:10D3B000117101FB062393F8200203281CD140F2CF
:10D3C000A067C1F2000701FB0675D5F81022D5F859
:10D3D0001412531AB3F5807F88BF03F580731C9332
:10D3E0001C98FF2884BFFF201C900DF1A80C1CF88E
:10D3F000380DFDF723F895E443F2CC04C2F20004A3
:10D400004FF04806267204F003BF4FF000061C964A
:10D410001C9B40F2A062C1F200024FF4117101FBAB
:10D42000032090F82062032E24D140F2A067C1F2BD
:10D43000000701FB037505F58876D6F80021D6F8BC
:10D440000411501AB0F5807F88BF00F580701C90E1
:10D450000DF1700CFDF70AF88DF86A001C9B9842DC
:10D4600038BF1C90D6F804711C9DEA19D1B2C6F8D9
:10D47000041157E443F2CC04C2F200044FF0480315
:10D48000237204F0C5BE4FF000061C964FF0020058
:10D490001B901C9B40F2A062C1F200024FF411717C
:10D4A00001FB032696F82002032815D140F2A0675D
:10D4B000C1F2000701FB03750DF1700C1B984AF2D5
:10D4C000ED51C0F602014AF20162C0F6020205F512
:10D4D0008873FDF705F825E443F2CC04C2F200049A
:10D4E0004FF04803237204F093BE4FF000021C92E9
:10D4F0001D991B911C9E40F2A060C1F200004FF4E8
:10D50000117303FB060292F82012032916D140F290
:10D51000A067C1F2000703FB06750DF1700C1B98A4
:10D520004AF2ED51C0F602014AF20162C0F602026F
:10D5300005F58873FEF7CCF8FFF7F4BB43F2CC0493
:10D54000C2F200044FF04806267204F061BE4FF0AC
:10D5500000001C901C9B40F2A062C1F200024FF43C
:10D56000117101FB032696F8200203283DD140F2F9
:10D57000A067C1F2000701FB037505F588750DF181
:10D58000700CFCF773FF8DF86A00D5F804211C922B
:10D590004FF000011B91D5F800711346974207D058
:10D5A000AE5C864219D04FF001024FF0000E0CE045
:10D5B0004FF0FF001B9010E002F10101EE5C86428B
:10D5C00002D11C931B9208E00A46FF2B14BF0133C3
:10D5D0007346BB42F0D11C93EAE70DF1700C9DF845
:10D5E0006C00FCF72BFFFFF79DBB43F2CC04C2F2AB
:10D5F00000044FF04803237204F00ABE4FF000030A
:10D600001C931C9E40F2A062C1F200024FF4117103
:10D6100001FB062090F82032032B27D140F2A065B1
:10D62000C1F2000501FB065707F58875D7F81462AB
:10D63000D7F81022964212D00DF1700CFCF716FFAD
:10D640008319DFB21C970DF1700CE85DFCF7F6FE54
:10D650004FF00005219E86F85050FFF763BB4FF056
:10D660000101219880F85010FFF75CBB43F2CC0415
:10D67000C2F200044FF04806267204F0C9BD4FF014
:10D6800000021C921C9840F2A063C1F200034FF408
:10D69000117101FB003696F82022032A28D140F2AE
:10D6A000A067C1F2000701FB007505F58876D6F882
:10D6B0000431D6F800118B4213D00DF1700CF05CE0
:10D6C000FCF7BCFED6F80471FF2F14BF013700270A
:10D6D000C6F804714FF00005219E86F85050FFF700
:10D6E00021BB4FF00102219880F85020FFF71ABBB0
:10D6F00043F2CC04C2F200044FF04800207204F060
:10D7000087BD4FF000031C931D991B9143F2DC125F
:10D71000C2F20002D2F800801B9F08EB070640F21D
:10D720000000C0F60200864208D943F2CC06C2F2DD
:10D7300000064FF01F02327204F06ABD1C9B032BDF
:10D7400008D943F2CC01C2F200014FF03700087251
:10D7500004F05EBDF1780D2908D943F2CC04C2F281
:10D7600000044FF03703237204F052BD40F2A0656D
:10D77000C1F200054FF4117202FB035090F8203201
:10D780003BB118F8071021B10FE04846FEF700F84A
:10D7900005E04CF24F354FF09609DDF828B0FBF765
:10D7A0005DF9CBEB0002AA42EFD918F80770032FFE
:10D7B0003FF6B8AADFE807F002080F169DF87000E0
:10D7C000FFF712F8FFF7AEBA9DF87000314608F087
:10D7D00083FAFFF7A7BA9DF87000314606F0BCFD4A
:10D7E000FFF7A0BA9DF870504DF61C29C0F603094A
:10D7F00096F8028008EB480809EB080728464FF026
:10D800000301FEF7C5FF4FF4117000FB05F340F272
:10D81000A061C1F20001C85800283FF483AAF6783D
:10D820004EF29022C0F6030252F8261019F8082092
:10D830007B78BF7800974FF0000601964AF6BD1737
:10D84000C0F6020702974AF6FD17C0F602070397D3
:10D850004AF62D27C0F6020704974AF64D47C0F650
:10D8600002070597069646682846B047FFF75ABA5A
:10D870004FF000031C931D991B918DF86A301C9B7F
:10D8800040F2A060C1F200004FF4117101FB0306E9
:10D8900096F82022032A79D140F2A065C1F2000552
:10D8A00001FB035707F5887943F2DC10C2F2000050
:10D8B0000168219EB26B01EB020B885CFF285CD0F3
:10D8C000D8464FF001074FF0000B0894CDF82CA07C
:10D8D000BA4698F8014004EB002343F2DC10C2F290
:10D8E00000000668F218D9F804111C919DF86A50DE
:10D8F0001DB1F75C02F1010200E05F4602F1FF3466
:10D900009DF86A302BB177B9089C5546DDF82CA0FC
:10D9100005E0607838B9089C5546DDF82CA01C99C4
:10D92000C9F804112BE01C99D9F800618E4218D077
:10D9300014F8016F19F801501B9A3AB930460BF0F0
:10D94000BDFFC6B228460BF0B9FFC5B2AE4208D142
:10D950001C9BFF2B14BF01335B461C9307F1FF3761
:10D96000CEE70AF1010A18F8020FFF28B1D1089C8E
:10D97000DDF82CA04FF0000501E04FF000050DF19F
:10D98000700CE8B2FCF75AFDFFF7CCB943F2CC04B7
:10D99000C2F200044FF04803237204F039BC4FF088
:10D9A00000001C901E9E1B964FF001028DF86A200D
:10D9B00065E74FF000021C921C9E40F2A063C1F28A
:10D9C00000034FF4117000FB063191F82022032A66
:10D9D00031D140F2A065C1F2000500FB065707F502
:10D9E00088750DF1700CFCF741FD8DF86A004FF061
:10D9F00000031C93D5F80471D5F800118F4212D0A2
:10DA0000EA5D82420FD14FF00006FF2F14BF0137AD
:10DA100037468F4202D1C5F8047104E0EB5D8342C2
:10DA2000F3D0C5F804710DF1700C4FF00000FCF755
:10DA300005FDFFF777B943F2CC04C2F200044FF0C2
:10DA40004806267204F0E4BBFBF708F80A9D401B69
:10DA50000DF1700C4CF24F37B8428CBF0020012002
:10DA6000FCF7ECFCFFF75EB94FF000001C901C9E29
:10DA700040F2A062C1F200024FF4117101FB0623D3
:10DA800093F82052032D7FF44DA940F2A067C1F214
:10DA9000000701FB067000F10406D0F80811D6F863
:10DAA000002102F10102914238BF01F580718B1A09
:10DAB000FF2B34BF1D46FF250DF1700CE8B2FCF7BB
:10DAC000BDFCFFF72FB91D9F41F25C00C2F20000C0
:10DAD000C65D06F1FF31C155FFF724B943F2DC0200
:10DAE000C2F20002137813F0280F06D01D98B0F58B
:10DAF000005F34BF0020012004E01D98FA2894BF85
:10DB00000020012040B143F2CC04C2F200044FF0E7
:10DB10001301217204F07CBB1D9E41F25C01C2F234
:10DB200000018A5D02F1FF33D8B2885500283FF426
:10DB3000F9A81E9E1C9601F01DBA43F2DC02C2F247
:10DB40000002137813F0280F06D01D98B0F5005F7F
:10DB500034BF0020012004E01D98FA2894BF002063
:10DB6000012040B143F2CC04C2F200044FF013068E
:10DB7000267204F04DBB1D9E41F25C01C2F2000111
:10DB80008A5D02F1FF33D8B28855002842F013872E
:10DB9000FFF7C8B843F2DC01C2F200010A7812F0C4
:10DBA000280F06D01D9BB3F5005F34BF002301236F
:10DBB00004E01D9BFA2B94BF0023012343B143F2E1
:10DBC000CC04C2F200044FF01300207204F020BB1A
:10DBD0001D9841F25C06C2F20006315C01F1FF3291
:10DBE000D3B23354002B02F0E686FFF79BB8219D99
:10DBF00095F8517007F1FF3685F85160FFF792B83C
:10DC0000219991F8472002F1FF3381F84730FFF75F
:10DC100089B82198C06C0BF0CBFC219DE864FFF71C
:10DC200081B8219F97ED137AD7ED127A37EE270A44
:10DC300087ED130A2199C86C0AF096FF30B14FF0B6
:10DC40000200219981F85000FFF76CB8219EF06C1A
:10DC50000AF09AFF30B14FF00102219B83F8502067
:10DC6000FFF760B84FF00007219D85F85070FFF76F
:10DC700059B89DF87400219901F14C01FEF7ACF8F8
:10DC80008DF86B0000283FF44DA843F2CC04C2F29B
:10DC90000004207204F0BCBA9DF87400219EF16C5F
:10DCA000FEF7CEF88DF86B0000283FF43BA843F256
:10DCB000CC01C2F20001087204F0AABA219AD06C19
:10DCC0000AF062FF20B9219B986C0AF05DFF30B129
:10DCD0004FF00302219B83F85020FFF723B82198CF
:10DCE000D0ED138A90ED128A78EEC80A10EE900AF1
:10DCF0000BF05EFC09EE100A18EE900A18EE101AEE
:10DD00000BF0D4F801464FF07E500BF0CFF89FEDAA
:10DD1000CF1A01EE900A21EE812AB4EEC29AF1EEFA
:10DD200010FA06D84FF00006219981F85060FEF7EE
:10DD3000F9BF219DD5ED132A95ED123AF4EEC32AD1
:10DD4000F1EE10FA05DD4FF0010785F85070FEF78F
:10DD5000E9BFF4EEC32AF1EE10FA4CBF022203220F
:10DD600085F85020FEF7DEBF2198D0ED133AB7EECC
:10DD7000004A73EEC44AC0ED134A219EF06C0AF0CB
:10DD800003FF30B14FF00305219B83F85050FEF79D
:10DD9000C9BF2199D1ED138A9FEDAD8A38EEC89A9B
:10DDA00019EE100A0BF004FC09EE100A18EE900AA6
:10DDB00018EE101A0BF07AF801464FF07E500BF077
:10DDC00075F8DFEDA23A04EE100A64EE234AB4EED1
:10DDD000E49AF1EE10FA22D9219F97ED138ADFED34
:10DDE0009C8A38EE285A15EE100A0BF0E1FB08EE7B
:10DDF000900A18EE100A6FF052510BF057F80146D6
:10DE00004FF07E500BF052F8DFED905A06EE100AFC
:10DE100066EE256AF4EEE68AF1EE10FA06D84FF0C7
:10DE20000407219A82F85070FEF77CBF219AD56CC6
:10DE300028460BF0BDFB08EE100A28464FF0000103
:10DE40000BF034F801464FF07E500BF02FF8DFED69
:10DE50007F7A07EE100A27EE270AB4EEC08AF1EEA9
:10DE600010FA06D84FF00006219981F85060FEF7AD
:10DE700059BF219BD3ED130AF5EEC00AF1EE10FA5B
:10DE800005DD4FF0010083F85000FEF74BBFF5EEC3
:10DE9000C00AF1EE10FA4CBF0222032283F8502090
:10DEA000FEF740BF219D95ED125AD5ED135A85EE30
:10DEB000256A85ED136ABDE6219EF06C0AF050FEDE
:10DEC000002841F05580FEF72DBF2199CE6C3046D9
:10DED0000BF06EFB08EE100A30464FF000010AF01E
:10DEE000E5FF01464FF07E500AF0E0FFDFED576A94
:10DEF00007EE100A67EE267AB4EEE78AF1EE10FA22
:10DF000001F33680FEF70EBF219AD06C0AF028FE8E
:10DF1000002801F02D80FEF705BF219B93ED130A29
:10DF2000D3ED120AB4EEE00AF1EE10FA81F220808D
:10DF3000FEF7F8BE219890ED131AD0ED121AB4EE48
:10DF4000E11AF1EE10FA01F31380FEF7EBBE21990E
:10DF500091ED132AD1ED122AB4EEE22AF1EE10FA75
:10DF600041F20680FEF7DEBE219E96ED133AD6ED15
:10DF7000123AB4EEE33AF1EE10FA00F1F987FEF747
:10DF8000D1BE219AD66C30460BF012FB08EE100A77
:10DF900030464FF000010AF089FF01464FF07E50F5
:10DFA0000AF084FF9FED294A04EE900A24EE845A79
:10DFB000B4EEC58AF1EE10FA40F2DA87FEF7B2BE8F
:10DFC000219FF86CFCF78AF8F8640DF1700C4FF0A3
:10DFD0000000FCF71FFBFEF7A5BE1D9BF62B08D922
:10DFE00043F2CC04C2F200044FF01203237204F097
:10DFF0000FB9219DE86C0AF0B3FD38B9219991ED74
:10E00000136AF6EE006A36EE268A06E0219890ED55
:10E01000138AF6EE005A38EE658A18EE100A0AF0F6
:10E020009FFDF8B99FED0B7AB4EEC78AF1EE10FAB6
:10E0300004DC18EE100A0AF097FD98B14FF00106C3
:10E04000219F87F850606FF000463AE000000034EE
:10E05000FFFF7F4BFEFFFF4AFEFFFFCA0000804329
:10E06000000080C318EE100A0AF07AFD98B15FED47
:10E07000067AB4EEE78AF1EE10FA04D418EE100A2C
:10E080000AF072FD38B14FF00100219981F850007B
:10E090004FF0004615E018EE100A0AF075FD38B191
:10E0A0004FF00205219B83F850504FF0000608E026
:10E0B000BDEEC88A18EE106A4FF00007219A82F868
:10E0C00050704FEA066242EA166506F47F4345EA5D
:10E0D000032006F47F0140EA112643F2E007C2F272
:10E0E00000071D9ABE50FEF71DBE1D98F62808D9E0
:10E0F00043F2CC04C2F200044FF01202227204F088
:10E1000087B843F2E005C2F200052E584FEA0661D7
:10E1100041EA166706F47F4247EA022306F47F00CD
:10E1200043EA102500EE105AF8EEC00A219EC6ED13
:10E13000130A1FED381AF4EEC10AF1EE10FA06DCEC
:10E140005FED3B1AF4EEE10AF1EE10FA05D54FF05F
:10E15000010786F85070FEF7E5BD4FF0000186F824
:10E160005010FEF7DFBD0DF1700C4FF00100FCF711
:10E1700051FA219BD86CFBF7DBFF219DE864FEF789
:10E18000D1BD219890ED132AF7EE002A32EE223A03
:10E1900080ED133AF1E52198C06C0AF0F5FC50B11E
:10E1A000219D4FF0000385F847304FF0040085F8BB
:10E1B0005000FEF7B7BD219E96ED131AB5EEC01ABA
:10E1C000F1EE10FA23DB1FED5B3AB4EEC31AF1EE69
:10E1D00010FA0FD5FCEEC13A13EE901A0DF1700C47
:10E1E000C8B2FCF72BF94FF00007219A82F8507063
:10E1F000FEF798BD0DF1700C4FF0FF00FCF71EF913
:10E200004FF00200219E86F85000FEF78BBDB5EE60
:10E21000C01AF1EE10FA7EF585AD5FED6F1AB4EE1F
:10E22000E11AF1EE10FA11DDB1EE412AFCEEC22A3C
:10E2300012EE902A0DF1700CD0B2FCF7FFF84FF0FF
:10E240000105219B83F85050FEF76CBD0DF1700C59
:10E250004FF0FF00FCF7F2F84FF00301219F87F821
:10E260005010FEF75FBD43F2DC06C2F200063178C3
:10E2700011F0280F08D01D9A02F10102B2F5005FDB
:10E2800034BF0022012206E01D9A02F10102FA2A9F
:10E2900094BF0022012242B143F2CC04C2F2000436
:10E2A0004FF01303237203F0B3BF219F97ED134A7E
:10E2B000FDEEC44A14EE905A2BB21C9398B2C5F3EB
:10E2C000072646EA002141F25C02C2F200021D9FCD
:10E2D000D153FEF727BD43F2DC00C2F200000678FE
:10E2E00016F0280F08D01D9901F10101B1F5005F6A
:10E2F00034BF0021012106E01D9901F10101FA2935
:10E3000094BF0021012141B143F2CC04C2F20004C8
:10E310004FF01302227203F07BBF219D95ED135A3B
:10E32000FCEEC55A15EE902A97B21C974FEA1723B8
:10E3300043EA072041F25C06C2F200061D997052C2
:10E34000FEF7F0BC1D9D219FBD64FEF7EBBC1D9840
:10E35000219BD864FEF7E6BC0DF1700CFCF786F843
:10E3600006EE100AF8EE466A219EC6ED136AFEF725
:10E37000D9BC43F2DC01C2F200010A7812F0280F86
:10E3800008D01D9800F10100B0F5005F34BF0020F7
:10E39000012006E01D9800F10100FA2894BF00203A
:10E3A000012040B143F2CC04C2F200044FF0130349
:10E3B000237203F02DBF41F25C05C2F200051D9FE0
:10E3C000EB5B4FEA132646EA03218AB207EE902A56
:10E3D000B8EE670A219880ED130A9FEDC97AB4EE72
:10E3E000C70AF1EE10FAFEF69DACDFEDC60A30EE7C
:10E3F000601A80ED131AFEF795BC43F2DC06C2F2F8
:10E400000006317811F0280F08D01D9A02F10102A0
:10E41000B2F5005F34BF0022012206E01D9A02F12E
:10E420000102FA2A94BF0022012242B143F2CC0435
:10E43000C2F200044FF01300207203F0E9BE41F273
:10E440005C05C2F200051D9FE85B4FEA102343EA1A
:10E450000026B1B201EE901AB8EE612A219A82ED3F
:10E46000132AFEF75FBC1D98072808D943F2CC0396
:10E47000C2F200034FF008061E7203F0C9BEFCF79B
:10E4800049FC02EE900AB8EE623A219D85ED133AFE
:10E49000FEF748BC219FD7ED133A97ED124A63EE81
:10E4A000844AC7ED134AFFF7C5BB219991ED135A72
:10E4B000F1EE455AC1ED135AFEF734BC4FF000009F
:10E4C0004FF001010A46FDF74BFC219A92ED136AC9
:10E4D000F1EE046A66EE267A4FF00000009001909B
:10E4E00043F22020C2F20000BCEEE70A10EE101A40
:10E4F0004FF0FF024BF6C553C0F60203FAF778FA65
:10E50000FEF710BC43F2DC03C2F200031E7816F0E3
:10E51000280F08D01D9901F10301B1F5005F34BF48
:10E520000021012106E01D9901F10301FA2994BFA0
:10E530000021012141B143F2CC04C2F200044FF0AA
:10E540001300207203F064BE41F25C05C2F20005C4
:10E550001D9FE859FBF7ECFD219A9064FEF7E2BBA2
:10E5600043F2DC03C2F200031E7816F0280F08D035
:10E570001D9901F10301B1F5005F34BF00210121B4
:10E5800006E01D9901F10301FA2994BF0021012140
:10E5900041B143F2CC04C2F200044FF013002072E8
:10E5A00003F036BE41F25C05C2F200051D9FE8593A
:10E5B000FBF7BEFD219AD064FEF7B4BB1D9B072B71
:10E5C00008D943F2CC04C2F200044FF008062672C8
:10E5D00003F01EBE219ED6ED130AF5EEC00AF1EE41
:10E5E00010FA0FDB9FED487AF4EEC70AF1EE10FA4D
:10E5F00008D8FCEEE01ACDED1C1A4FF0000586F8A5
:10E60000505021E09FED401AF4EEC10AF1EE10FAED
:10E6100007DD6FF07F431C934FF0010186F8501027
:10E6200012E04FF000011C9110EE900A0AF098FAE7
:10E6300028B14FF00202219880F8502004E04FF0FA
:10E640000305219F87F850501D981C99FCF734FB57
:10E65000FEF768BB219FF86C0AF096FA00287EF45A
:10E6600061AB219890ED132AB5EEC02AF1EE10FAB5
:10E6700004DD4FF07E53C364FEF754BBB5EEC02AF1
:10E68000F1EE10FA7EF54EAB4FF00002CBF6807241
:10E69000C264FEF747BB21998D6ACDB1FAF7DEF966
:10E6A000219FBA6AC2F1040318184CF6CD41CCF68A
:10E6B000CC41A1FB00154FEA95067A6AB6FBF2F34E
:10E6C00002EE903AB8EE623A87ED133AFEF72ABBB3
:10E6D0004FF6FF76C7F67F76CE64FEF723BB43F294
:10E6E000DC00C2F20000017811F0280F10D01D9E4E
:10E6F00006F10306B6F5005F34BF002601260EE0E2
:10E700000000004700008047FFFF7F4B00000034FF
:10E710001D9E06F10306FA2E94BF0026012646B17F
:10E7200043F2CC04C2F200044FF01303237203F04F
:10E730006FBD1D9F219DE86CFBF7D0FC41F25C0290
:10E74000C2F20002D051FEF7EDBA2198D0ED123A94
:10E7500090ED134A73EEC44AC0ED134AFFF76ABA4C
:10E76000219EF76C1C97B56CF564B764FEF7DABAB6
:10E77000219AD06C0AF008FA30B14FF003062199C3
:10E7800081F85060FEF7CEBA219BD86C0AF0ECF904
:10E7900030B14FF00400219B83F85000FEF7C2BA5D
:10E7A0002198C66C30460AF003FF08EE100A304686
:10E7B0004FF000010AF07AFB01464FF07E500AF05C
:10E7C00075FB1FED2E5A05EE900A25EE856AB4EE14
:10E7D000C68AF1EE10FA06D84FF00005219A82F8A9
:10E7E0005050FEF79FBA2199D1ED136AF5EEC06A39
:10E7F000F1EE10FA05DD4FF0010781F85070FEF7D9
:10E8000091BAF5EEC06AF1EE10FA4CBF0222032273
:10E8100081F85020FEF786BA219FD7ED138A97ED35
:10E82000128A38EEC89A19EE100A0AF0C1FE09EEF3
:10E83000100A18EE900A18EE101A0AF037FB01467B
:10E840004FF07E500AF032FB5FED507A00EE100A76
:10E8500060EE270AB4EEE09AF1EE10FA0DF1700CBA
:10E860008CBF00200120FBF7E9FDFEF75BBA219D7C
:10E87000EE6C30460AF09CFE08EE100A30464FF06F
:10E8800000010AF013FB01464FF07E500AF00EFB28
:10E890001FED621A07EE100A67EE011AB4EEE18A64
:10E8A000F1EE10FA0DF1700C8CBF00200120FBF787
:10E8B000C5FDFEF737BA219A92ED132AD2ED122A3E
:10E8C000B4EEE22AF1EE10FA0DF1700CB4BF0020A4
:10E8D0000120FBF7B3FDFEF725BA219890ED133A1E
:10E8E000B5EEC03AF1EE10FA0DF1700CB4BF002095
:10E8F0000120FBF7A3FDFEF715BA219BD3ED133AD8
:10E9000093ED124AF4EEC43AF1EE10FA0DF1700CE8
:10E91000D4BF00200120FBF791FDFEF703BA219937
:10E92000D1ED134A91ED125AF4EEC54AF1EE10FA08
:10E930000DF1700C8CBF00200120FBF77FFDFEF76E
:10E94000F1B9219FD7ED135A97ED126AF4EEC65A2A
:10E95000F1EE10FA0DF1700C54BF00200120FBF70E
:10E960006DFDFEF7DFB9219DD5ED136AF5EEC06AA6
:10E97000F1EE10FA0DF1700C54BF00200120FBF7EE
:10E980005DFDFEF7CFB9219ED6ED138A96ED128A72
:10E9900038EEC89A19EE100A0AF00AFE09EE100ABB
:10E9A00018EE900A18EE101A0AF080FA01464FF09D
:10E9B0007E500AF07BFA5FEDAB7A00EE100A60EE53
:10E9C000270AB4EEE09AF1EE10FA0DF1700CD4BF04
:10E9D00000200120FBF732FDFEF7A4B9219AD76C85
:10E9E00038460AF0E5FD08EE100A38464FF00001FF
:10E9F0000AF05CFA01464FF07E500AF057FA1FED1C
:10EA0000BD1A07EE100A67EE011AB4EEE18AF1EEC4
:10EA100010FA0DF1700CD4BF00200120FBF70EFDA1
:10EA2000FEF780B943F2DC00C2F20000037813F075
:10EA3000280F08D01D9901F10201B1F5005F34BF24
:10EA40000021012106E01D9901F10201FA2994BF7C
:10EA50000021012141B143F2CC04C2F200044FF085
:10EA60001300207203F0D4BBF9F7F8FF219F00F1E7
:10EA700004004CF6CD45CCF6CC45A5FB00164FEA7C
:10EA800096007A6AB0FBF2F31D9D41F25C00C2F27F
:10EA9000000041194E78425D4FEA024545EA0620E2
:10EAA000897840EA01061B969B1B23F07F421C924B
:10EAB00002EE102AF8EE422AC7ED132AFEF732B909
:10EAC000219FFD6CBD64FEF72DB9219991F851602D
:10EAD000002E40F04D82FEF725B9219B93F851207E
:10EAE000002A00F04582FEF71DB943F2DC00C2F2B5
:10EAF0000000017811F0280F06D01D9EB6F5005FCA
:10EB000034BF0026012604E01D9EFA2E94BF002685
:10EB1000012646B143F2CC04C2F200044FF01306C2
:10EB2000267203F075BB41F25C02C2F200021D9B2B
:10EB3000D05C00287EF4F6A81E991C911AE243F2DC
:10EB4000DC02C2F20002137813F0280F06D01D98E1
:10EB5000B0F5005F34BF0020012004E01D98FA28C2
:10EB600094BF0020012040B143F2CC04C2F2000463
:10EB70004FF01300207203F04BBB41F25C01C2F274
:10EB800000011D9E8A5D002A3EF4CCA81E9B1C93AA
:10EB9000F0E11D990F2908D943F2CC03C2F200031A
:10EBA0004FF027021A7203F033BBC8B2FCF7E4FB44
:10EBB00000283EF4B7A81E9E1C96DBE11D98F9289C
:10EBC00008D943F2CC04C2F200044FF012002072C4
:10EBD00003F01EBB43F2E001C2F200010E5C1E9B7B
:10EBE0001E427EF49FA81F9A1C92C3E11D99F92929
:10EBF00008D943F2CC04C2F200044FF01201217292
:10EC000003F006BB43F2E006C2F20006725C1E9BF4
:10EC10001A423EF487A81F981C90ABE143F2DC0631
:10EC2000C2F20006327812F0280F06D01D9BB3F511
:10EC3000005F34BF0023012304E01D9BFA2B94BF27
:10EC40000023012343B143F2CC04C2F200044FF08D
:10EC50001303237203F0DCBA41F25C00C2F200003D
:10EC60001D99465C002E7EF45DA81E9A1C92B2E1AE
:10EC700043F2DC00C2F20000017811F0280F06D048
:10EC80001D9EB6F5005F34BF0026012604E01D9EE0
:10EC9000FA2E94BF0026012646B143F2CC04C2F2FC
:10ECA00000044FF01306267203F0B2BA41F25C0280
:10ECB000C2F200021D9BD05C00283EF433A81E99CE
:10ECC0001C9188E143F2DC02C2F20002137813F0D7
:10ECD000280F06D01D98B0F5005F34BF002001203A
:10ECE00004E01D98FA2894BF0020012040B143F2AF
:10ECF000CC04C2F200044FF01301217203F088BA71
:10ED000041F25C01C2F200011D9E8A5D1E9B9A4287
:10ED10007EF608A81F981C902CE143F2DC06C2F294
:10ED20000006327812F0280F06D01D9BB3F5005F65
:10ED300034BF0023012304E01D9BFA2B94BF002362
:10ED4000012343B143F2CC04C2F200044FF013009C
:10ED5000207203F05DBA41F25C00C2F200001D991E
:10ED6000465C1E9A9642FDF4DDAF1F9B1C9301E1A9
:10ED700043F2DC01C2F200010E7816F0280F06D033
:10ED80001D9AB2F5005F34BF0022012204E01D9AF3
:10ED9000FA2A94BF0022012242B143F2CC04C2F20B
:10EDA00000044FF01300207203F032BA41F25C000D
:10EDB000C2F200001D9BC15C1E9EB1427DF4B2AF49
:10EDC0001F9A1C92D6E043F2DC03C2F200031978CA
:10EDD00011F0280F06D01D9EB6F5005F34BF002647
:10EDE000012604E01D9EFA2E94BF0026012646B19E
:10EDF00043F2CC04C2F200044FF01302227203F07B
:10EE000007BA41F25C02C2F200021D98115C1E9B1F
:10EE100099423DF487AF1F9E1C96ABE043F2DC00A5
:10EE2000C2F20000017811F0280F06D01D9BB3F547
:10EE3000005F34BF0023012304E01D9BFA2B94BF25
:10EE40000023012343B143F2CC04C2F200044FF08B
:10EE50001306267203F0DCB941F25C06C2F200062A
:10EE60001D9AB05C1E9988423DF65CAF1F9B1C93B7
:10EE700080E043F2DC02C2F20002107810F0280FAA
:10EE800006D01D99B1F5005F34BF0021012104E0D7
:10EE90001D99FA2994BF0021012141B143F2CC040C
:10EEA000C2F200044FF01306267203F0B1B941F22A
:10EEB0005C06C2F200061D9BF25C1E988242BDF405
:10EEC00031AF1F991C9155E0219B93F847201D9865
:10EED00082427DF427AF1E991C917CE0219E96F81A
:10EEE00047201D9B9A423DF41DAF1E981C9072E076
:10EEF000219991F847601D9A96427DF613AF1E9BAB
:10EF00001C9368E0219890F847101D9EB142FDF4D3
:10EF100009AF1E9A1C925EE0219B93F847001D9951
:10EF20008842BDF4FFAE1E9E1C9654E0219A92F8D2
:10EF300047001D9B98423DF6F5AE1E991C914AE094
:10EF40009DF874000DF16B01FCF726FE8DF86A0048
:10EF50009DF86B6036B143F2CC04C2F20004267215
:10EF600003F056B900283DF4DDAE1E9A1C9201E074
:10EF70001D981C901C9E40F20000C0F6010090F805
:10EF80002E1090F82F3043EA0122B24208D243F209
:10EF9000CC04C2F200044FF00906267203F038B91F
:10EFA00043F2E017C2F200073E60FDF7BBBE0DF171
:10EFB000700CFBF75BFA1C900028D9D0FDF7B2BEAD
:10EFC0000DF1700CFBF752FA1C900028D0D1FDF720
:10EFD000A9BE1D9B1C93219A136A052B08D943F2E5
:10EFE000CC04C2F200044FF00A03237203F010B9FC
:10EFF00003F1020043F2E011C2F200010E6842F890
:10F00000206003F10103219A1362B3E70DF1700C44
:10F01000FBF72CFA1C900028DBD0FDF783BE0DF126
:10F02000700CFBF723FA1C900028D2D1FDF77ABEB2
:10F030000DF1700CFBF71AFA1C901D9988427DF4B3
:10F0400071AE1E9E1C9695E70DF1700CFBF70EFA43
:10F050001C901D9A90423DF465AE1E981C9089E765
:10F060000DF1700CFBF702FA1C901D9B98427DF687
:10F0700059AE1E991C917DE70DF1700CFBF7F6F966
:10F080001C901D9EB042FDF44DAE1E9A1C9271E77D
:10F090000DF1700CFBF7EAF91C901D9B9842BDF432
:10F0A00041AE1E981C9065E70DF1700CFBF7DEF980
:10F0B0001C901D9988423DF635AE1E9E1C9659E760
:10F0C0009DF874000DF16B01FCF734FD8DF86A00BA
:10F0D0009DF86B3033B143F2CC04C2F200042372CA
:10F0E00003F096B800283DF41DAE1E9A1C9241E72D
:10F0F0009DF874000DF16B01FCF71CFD8DF86A00A2
:10F100009DF86B1031B143F2CC06C2F200063172A9
:10F1100003F07EB800287DF405AE1E981C9029E708
:10F120000DF1700CFBF7CAF941F25C02C2F2000269
:10F130001E9BD15C1D9801423DF4F4AD1F9E1C96B0
:10F1400018E70DF1700CFBF7B9F941F25C02C2F25D
:10F1500000021E9BD15C1D9801427DF4E3AD1F9E11
:10F160001C9607E70DF1700CFBF7A8F941F25C0261
:10F17000C2F200021E9BD15C1D9801427DF4D2AD0B
:10F180001F9E1C9627E70DF1700CFBF797F941F2D3
:10F190005C02C2F200021E9BD15C1D9801423DF44C
:10F1A000C1AD1F9E1C9616E798F8005045F0080068
:10F1B00088F80000FDF717BE0DF1700CFBF756F94B
:10F1C0008DF86A00219991F851601D9AB3181C932B
:10F1D00043F2DC01C2F200010E7816F0280F09D0CC
:10F1E0001E9E06F1FF32D318B3F5005F34BF002333
:10F1F000012307E01E9A02F1FF31CB18FA2B94BFCE
:10F200000023012343B143F2CC04C2F200044FF0C7
:10F210001303237202F0FCBF4FF000071B971E9DE3
:10F22000D5B11C9E41F25C01C2F200018B5D8342AC
:10F2300033D005F1FF3241F25C07C2F20007BB197F
:10F2400041F25C05C2F20005C5F101018F1B12F00D
:10F25000010F1AD003F065B84FF0FF001B901CE0BF
:10F2600013F8019F02F1FF38484504D11C95CDF8F1
:10F270006CE01E9211E04246CD1807EB030E13F826
:10F28000016FB04243F05A80F0E7CD1807EB030E50
:10F29000002AE5D11C951E92DEE70DF1700C9DF859
:10F2A0006C00FBF7CBF8FDF73DBD0DF1700CFBF7E3
:10F2B000DDF843F2E41BC2F2000B8BF800004FF0C4
:10F2C00001011C91CDF830B0BBE0219E96F8512091
:10F2D0001D9813181C9343F2DC01C2F200010E7852
:10F2E00016F0280F07D003F10103B3F5005F34BF18
:10F2F0000023012305E003F10103FA2B94BF00234F
:10F30000012343B143F2CC04C2F200044FF01302D4
:10F31000227202F07DBF1E981B900DF1700C26AF7B
:10F3200047F0010122AD45F001024FF00003FBF769
:10F33000D7F8FDF7F7BC219890F851101D9BCE1817
:10F340001C9643F2DC02C2F20002107810F0280F83
:10F3500005D0B6F5005F34BF0026012603E0FA2E83
:10F3600094BF0026012646B143F2CC04C2F2000449
:10F370004FF01301217202F04BBF1F9F1E98B8423D
:10F3800028BF38461B900DF1700C26AD45F00101E9
:10F3900022AB43F001024FF00003FCF799F9FDF7AF
:10F3A000C1BC0DF1700CFBF761F8034643F2E41B9E
:10F3B000C2F2000B58464FF010014EF27432C0F604
:10F3C00003020AF0D7FA1C90CDF830B039E01E9E47
:10F3D0001C961F9A1B924FF000000C9031E04FF0EA
:10F3E000FF331C930C932CE02199C86C9DF8781086
:10F3F0009DF87C2043F2E416C2F2000600964FF01E
:10F40000100301934FF00103FDF720F84FF0FF3296
:10F410001C920C9615E02198C06C9DF878109DF810
:10F420007C2043F2E416C2F2000600964FF010036F
:10F4300001934FF00003FDF709F84FF0FF311C91E5
:10F440000C961D99A1F1FB0086B20B96A1F1FB036E
:10F45000032B23D840F2A060C1F200004FF41176D4
:10F460000B9906FB010393F82022032A08D043F2EC
:10F47000CC06C2F200064FF04803337202F0C8BE59
:10F4800040F2A067C1F200074FF411700B9E00FB21
:10F49000067707F104074FF0000605E0219F97F873
:10F4A000512056184FF00007DDF870B0BBF1FF3F58
:10F4B00011D14FF0FF0B4FF00009C84643F2DC01B9
:10F4C000C2F200010D9141F25C03C2F200030E93FF
:10F4D0000F950C9D05E0BBF1000FECD14FF000093A
:10F4E0006FE01D9AA2F1FB02032A10D8D7F8006141
:10F4F000FF2E14BF01364646D7F80401864206D1D6
:10F500004046FCF745F9D7F804118E42F8D0B5F122
:10F51000FF3F15D1219850F8341F0B68D3F800C075
:10F52000494610AA4FF00103E0478DF86B0080B107
:10F530000F9D43F2CC04C2F20004207202F068BEB8
:10F5400025B115F809208DF8402002E01B9B8DF8AD
:10F5500040301C98B0F1FF3F02D19DF8402082B3AB
:10F560001D99A1F1FB01032907D8D7F800319DF8B7
:10F570004000F854C7F800611FE00D9B187810F0A8
:10F58000280F05D0B6F5005F34BF0020012003E04E
:10F59000FA2E94BF0020012048B10F9D43F2CC0405
:10F5A000C2F200044FF01306267202F031BE9DF83D
:10F5B00040200E998A5506F1010609F10109D94545
:10F5C0008FD31D9FA7F1FB07032F05D80B99C8B256
:10F5D000FBF7DCF9FDF7A6BB219D95F8512009EB5F
:10F5E000020E85F851E0FDF79DBB1D9AA2F1FB00CC
:10F5F000032858D887B240F2A060C1F200004FF44F
:10F60000117101FB070292F82032032B08D043F25C
:10F61000CC04C2F200044FF04803237202F0F8BD9C
:10F6200040F2A066C1F200064FF4117505FB0765B4
:10F6300005F104051E9800F1FF311E9170B34FF0E3
:10F64000000843F2E019C2F2000940F200029346BA
:10F65000C0F6010BD5F80061FF2E14BF01364646F7
:10F66000D5F804319E4206D14046FCF791F8D5F812
:10F6700004018642F8D0D9F80030D5F800211BF8F3
:10F680000310A95403F10103C9F80030C5F8006163
:10F690001E9E06F1FF301E90002EDBD1F8B2FBF764
:10F6A00075F9FDF73FBB1E9B1C93219991F8510002
:10F6B00082181B9243F2DC06C2F20006367816F07E
:10F6C000280F08D003F1FF36B218B2F5005F34BF3F
:10F6D0000022012206E003F1FF36B218FA2A94BF95
:10F6E0000022012242B143F2CC04C2F200044FF0E6
:10F6F0001306267202F08CBDC71881F851701C9A4F
:10F7000002F1FF351C95002A3DF40CAB43F2E013E7
:10F71000C2F200031E681B9F41F25C01C2F20001AD
:10F72000C91940F20000C0F6010030184FF0000384
:10F7300005F0010910F803C001F803C003F101034B
:10F74000934242F0DF850DE010F803E001F803E09A
:10F7500003F1010310F8039001F8039003F1010392
:10F760009342F1D1E819A91901F1010143F2E01224
:10F77000C2F2000211604FF0FF331C9300F1010050
:10F780001B90FDF7CFBA4FF000028DF86A20219E42
:10F7900096F851001D9BC1181C911E9A1B9243F2B2
:10F7A000DC00C2F20000037813F0280F08D002F149
:10F7B000FF335818B0F5005F34BF0020012006E089
:10F7C00002F1FF325018FA2894BF0020012040B106
:10F7D00043F2CC04C2F200044FF01302227202F092
:10F7E00017BD41F25C07C2F2000707EB01099DF863
:10F7F0007CB043F2DC15C2F200052A68B66B9119A1
:10F80000905DFF2859D088464FF001070894CDF845
:10F810002CA0BA4698F8014004EB002343F2DC1513
:10F82000C2F200052A68D6184FF000011C919DF81D
:10F830006A00002802F03C85D75C06F1010602F060
:10F8400039BD9DF86A402CB18FB9089C5046DDF84F
:10F850002CA005E0727852B9089C5046DDF82CA027
:10F86000219F97F851609B1987F8513027E016F8CF
:10F87000014F19F803B045B920460AF01FF8C4B289
:10F8800058460AF01BF85FFA80FB5C4508D11C9BC8
:10F8900003F101031C9307F1FF371B999942D0D262
:10F8A000AB460AF1010A18F8020FFF28B2D1089CF2
:10F8B000DDF82CA04FF0000001E04FF000000DF14A
:10F8C000700CC0B2FAF7BAFDFDF72CBA4FF0010187
:10F8D0008DF86A105BE70DF1700CFAF7C7FD03466F
:10F8E00043F2E41BC2F2000B58464FF010014EF2F7
:10F8F0007C32C0F603020AF03DF81C90CDF830B01F
:10F900009FE50DF1700CFAF7B1FD034643F2E41BDD
:10F91000C2F2000B58464FF010014EF28432C0F68E
:10F9200003020AF027F81C90CDF830B089E50DF1FC
:10F93000700CFAF79BFD034643F2E41BC2F2000B86
:10F9400058464FF010014EF28832C0F603020AF01A
:10F9500011F81C90CDF830B073E50DF1700CFAF78A
:10F9600085FD034643F2E41BC2F2000B58464FF0FC
:10F9700010014EF29032C0F6030209F0FBFF1C901A
:10F98000CDF830B05DE5219890F8517007F101078E
:10F9900080F85170FDF7C6B91D9D41F25C02C2F2BC
:10F9A0000002515D01F101015155FDF7BBB9219EE6
:10F9B00096F8473003F1010386F84730FDF7B2B9F6
:10F9C0009DF874000DF16B01FCF7B4F80DF1700CAB
:10F9D000FAF734FD9DF86B0000283DF4A3A943F22B
:10F9E000CC04C2F20004207202F012BC9DF8740034
:10F9F0000DF16B01FCF70AF90DF1700CFAF71EFD21
:10FA00009DF86B1000293DF48DA943F2CC02C2F29F
:10FA10000002117202F0FCBB1D9E1C964FF0000309
:10FA20001B934FF001008DF86A009DF870000DF1F6
:10FA30006B01FCF77FF89DF86B1099B920B19DF828
:10FA40006A201B9E16431B969DF86A304FEA4300BE
:10FA50008DF86A001C9901F101011C9110F0FE0F54
:10FA6000E3D10AE09DF86A20012A06D143F2CC04D2
:10FA7000C2F20004217202F0CBBB0DF1700C9DF8B4
:10FA80006C00FAF7DBFCFDF74DB91D9E1C964FF09C
:10FA900000031B934FF001008DF86A009DF8700081
:10FAA0000DF16B01FCF7B2F89DF86B1099B920B11C
:10FAB0009DF86A201B9E16431B969DF86A304FEAFC
:10FAC00043008DF86A001C9901F101011C9110F0AE
:10FAD000FE0FE3D10AE09DF86A20012A06D143F225
:10FAE000CC04C2F20004217202F092BB0DF1700C42
:10FAF0009DF86C00FAF7A2FCFDF714B99DF87400AC
:10FB00000DF16B01FCF748F88DF86A009DF86B6009
:10FB100036B143F2CC03C2F200031E7202F078BB8E
:10FB20000DF1700CFAF78AFCFDF7FCB81D981C90DB
:10FB30004FF000011B914FF001008DF86A00219AEF
:10FB400092F8476030420ED09DF870000DF16B01C5
:10FB5000FCF722F89DF86B309BB920B19DF86A0044
:10FB60001B9901431B919DF86A204FEA42068DF8CC
:10FB70006A601C9B03F101031C9316F0FE00DED1AA
:10FB80000AE09DF86A10012906D143F2CC04C2F2C2
:10FB90000004237202F03CBB1B9F219D85F8477037
:10FBA000FDF7C0B89DF874000DF16B01FCF760F82B
:10FBB0000DF1700CFAF742FC9DF86B60002E3DF4DD
:10FBC000B1A843F2CC02C2F20002167202F020BBCE
:10FBD0001D9B1C93D8B20DF16B01FCF749F81B90EB
:10FBE0009DF86B0030B143F2CC04C2F200042072E5
:10FBF00002F00EBB4FF001018DF86A101C9F7A18BD
:10FC00001C92D0B20DF16B01FCF732F89DF86A50EE
:10FC100000FA05F01B9E06431B9605F101058DF8C1
:10FC20006A501C9A02F101021C92EBB2072BE8D930
:10FC30000DF1700C9DF86C00FAF700FCFDF772B83E
:10FC40000DF1700C219890F85100FAF7F7FBFDF7D1
:10FC500069B8FDF767B843F2B401C2F200014FF092
:10FC600001070F70FDF75EB843F2B405C2F200055C
:10FC70004FF000062E70FDF755B821984FF00001A7
:10FC80004FF054020AF0ACFA4FF00002219243F216
:10FC90009003C2F200031C6804F1FF30186002F008
:10FCA00014BA43F29002C2F2000213687F2B08D903
:10FCB00043F2CC04C2F200044FF03000207202F094
:10FCC000A7BA4FF001071C9740F2A065C1F20005EA
:10FCD000D5F8E809002842F0F88205E0D6F8AC2013
:10FCE000002A4ED11C9301E04FF001031D9840F211
:10FCF000A066C1F200064FF0540505FB03F3F218AD
:10FD0000C2F89009C2F894091E9982F8E2194FF0DE
:10FD10000A07C2F8B47906F51967F81800F134003B
:10FD2000219901F134014FF010020AF035FA1C9BC1
:10FD300005FB037000F14400219901F144014FF0EB
:10FD400004020AF029FA1C9805FB007000F1480033
:10FD5000219901F148014FF008020AF01DFA219A99
:10FD600092F851101C9F05FB076686F8E11943F2D3
:10FD70009005C2F200052B6803F101032B60FCF72C
:10FD8000D1BF03F101073B4606F15406D6F8AC504B
:10FD9000002D42F0AE82A5E71C93FCF7C3BF21996A
:10FDA00091F852601E967CE70DF1700CFAF75EFB3D
:10FDB0001E9076E71D9A219981F85120FCF7B2BF79
:10FDC0000DF1700C9DF87400FAF738FBFCF7AABF30
:10FDD000219EB36A002B3CF4A5AFF8F73FFE2199B2
:10FDE0008A6A801A4E6A1D9B06FB03F303EB8301AC
:10FDF0008842BCF497AF1E9A1C92FFF7BBB8F8F785
:10FE00002DFE219FB862FCF78DBF43F2E000C2F2E5
:10FE1000000090F8FB201E9E9319FB2B08D943F29B
:10FE2000CC00C2F200004FF01203037202F0F0B9EE
:10FE300043F2DC01C2F20001087810F0280F09D06B
:10FE40001D9BD11801F1FF30B0F5005FB4BF002059
:10FE5000012007E01D9BD11801F1FF30FA28D4BF23
:10FE60000020012040B143F2CC04C2F200044FF064
:10FE70001302227202F0CCB943F2E005C2F200058F
:10FE8000A81941F25C07C2F200071D9EB9190AF0D9
:10FE900083F9FCF747BF98F8001041F0100588F887
:10FEA0000050FCF7A0BF219F97F84760002E0CBFC1
:10FEB000FF22002287F84720FCF734BF219890F8F2
:10FEC00047306FEA030180F84710FCF72BBF0DF1B4
:10FED000700CFAF7F3FA1E9D41F25C07C2F20007BC
:10FEE0007E5D1D9A72407A55FCF71CBF2198816B8C
:10FEF0001D9B5E181C96BDE12198C26B816B531847
:10FF00001C93B7E1219E306C40B943F2CC04C2F29D
:10FF100000044FF02002227202F07AB900F1FF359E
:10FF20003564FCF7FFBE21990B6C03F101030B64F0
:10FF3000002B7CF4F7AE43F2CC06C2F200064FF081
:10FF40002000307202F064B9219A516B0B685E6830
:10FF500046B943F2CC00C2F200004FF01E03037218
:10FF600002F056B90DF1700CFAF780FA1C90219846
:10FF700050F8342F11684E681D991CAA4FF00103E8
:10FF8000B0478DF86B0000283CF4CCAE43F2CC04B3
:10FF9000C2F20004207202F03BB90DF1700CFAF7C6
:10FFA00065FA1C9054E10DF1700CFAF75FFA219F8D
:10FFB000F863FCF7B7BE0DF1700CFAF757FA219D04
:10FFC0002864FCF7AFBE219850F8342F11680E68F2
:10FFD0001D991CAA4FF00103B0478DF86B0030B19A
:10FFE00043F2CC04C2F20004207202F011B90DF108
:10FFF000A80C1CF8380DFAF721FAFCF793BE2198EB
:020000040803EF
:10000000436B0DF1700C187AFAF718FAFCF78ABEF8
:100010000DF1700C219F97F83C00FAF70FFAFCF7EE
:1000200081BE219A116CFF2908D943F2CC06C2F295
:1000300000064FF02004347202F0EAB80DF1700CA3
:10004000C8B2FAF7FBF9FCF76DBE219850F8345F9F
:100050002B689F68B84703EE100AF8EE433A2198E0
:10006000C0ED133AFCF75EBE219A92ED0E4AF8EE0F
:10007000444AC2ED134AFCF755BE219991ED105A3E
:10008000F8EE455AC1ED135AFCF74CBE219E96ED91
:10009000136AFCEEC66ACDED1C6AEBE0219BD3ED42
:1000A000137A9FEDB40AF4EEC07AF1EE10FA08DB91
:1000B00043F2CC04C2F200044FF02000207202F0A0
:1000C000A7B8FCEEE70AC3ED100AFCF72BBE219897
:1000D00050F8342F11680E681D991CAA4FF00403C4
:1000E000B0478DF86B0030B143F2CC03C2F200038D
:1000F000187202F08DB81C98FAF71AF8219DA864BE
:10010000FCF710BE219850F8342F11680E681D9925
:100110001CAA4FF00403B0478DF86B0030B143F2D6
:10012000CC04C2F20004207202F072B81C98F9F7F5
:10013000FFFF219FF864FCF7F5BD2198436B1A6817
:10014000516841B943F2CC00C2F200004FF01E02E8
:10015000027202F05DB8C06CF9F7C0FF1C902198E4
:1001600050F8346F33685E681D991CAA4FF0040381
:10017000B0478DF86B0000283CF4D4AD43F2CC04BA
:10018000C2F20004207202F043B843F2DC01C2F272
:1001900000010B7813F0280F0BD0219EF06B1D9AF5
:1001A000111801F1FF33B3F5005F34BF00230123C1
:1001B00009E0219EF06B1D9A111801F1FF33FA2B13
:1001C00094BF0023012343B143F2CC00C2F20000EC
:1001D0004FF01301017202F01BB8219B184650F832
:1001E000347F3E6836684FF0000141F25C07C2F28E
:1001F00000071D9ABA18DB6BB0478DF86B0000281A
:100200003CF490AD43F2CC04C2F20004207201F041
:10021000FFBF219850F8343F1E6836681D991BAA0D
:100220004FF00403B0478DF86B0030B143F2CC04BB
:10023000C2F20004207201F0EBBF1B9882B2C0F33F
:10024000072141EA02239EB21C9613E01D981C90E0
:100250001C982199FAF7A8F98DF86B0000283CF456
:1002600061AD43F2CC02C2F20002107201F0D0BFC5
:100270001D991C911C9BB3F5803F08D343F2CC041D
:10028000C2F200044FF01F00207201F0C1BF219D97
:10029000AB63FCF747BD1D9D219FFD63FCF742BD8D
:1002A0001D9E219B1E64FCF73DBD2198826B1D990C
:1002B000561A1C96DEE71E9A219BD96B8E18FB2ED0
:1002C00008D943F2CC00C2F200004FF012020272D1
:1002D00001F09EBF43F2E007C2F2000787F8FB106F
:1002E000184650F8341F0E6836681D99BA18DB6B33
:1002F000B0478DF86B0000283CF414AD43F2CC04F9
:10030000C2F20004207201F083BF219B596B0E687A
:10031000766846B943F2CC01C2F200014FF01E00EC
:10032000087201F075BF43F2DC00C2F200000278EF
:1003300012F0280F0AD0DA6B1D99881800F1FF30EF
:10034000B0F5005F34BF0020012008E0D86B1D9994
:100350000A1802F1FF30FA2894BF0020012058B19A
:1003600043F2CC03C2F200034FF013061E7201F0F9
:100370004FBF00BF0000804703F134004FF0000181
:1003800041F25C07C2F200071D9ABA18DB6BB04756
:100390008DF86B0000283CF4C5AC43F2CC04C2F2EB
:1003A0000004207201F034BFF6F770FA00287CF4E4
:1003B000B9AC1D9A1C92FEF7DDBDF6F767FA00286E
:1003C0003CF4B0AC1D9B1C93FEF7D4BD1D9E0C2EBF
:1003D00008D943F2CC04C2F200044FF005012172A7
:1003E00001F016BFF0B24FF00001F6F70DFA01EE82
:1003F000100AB8EE417A219F87ED137AFCF792BC80
:100400001D980C2808D943F2CC03C2F200034FF028
:1004100005021A7201F0FCBEC0B24FF00101F6F7FE
:10042000F3F901EE900AB8EE612A219D85ED132AB9
:10043000FCF778BC1D9E0C2E08D943F2CC04C2F206
:1004400000044FF00501217201F0E2BEF0B24FF05E
:100450000001F6F749F9FCF765BC1D980C2808D98E
:1004600043F2CC03C2F200034FF005021A7201F00E
:10047000CFBEC0B24FF00101F6F736F9FCF752BC1F
:100480001D9E0C2E08D943F2CC04C2F200044FF09A
:100490000501217201F0BCBEF0B24FF00001F6F789
:1004A00073F9FCF73FBC1D980C2808D943F2CC0324
:1004B000C2F200034FF005021A7201F0A9BEC0B2E9
:1004C0004FF00101F6F760F9FCF72CBC9DF87400C1
:1004D000F1F774FB00287CF425AC43F2CC06C2F2A1
:1004E00000064FF02804347201F092BE9DF87400AB
:1004F000219901F14C01F1F781FB00287CF412AC49
:1005000043F2CC01C2F200014FF02800087201F062
:100510007FBE219BD3ED132A9DF87400BCEEE23A16
:1005200013EE101AF1F79CFB00287CF4FBAB43F2AE
:10053000CC06C2F200064FF02802327201F068BE0B
:10054000FCF7F0BB0DF1700CF9F790FF30B9219F6B
:1005500097F84750291C18BF012101E04FF0010115
:10056000219880F84710FCF7DDBB9DF874600DF111
:10057000700CF9F77BFF014630464FF00102FBF7A4
:10058000EFFB8DF86B0000283CF4CCAB43F2CC04BD
:10059000C2F20004207201F03BBE0DF1700CF9F7BD
:1005A00065FF01468DF86A009DF87400FBF796FB25
:1005B0008DF86B0000283CF4B5AB43F2CC03C2F2DB
:1005C0000003187201F024BE1D9A1C924FF0010323
:1005D0008DF86A301E46219890F847100B420AD0D9
:1005E00090F846109DF8700019403246FBF7B8FBB2
:1005F0008DF86B0068B99DF86A304FEA43008DF8BA
:100600006A001C9A02F101021C9210F0FE03E2D172
:100610000AE09DF86A60012E06D143F2CC04C2F2D2
:100620000004207201F0F4BD4FF000078DF86B70EC
:100630000DF1700CF9F71AFF0DF1700CF9F716FFB8
:10064000FCF770BB9DF874004FF001010A46FBF700
:1006500087FB8DF86B0000283CF464AB43F2CC01BF
:10066000C2F20001087201F0D3BD9DF874004FF092
:1006700000014FF00102FBF773FB8DF86B000028BF
:100680003CF450AB43F2CC02C2F20002107201F013
:10069000BFBD0DF1700CF9F7E9FE219D95F84730CB
:1006A000184385F84700FCF73DBB1D980DF1A80CD9
:1006B0004CF8380DFAF788FB00287CF433AB43F292
:1006C000E016C2F200060898306001F015BD10A8CF
:1006D000FAF70CFA014640B19DF84070022F04D0A1
:1006E000C2484FF00D0209F057FD0DF1700C9DF856
:1006F0004000F9F7A3FEFCF715BBFAF769FFFCF71A
:1007000011BB0DF1700CF9F7B1FEFCF70BBB1D9E90
:10071000FA2E08D943F2CC04C2F200044FF01202C0
:10072000227201F075BD0DF1700CF9F79FFE43F2D6
:10073000E001C2F200018855FCF7F4BA0DF1700C2B
:10074000F9F794FE43F2E005C2F2000585F8FB00DC
:10075000FCF7E8BA0DF1700C219B93F84700F9F70C
:100760006DFEFCF7DFBA1D98FA2808D943F2CC06D3
:10077000C2F200064FF01201317201F049BD0DF1D5
:10078000700C43F2E007C2F20007385CF9F756FE3E
:10079000FCF7C8BA0DF1700C43F2E002C2F200029D
:1007A00092F8FB00F9F74AFEFCF7BCBA1D9EF62E44
:1007B00008D943F2CC04C2F200044FF012002072B8
:1007C00001F026BD219DA86CF9F788FC43F2E003F7
:1007D000C2F200039851FCF7A5BA43F2DC01C2F261
:1007E00000010A7812F0280F06D01D9EB6F5005FB2
:1007F00034BF0026012604E01D9EFA2E94BF002679
:10080000012646B143F2CC03C2F200034FF01304B9
:100810001C7201F0FDBC0DF1700C41F25C07C2F2DC
:1008200000071D9D785DF9F709FEFCF77BBA0DF115
:10083000700CF9F743FE41F25C00C2F200001E9911
:10084000425C1D9E32420DF1700C0CBF0020FF2057
:10085000F9F7F4FDFCF766BA43F2DC03C2F20003D9
:10086000187810F0280F08D01D9901F10101B1F599
:10087000005F34BF0021012106E01D9901F1010153
:10088000FA2994BF0021012141B143F2CC00C2F208
:1008900000004FF01301017201F0BABC1D9A41F241
:1008A0005C06C2F20006B05CB318597841EA002237
:1008B0001C92002A3CF436AAFEF75CBB43F2DC0330
:1008C000C2F200031A7812F0280F06D01D9EB6F56A
:1008D000005F34BF0026012604E01D9EFA2E94BF5F
:1008E0000026012646B143F2CC04C2F200044FF0C8
:1008F0001302227201F08CBC41F25C00C2F20000D3
:100900001D99435C002B56D1FCF70CBA43F2DC0670
:10091000C2F20006307810F0280F06D01D99B1F50C
:10092000005F34BF0021012104E01D99FA2994BF22
:100930000021012141B143F2CC04C2F200044FF086
:100940001300207201F064BC41F25C02C2F20002AA
:100950001D9BD65C7EB3FCF7E5B90DF1700CF9F781
:1009600085FD1C9038BBFCF7DDB90DF1700CF9F773
:10097000A5FD41F25C01C2F200011E9A8E5C1D9B36
:100980001E4218D0FCF7CEB90DF1700CF9F796FDA8
:1009900041F25C00C2F200001E99425C1D9E324290
:1009A00009D1FCF7BFB90DF1700CF9F75FFD1C9090
:1009B00000287CF4B7A9219B1E6A46B943F2CC04F7
:1009C000C2F200044FF00300207201F021BC06F1D6
:1009D000FF351D6206F1010653F8267043F2E0115F
:1009E000C2F200010F60FCF79DB900BF6210002049
:1009F00098F8005045F0200388F80030FCF7F3B970
:100A0000219F97F847004FEAD01141EA400287F84A
:100A10004720FCF787B9219E96F847504FEA5503C7
:100A200043EAC51786F84770FCF77CB9FAF730F946
:100A3000FCF778B943F26000C2F20000C2784FF0D0
:100A4000010101FA02F1067926EA01060671FCF7B6
:100A500069B943F2E005C2F2000543F26007C2F251
:100A600000073B7878780090BA78019228464FF0DA
:100A7000FB014EF29432C0F6030208F07BFF85F8CA
:100A8000FB00FCF74FB943F26003C2F20003D978D0
:100A900041B943F26007C2F200074FF00600F87058
:100AA000FCF740B901F1FF3643F26005C2F20005E0
:100AB000EE70FCF737B943F26002C2F2000213781D
:100AC00003F1FF31CEB216701579FF2D0BD1632ED5
:100AD0007CF628A943F26003C2F200034FF06302E0
:100AE0001A70FCF71FB9172E7CF61CA943F2600799
:100AF000C2F200074FF017003870FCF713B943F249
:100B00006001C2F200014E7806F1FF35EFB24F707E
:100B10000879FF280BD1002F7CF404A943F260016F
:100B2000C2F200014FF00C064E70FCF7FBB83B2FF1
:100B30007CF6F8A843F26003C2F200034FF03B02D8
:100B40005A70FCF7EFB843F26005C2F20005AF78C7
:100B500007F1FF30C2B2AA702B79FF2B17D143F2F5
:100B60006005C2F200052F78687807F5FA61F7F79B
:100B700073F88DF86A00AA7812B19042BCF4D2A83A
:100B800043F26003C2F200039870FCF7CBB83B2A33
:100B90007CF6C8A843F26001C2F200014FF03B06A8
:100BA0008E70FCF7BFB843F2E000C2F200004FF0D5
:100BB000000180F8FB1043F26006C2F20006F578EF
:100BC000457037790770FCF7ADB843F2E006C2F222
:100BD000000643F26002C2F20002137850780090DF
:100BE0009178019130464FF0FB014EF2A432C0F6ED
:100BF000030208F0BFFE86F8FB00FCF793B843F24F
:100C0000E005C2F2000543F26007C2F200073B783C
:100C10007E78009628464FF0FB014EF2B432C0F6C3
:100C2000030208F0A7FE85F8FB00FCF77BB843F24F
:100C30006003C2F20003D878052808D943F26001A6
:100C4000C2F200014FF00005CD70FCF76BB800F167
:100C5000010043F26002C2F20002D070FCF762B8F9
:100C600043F26007C2F200073E7806F10106F3B2D4
:100C70003B703879FF280BD1632B7CF653A843F2E5
:100C80006005C2F200054FF000072F70FCF74AB86C
:100C9000172B7CF647A843F26001C2F200014FF027
:100CA00000020A70FCF73EB843F26006C2F200068A
:100CB000737803F10103D8B270703179FF290BD139
:100CC0000C287CF62FA843F26007C2F200074FF011
:100CD00001067E70FCF726B83B287CF623A843F279
:100CE0006005C2F200054FF000026A70FCF71AB806
:100CF00043F26003C2F20003987800F10100C5B22C
:100D00009D701979FF291DD15DB143F26002C2F2D5
:100D100000021778507807F5FA61F6F79DFF8542D3
:100D200008D943F26007C2F200074FF00106BE7017
:100D3000FBF7F8BF43F26006C2F200063379FF2BDF
:100D40003BF4F0AF43F26000C2F2000085783B2D27
:100D50007BF6E8AF43F26001C2F200014FF00002FF
:100D60008A70FBF7DFBF43F26003C2F20003D8785A
:100D70004FF0010505FA00F5197985EA01021A71AB
:100D8000FBF7D0BF0DF1700CF9F770FB43F2600771
:100D9000C2F200073871FBF7C5BF0DF1700CF9F70F
:100DA00065FB062843F26006C2F2000692BFF070AF
:100DB0000023F370FBF7B6BF0DF1700CF9F756FB8B
:100DC00043F26005C2F200052870FBF7ABBF0DF1DE
:100DD000700CF9F74BFB43F26001C2F2000148705E
:100DE000FBF7A0BF0DF1700CF9F740FB43F2600276
:100DF000C2F200029070FBF795BF0DF1700C43F248
:100E00006000C2F200000079F9F718FBFBF78ABF17
:100E10000DF1700C43F26007C2F20007F878F9F7A1
:100E20000DFBFBF77FBF0DF1700C43F26006C2F2C1
:100E300000063078F9F702FBFBF774BF0DF1700C78
:100E400043F26003C2F200035878F9F7F7FAFBF7B0
:100E500069BF0DF1700C43F26005C2F20005A8787D
:100E6000F9F7ECFAFBF75EBF11A8F0F7F7FF43F2D2
:100E70006003C2F20003169D48F21F50C5F2EB104A
:100E800080FB05024FEAE577C7EB62164FF064017D
:100E900001FB16551D70159800F101005870149A49
:100EA0009A70179B1BB103F1FF36F7B201E04FF0C8
:100EB000060743F26001C2F20001CF704FF0FF0558
:100EC0000D71FBF72FBF1D9A0F2A08D943F2CC04EE
:100ED000C2F200044FF02700207201F099B9C64811
:100EE00000EB820143F26007C2F2000710F82260B3
:100EF0003E704B787B704FF00005BD70FD708A78B6
:100F00003A71FBF70FBF43F26000C2F20000FAF73C
:100F100017FAFBF707BF43F26007C2F20007FE783B
:100F20004FF0010101FA06F13B7941EA03053D71F9
:100F3000FBF7F8BE11A8F0F791FF43F26000C2F290
:100F40000000027802F164021692477807F1FF363A
:100F500015968178149111A8F0F7E6FF84E71D98A3
:100F60000F2808D943F2CC04C2F200044FF0270244
:100F7000227201F04DB9C0B2FAF7FEF90DF1700C12
:100F8000F9F75CFAFBF7CEBE4FF000031393129310
:100F90001193199343F26007C2F200073E7806F1FD
:100FA00064061696797801F1FF351595B878149096
:100FB00011A808F017FF179A1AB102F1FF37FBB218
:100FC00001E04FF0060343F26006C2F20006F37040
:100FD000FBF7A8BE1D9A0F2A08D943F2CC04C2F22F
:100FE00000044FF02702227201F012B9824800EB90
:100FF000820143F26003C2F200031D7800F8225020
:101000005F784F701E798E70FBF78CBE11A8F0F7D9
:1010100025FF43F26000C2F200000178139143788B
:1010200012938578119511A8F0F77EFFFBF77ABE31
:101030000DF1700C219F97F85000F9F7FFF9FBF7BD
:1010400071BE43F2DC06C2F20006347814F0010FE0
:1010500008D143F2CC06C2F200064FF030043472DD
:1010600001F0D6B843F29002C2F20002106840B913
:1010700043F2CC01C2F200014FF031030B7201F0D8
:10108000C7B843F2DC01C2F200010B7803F0FE06A0
:1010900046F004040C7043F2A400C2F200004FF0CA
:1010A0000002026001F011B843F2DC00C2F200005D
:1010B000027812F0010F08D143F2CC00C2F2000016
:1010C0004FF03002027201F0A3B843F29001C2F275
:1010D00000010B6843B943F2CC06C2F200064FF0A0
:1010E0003404347201F094B843F2DC06C2F2000614
:1010F000347804F0FE0040F00202327043F2A401A2
:10110000C2F200014FF000030B6000F0DEBF219D32
:1011100095F846700DF1700CF9F7A8F921993B1A72
